:020000040800F2
:1080000000800120B96102083521020837210208E9
:10801000392102083B2102083D210208000000002E
:108020000000000000000000000000003F210208E6
:108030004121020800000000432102084DBF010851
:10804000FD610208FD610208FD610208FD61020890
:10805000FD610208FD610208C1E1010829E2010891
:10806000FD610208FD610208FD610208FD61020870
:10807000FD610208FD610208FD610208FD61020860
:10808000FD610208FD610208FD610208FD61020850
:10809000FD610208FD610208FD610208FD61020840
:1080A000FD610208FD610208FD610208FD61020830
:1080B00015ED0108FD610208FD610208FD6102087D
:1080C000FD610208FD610208FD610208FD61020810
:1080D000FD610208FD61020865D50108F5D10108BE
:1080E000FD610208FD610208FD610208FD610208F0
:1080F000FD610208FD610208FD610208FD610208E0
:10810000FD610208FD61020891E20108FD610208BB
:10811000FD610208FD610208FD610208FD610208BF
:10812000FD610208FD610208FD610208FD610208AF
:10813000FD610208FD610208FD610208FD6102089F
:10814000FD610208FD610208FD6102083BCB0108E8
:10815000FD610208FD610208FD61020875CF01089A
:10816000FD610208FD610208FD610208FD6102086F
:10817000FD610208FD610208FD610208FD6102085F
:04818000FD61020893
:1081880010B5054C237833B9044B13B10448AFF349
:1081980000800123237010BD600F00200000000044
:1081A800348B0208084B10B51BB108490848AFF3D7
:1081B80000800848036803B910BD074B002BFBD0AB
:1081C800BDE81040184700BF00000000640F002001
:1081D800348B0208600F002000000000000000003F
:1081E80010B516F07DF8064B00221A70054B1B6877
:1081F8009847BDE81040044B9B695B69184700BF6E
:10820800300A0020D400002028660208431E2DE909
:10821800F0471446052B00F22281DFE813F0060030
:108228000B000B004C007B00CC00FFF7D9FF47F692
:10823800A8536DE0924B934D02280EBF9946A9466C
:108248001D46914B4FF0FF36DF684FF000084FF0A6
:10825800010A3B68D9F800001B6998473B68286801
:10826800DB6898473B6828685B6998473B68D9F89A
:1082780000001B6A984718B90AFA08F326EA0306A9
:108288003B6828689B6998473B68D9F800001B6AD7
:10829800984718B10AFA08F326EA030608F1010814
:1082A800B8F1110F09F1040905F10405D1D1C6F39C
:1082B800100626601FE02160032900F2D380DFE862
:1082C80001F0021D2125704BDB691B68188880B2FC
:1082D8001DF08CF966A3D3E900231DF017FB66A3F4
:1082E800D3E900231DF0E8F90022684B1DF0E4F9FA
:1082F8001DF0F4FB20600020BDE8F087624BDB69CD
:108308005B68E3E7604BDB699B68DFE7604B1B69F1
:108318002360F0E70129216033D01CD3022940F003
:10832800A180594BDC686068236858309B6898477F
:10833800606823682030DB689847606823683C30B1
:10834800DB6898476068236820305B699847236832
:1083580060685B6980E04C4BDC68606823682030AB
:108368009B689847606823683C30DB68984760687A
:1083780023685830DB689847606823683C305B693D
:1083880014E0414BDC68606823683C309B68984780
:10839800606823682030DB68984760682368583035
:1083A800DB689847236860685B69203098472368D2
:1083B80060685B6938E00129216037D01BD3022946
:1083C80050D1314BDC686068236858309B68984707
:1083D800606823682030DB689847606823683C3011
:1083E800DB6898476068236820305B699847236892
:1083F80060689B6930E0244BDC6860682368203043
:108408009B689847606823683C30DB6898476068D9
:1084180023685830DB689847236860685B693C309C
:108428009847236860689B69583016E0164BDC68EB
:10843800606823683C309B689847606823682030F0
:10844800DB689847606823685830DB68984760683D
:10845800236820305B69E3E73C3098474BE704200A
:10846800BDE8F0870220BDE8F08700BFAFF30080C9
:108478000000000000FEAF40AAF1D24D6210144087
:10848800EC390020D4380020286602080000244077
:10849800300A002038B5064C05462368C31AB3F5E0
:1084A800FA7F04D3034B9B699B699847256038BDC5
:1084B8007C0F002028660208484B494ADB68596847
:1084C80001F5B870AC31106051605968E4319160C1
:1084D800596801F58E71D160596801F5AA71116169
:1084E800596801F5D4715161596801F5F0719161CC
:1084F800596801F50671D161596801F51471116265
:10850800596801F522715162596801F5307191621B
:10851800596801F53E71D162596801F54C711163D2
:10852800596801F55A715163596801F56871916389
:10853800596801F57671D163596801F58261116452
:108548005968284A01F174009031106051605968E7
:10855800C8319160596801F58071D160596801F599
:108568009C711161596801F5C6715161596801F52D
:10857800E2719161596801F5FE71D161596801F59F
:108588000D711162596801F51B715162596801F545
:1085980029719162596801F53771D162596801F5FD
:1085A80045711163596801F553715163596801F5B3
:1085B80061719163596801F56F71D1635B6803F567
:1085C8007D731364084B01221A70084B084A1A6518
:1085D800084A9A65084A5A6519F02ABC28660208AA
:1085E800D4380020EC390020300A00201839002047
:1085F80015820008E98100089D8400087047022060
:108608007047022070477047704702207047022069
:1086180070470220704701207047704770474369D0
:10862800114A10B5C3F80422C3F808220F4B1049A9
:108638008365104B104A836183620363C3610F4BE8
:108648000F4C43640F4B416283640F4B0F494363E4
:10865800C36303640E4B4265C16284630465C164ED
:10866800C265036610BD00BF1F86000805860008A6
:10867800078600080B860008258600080F86000874
:108688001B86000811860008178600081386000854
:1086980023860008704700BF0748084A0023C267BE
:1086A800137053704FF0FF3280F8783043670267D9
:1086B800C3666830FFF7B3BF183900208C0F00205D
:1086C8000648074A00234261137053704FF0FF3287
:1086D8000374C36082604360FFF7A1BF18390020AC
:1086E800A41100200023184610B5064C1A5D590045
:1086F80002F0030201338A40072B40EA0200F5D159
:1087080010BD00BFBC130020044900235A5C02F0CE
:108718000302C2540133072BF8D17047BC13002061
:10872800074B1A7802705A7842709A788270DA7811
:10873800C2701A7902715A7942719B7983717047B4
:10874800BC130020F8B5094B094F0A4DDE68002418
:10875800E15D33686A6CDB6952F8240001F00301BB
:1087680001349847072CF3D1F8BD00BF28660208EA
:10877800BC13002000000020054A002300F003017C
:1087880099540133072B4FEA9000F7D1DAE700BF7D
:10879800BC130020014B586AEEE700BF0000002020
:1087A80004490023C25C02F003025A540133072B28
:1087B800F8D1C7E7BC1300200278074B1A7042783B
:1087C8005A7082789A70C278DA7002791A7142798E
:1087D8005A7182799A71B5E7BC130020074B1A6861
:1087E800821AB2F57A7F04D39A6818605A60002218
:1087F8009A609A6801329A60704700BFD0130020CF
:108808000020704701207047014B00225A607047D2
:108818001839002010B50C4613F024FF206010BD55
:1088280013F04CBF022804BF0B4B93F8D00020B9BB
:108838000A4BDB681B689B690AE001280BD1064BD1
:1088480093F8D030012B06D1044BDB681B685B69B9
:10885800034A10681847704718390020286602082C
:10886800343A002010B50020FFF7DCFFBDE81040C7
:10887800034B044ADB6810681B689B68184700BFF5
:1088880028660208343A00204B2938B504461546B4
:1088980000F0D78256D83B2900F0C9812ED82E295E
:1088A80000F04B8113D82A2900F0DF8009D8282945
:1088B80000F0A58000F2BE80272900F0928000F029
:1088C80016BC2C2900F0038140F2E6801AE1332916
:1088D80000F0798109D8302900F05A81C0F045812B
:1088E800312900F05E8100F002BC392900F0858151
:1088F80000F28D81342900F06F81F8E3432900F0FC
:108908002A820FD83F2900F0DE8105D83D2900F0E2
:10891800B48140F29F81C3E1412900F0F88140F21F
:10892800E48106E2472900F05F8205D8452900F076
:10893800368240F2228244E2492900F0788240F2ED
:1089480066822EE15B2900F0368323D8532900F094
:10895800C0820FD84F2900F0948205D84D2900F025
:108968007A8240F2158181E2512900F09E8240F21C
:108978009282A4E2572900F0DE8205D8552900F03A
:10898800BA8240F2AF82C6E2592900F0F48240F27E
:10899800E28200E3632900F064830FD85F2900F0C6
:1089A8003C8305D85D2900F0268340F214832BE32D
:1089B800612900F0448340F2398349E3672900F0D4
:1089C800748305D8652900F05E8340F2538363E31E
:1089D800692900F07C83C0F07183FF2900F080834F
:1089E80085E338B90146142013F0C7FE00B22860A9
:1089F800204638BD012C14BF0020042038BD38B9EA
:108A0800112013F02FFEC0F302402860002038BD6B
:108A1800012840F06E83112013F024FE2B6820F407
:108A2800E0211B0403F4E0231943112013F046FE50
:108A3800002038BD38B9112013F014FEC0F3C4402B
:108A48002860204638BD012840F05583112013F0D6
:108A580009FE2B6820F47801DB0403F4780319433A
:108A6800112013F02BFE002038BD30B9112013F06F
:108A7800F9FD80B22860204638BD012840F03D83CA
:108A8800112013F0EFFD2988000C00040143112088
:108A980013F014FE002038BD38B9112013F0E2FDA0
:108AA800C0F302602860204638BD012840F02783C3
:108AB800112013F0D7FD2B6820F0E0611B0603F0AE
:108AC800E0631943112013F0F9FD002038BD38B9CF
:108AD800112013F0C7FDC0F3C2602860002038BD24
:108AE800012840F00E83112013F0BCFD2B6820F004
:108AF8006051DB0603F060531943112013F0DEFDCB
:108B0800002038BD38B9112013F0ACFDC0F38070D7
:108B18002860204638BD012840F0F582112013F066
:108B2800A1FD2B6820F080419B0703F08043194387
:108B3800112013F0C3FD002038BD30B9112013F007
:108B480091FDC00F2860204638BD012840F0DD8225
:108B5800112013F087FD296820F0004040EAC17118
:108B6800112013F0ABFD002038BD38B901461220A2
:108B780013F003FE00B22860204638BD012C40F0F7
:108B8800C6822A880021122013F029FE002038BD51
:108B9800002C7FF42FAF152013F064FD286000200F
:108BA80038BD34B90021132013F0E7FD28600020F8
:108BB80038BD012C40F0AD822A880021132013F023
:108BC8000EFE002038BD00287FF414AF014613F0D4
:108BD800D4FD2860204638BD30B90146012013F085
:108BE800CCFD2860204638BD012840F094821288C8
:108BF800002113F0F4FD002038BD00287FF4FAAE00
:108C08000021022013F0B9FD2860002038BD28B9E2
:108C1800032013F027FD2860204638BD012840F0C6
:108C28007C821168032013F049FD002038BD38B953
:108C38000146042013F0A1FD00B22860204638BD8B
:108C4800012840F06C8212880021042013F0C7FD2F
:108C5800002038BD38B90146052013F08EFD00B25A
:108C68002860204638BD012840F05B821288002128
:108C7800052013F0B4FD002038BD38B900210620C6
:108C880013F07BFD00B22860002038BD012840F0B9
:108C98004A8212880021062013F0A1FD002038BD69
:108CA80038B90146072013F068FD00B22860204655
:108CB80038BD012840F0398212880021072013F0BE
:108CC8008EFD002038BD30B90146082013F055FD4F
:108CD8002860204638BD012840F0298212880021EA
:108CE800082013F07CFD002038BD30B9014609206A
:108CF80013F043FD2860204638BD012840F0198252
:108D080012880021092013F06AFD002038BD30B90F
:108D180000210A2013F031FD2860002038BD012809
:108D280040F00982128800210A2013F058FD002023
:108D380038BD30B901460B2013F01FFD28602046CE
:108D480038BD012840F0F981128800210B2013F06A
:108D580046FD002038BD30B901460C2013F00DFD4A
:108D68002860204638BD012840F0E981128800219A
:108D78000C2013F034FD002038BD30B901460D2019
:108D880013F0FBFC2860204638BD012840F0D9814B
:108D9800128800210D2013F022FD002038BD30B9C3
:108DA80000210E2013F0E9FC2860002038BD0128BE
:108DB80040F0C981128800210E2013F010FD002018
:108DC80038BD38B901460F2013F0D7FC00B228602F
:108DD800204638BD012840F0B881128800210F20B4
:108DE80013F0FDFC002038BD38B90146102013F0FF
:108DF800C4FC00B22860204638BD012840F0A78195
:108E080012880021102013F0EAFC002038BD28B990
:108E1800112013F027FC2860204638BD012840F0B7
:108E280098811168112013F049FC002038BD0028F2
:108E38007FF4A4AE0021122013F09FFC28600020CC
:108E480038BD00287FF4D6AD0146142013F095FCF8
:108E58002860204638BD00287FF4CCAD00212020B2
:108E680013F08BFC00B22860002038BD00287FF486
:108E7800C1AD0146212013F080FC00B228602046D5
:108E880038BD00287FF4B6AD0146222013F075FCEA
:108E98002860204638BD00287FF4ACAD0146232069
:108EA80013F06BFC2860204638BD00287FF4A2AD83
:108EB8000021242013F061FC2860002038BD002820
:108EC8007FF498AD0146252013F057FC2860204612
:108ED80038BD00287FF48EAD262013F0C3FB286030
:108EE800204638BD00287FF485AD272013F0BAFB53
:108EF8002860204638BD28B9302013F0B3FB28601D
:108F0800002038BD012840F026811168302013F078
:108F1800D5FB002038BD28B9312013F0A3FB286009
:108F2800204638BD012840F018811168312013F01F
:108F3800C5FB002038BD28B9322013F093FB286008
:108F4800204638BD012840F00A811168322013F00C
:108F5800B5FB002038BD28B9332013F083FB286007
:108F6800204638BD012840F0FC801168332013F0FA
:108F7800A5FB002038BD28B9342013F073FB286006
:108F8800002038BD012840F0EE801168342013F02D
:108F980095FB002038BD28B9352013F063FB286005
:108FA800204638BD012840F0E0801168352013F0D4
:108FB80085FB002038BD28B9362013F053FB286004
:108FC800204638BD012840F0D2801168362013F0C1
:108FD80075FB002038BD28B9372013F043FB286003
:108FE800204638BD012840F0C4801168372013F0AE
:108FF80065FB002038BD00287FF4FCAC382013F056
:1090080031FB2860002038BD00287FF4F3AC3920FC
:1090180013F028FB2860204638BD00287FF4EAAC0E
:109028003A2013F01FFB2860204638BD00287FF443
:10903800E1AC3B2013F016FB2860204638BD002821
:109048007FF4D8AC3C2013F00DFB2860002038BD1D
:1090580000287FF4CFAC3D2013F004FB28602046A5
:1090680038BD00287FF4C6AC3E2013F0FBFA286018
:10907800204638BD00287FF4BDAC3F2013F0F2FA3B
:109088002860204638BD00287FF4B4AC762013F061
:10909800E9FA2860002038BD00287FF4ABAC7720BF
:1090A80013F0E0FA2860204638BD00287FF4A2AC0F
:1090B8007C2013F0D7FA2860204638BD00287FF4BA
:1090C80099AC7D2013F0CEFA2860204638BD0028E0
:1090D8007FF490AC7E2013F0C5FA2860002038BDDC
:1090E80000287FF487AC244B5B68136038BD0420EC
:1090F80038BD002038BD002038BD002038BD002014
:1091080038BD002038BD002038BD002038BD002003
:1091180038BD002038BD002038BD002038BD0020F3
:1091280038BD002038BD002038BD002038BD0020E3
:1091380038BD002038BD002038BD002038BD0020D3
:1091480038BD002038BD002038BD002038BD0020C3
:1091580038BD002038BD002038BD002038BD0020B3
:1091680038BD002038BD002038BD002038BD0020A3
:1091780038BD002038BD00BFD01300200B4619B9F8
:1091880001461846FFF780BB08207047012070474A
:1091980007B5019229B9014601AA0120FFF774FB1E
:1091A80000E0082003B05DF804FB084613F05ABA43
:1091B8000846114613F082BA13F0DFBA13F00FBB5A
:1091C80038B51B4B1B4DDC6860682368C8302860C5
:1091D800DB689847236828685B699847164B1749E6
:1091E8005A6901200A6016491070C2F8041215491C
:1091F800C2F8081200215170134A18749A63134A6E
:109208005A63134A9A64134A5A64134A5A65134AAA
:109218001A65134A1A66134ADA65134A9A6532229E
:10922800DA604FF48C729A60BDE83840FFF7FABAFA
:1092380028660208343A002018390020303A002005
:10924800959100080D8800088591000899910008FB
:10925800298800081D880008E58700080988000893
:109268002D880008118800086D880008014B00222D
:10927800DA6670471839002070B50446074E084D65
:1092880033682A460146002016F093F833682A46C8
:109298002146BDE87040012016F08BB8243D00201F
:1092A800383A0020014B186816F0CDB8243D00204C
:1092B80010B5104C23681868C8B963681B68BBB937
:1092C8000D4B186816F0B6F8022015F087FE0B4B08
:1092D8000B4918680A6850629868226090624A6868
:1092E8005968DB68626051629362012010BD0020FA
:1092F80010BD00BF80000020243D0020E81300209E
:10930800640A0020012805D820B9034B1B681B6894
:109318000B60704708207047640A0020012810B5C8
:10932800144608D0022813D10A4B0B4ADB68506A4E
:109338001B681B6A05E0074B074ADB68106A1B6855
:109348001B6A9847003018BF01202060002010BD1C
:10935800042010BD28660208E8130020022804BF74
:109368000B4B93F8D00020B90A4BDB681B685B698C
:109378000AE001280BD1064B93F8D030012B06D117
:10938800044BDB681B689B69034A106918477047E0
:109398001839002028660208E813002070B500205C
:1093A800FFF7DCFF0A4B0B4CDD6820692B689B68D4
:1093B80098472B68206A9B6898472B68606A9B6867
:1093C800984715F06DFEBDE87040034B5B68184781
:1093D80028660208E8130020B80900202DE9F843A0
:1093E8000F4691469846174C0021236847F08000A5
:1093F8009B689DF820609DF82450984723680021B9
:109408009B6848469847236800219B6840469847D0
:10941800236800219B6830469847236828469B6844
:1094280001219847084B48EA09281B6846EA08269C
:1094380007F07F0703EB870745EA06257D60BDE84F
:10944800F88300BF283D0020243D002007B5D3B293
:109458000193C2F307230093C2F30743120EFFF7E9
:10946800BDFF03B05DF804FB0A4601460020FFF784
:10947800EDBF38B5234B01F07F04234493F8143231
:10948800DB0705D4204B1B6803EB8404606838BDF8
:109498001E4D00212B6820469B6898472B680021A9
:1094A8009B68084698472B6800219B6808469847A0
:1094B8002B6800219B68084698472B6801219B6808
:1094C800002098472B6800219B68204698472B6806
:1094D80000219B68084698472B68002104029B6876
:1094E800084698472B680021204304029B680846D9
:1094F80098472B68204304029B6801210020984765
:10950800204338BD383A0020243D0020283D002063
:1095180010B50C4601460020FFF7ABFF206010BDD8
:10952800012838B504460D4618D80021FFF7A1FFD9
:10953800002140F006022046FFF788FF084B002074
:1095480053F82430187683F84C009A685A645A6C99
:109558001A6101229D6483F84C2038BD082038BD6B
:1095680080000020012838B504460D4611D8002196
:10957800FFF77FFF002140F006022046FFF766FF55
:10958800054B002053F824301D61187683F84C00F1
:1095980038BD082038BD00BF80000020012808D849
:1095A800054A52F820309A680B6813440B60194634
:1095B800D8E70820704700BF80000020A32A2DE9C3
:1095C800F04104460D461E4600F0C8812DD8072AF2
:1095D80000F0D9800DD8032A00F0868003D8012A2C
:1095E80064D055D971E0052A00F09F8040F28B8045
:1095F800AAE0182A00F0088108D8162A00F0E880A6
:1096080000F2F480082A00F0DC80B6E31D2A00F09E
:109618002D8103D81C2A00F00B81AEE38C2A00F0C0
:109628002C81A22A00F07781A7E3AC2A00F0C88237
:1096380015D8A72A00F03F8205D8A52A00F0CA81CC
:1096480040F2AA8103E2A92A00F06082C0F04182B8
:10965800AA2A00F07982AB2A00F094828DE3B42A1A
:1096680000F02C8308D8AE2A00F0E582C0F0C5824D
:10967800B32A00F0068380E3B62A00F0A980C0F080
:109688002A83B82A00F04783CE2A00F0688374E35F
:1096980020B9B04B53F821301B69DFE2012801BF24
:1096A800AC4B326853F821301A6155E320B9A94B05
:1096B80053F821309B68D1E2012840F04D83A54B37
:1096C800326853F821309A6046E320B9A14B53F829
:1096D8002130DB68C2E2012840F03E839D4B3268AE
:1096E80053F82130DA6037E348B99A4B53F8213000
:1096F8001A6812F4000318BF4FF07F43ADE2012C43
:1097080000F03B8328E320B9924B53F821305B6982
:10971800A4E2012840F020838E4B53F821203368BF
:10972800002BB8BF5B42536116E320B9894B53F84D
:1097380021305B6892E2012840F00E83854B326845
:1097480053F821305A6007E350B92021A94041F06D
:109758001001C9B22846FFF78CFEC0F304200AE3C3
:10976800012840F0F98220248C4044F01004E4B22F
:1097780021462846FFF77DFE336820F4F8521B0285
:1097880003F4F853E3E250B92021A94041F0100155
:10979800C9B22846FFF76DFE00F01F00EBE2012872
:1097A80040F0DA8220248C4044F01004E4B22146D0
:1097B8002846FFF75EFE336820F01F0203F01F0300
:1097C800C5E200289BD1634B53F821305B7E45E20C
:1097D80024B92021A94041F011011AE0012C40F0E0
:1097E800BB822021A94041F011011EE020B92021AF
:1097F800A94041F012010CE0012840F0AD8220217F
:10980800A94041F0120110E040B92021A94041F0DF
:109818001301C9B22846FFF72CFEACE2012840F03C
:109828009B822021A94041F013013268C9B290E21D
:1098380050B9090141F06C0101F0FC012846FFF71D
:1098480018FEC0F3804096E2012840F085820C01A2
:1098580044F06C04E4B221462846FFF70AFE336858
:1098680020F480229B0403F4802370E200287FF414
:1098780046AF394B1B681B68F0E150B9090141F04C
:109888006C0101F0FC012846FFF7F3FDC0F303600B
:1098980071E2012840F060821B68102B1FD00CDC9D
:1098A800022B18D003DC012B1FD108231FE0042B47
:1098B80013D0082B19D1052319E0402B11D003DC54
:1098C800202B12D1032312E0802B0CD0B3F5807F1C
:1098D8000BD100230BE0072309E0062307E004234C
:1098E80005E0022303E0306002E04FF0FF3333600D
:1098F8003368013300F030822C0144F06C04E4B288
:1099080021462846FFF7B5FD336820F070621B0634
:1099180003F070631BE250B9090141F06C0101F0DA
:10992800FC012846FFF7A5FDC0F3C13023E201285A
:1099380040F012820C0144F06C04E4B2214628463F
:10994800FFF797FD336820F4C032DB0303F4C0331C
:10995800FDE100BF80000020640A002050B9090121
:1099680041F06C0101F0FC012846FFF782FDC0F3CD
:10997800803000E2012840F0EF810C0144F06C04D3
:10998800E4B221462846FFF774FD336820F480428C
:109998009B0303F48043DAE150B9090141F06C01FB
:1099A80001F0FC012846FFF764FDC0F30030E2E156
:1099B800012840F0D1810C0144F06C04E4B2214646
:1099C8002846FFF756FD336820F480521B0303F442
:1099D8008053BCE10F0147F06C07FFB239462846B7
:1099E800FFF747FD804674B918F4804F394628467A
:1099F80040D1FFF73EFD18F4006FC0F3021018BF06
:109A080040F00800B7E1012C40F0A68118F4804826
:109A18003946284644D1FFF72CFD326820F0700003
:109A2800120102F07002024339462846FFF70EFD84
:109A380039462846FFF71DFD336820F4006213F00D
:109A4800080F18BF4FF4006842EA080231E00F011E
:109A580047F06C07FFB239462846FFF70AFD74B98C
:109A680010F4804F3946284604D0FFF702FDC0F3B2
:109A7800021080E1FFF7FDFCC0F3C3107BE1012C6D
:109A880040F06A8110F480443946284608D0FFF730
:109A9800F0FC336820F070021B0103F0700307E04C
:109AA800FFF7E7FC336820F4F062DB0103F4F063AE
:109AB8001A4339464DE128B9090141F06C0101F01A
:109AC800FC0183E0012840F047810C0144F06C045C
:109AD80088E050B9090141F06D0101F0FD01284607
:109AE800FFF7C7FCC0F3C03045E1012840F03481DE
:109AF8000C0144F06D04E4B221462846FFF7B9FC96
:109B0800336820F40042DB039BB220E150B909011D
:109B180041F06D0101F0FD012846FFF7AAFCC0F3F2
:109B2800413028E1012840F017810C0144F06D0410
:109B3800E4B221462846FFF79CFC336820F4C04273
:109B48005B0303F4C04302E150B9090141F06D0120
:109B580001F0FD012846FFF78CFCC0F303200AE161
:109B6800012840F0F9800C0144F06D04E4B221466C
:109B78002846FFF77EFC336820F470621B0203F46A
:109B88007063E4E050B9090141F06D0101F0FD0195
:109B98002846FFF76EFCC0F34110ECE0012840F0C6
:109BA800DB800C0144F06D04E4B221462846FFF73F
:109BB80060FC336820F060025B0103F06003C6E0DC
:109BC80050B9090141F06D0101F0FD012846FFF788
:109BD80050FC00F00F00CEE0012840F0BD800C01E1
:109BE80044F06D04E4B221462846FFF742FC33688E
:109BF80020F00F0203F00F03A9E050B9090141F06A
:109C08006D0101F0FD012846FFF733FCC0F3006049
:109C1800B1E0012840F0A0800C0144F06D04E4B2EA
:109C280021462846FFF725FC336820F080721B0682
:109C380003F080738BE098B9090141F06D0101F0E0
:109C4800FD012846FFF715FC001410F0400F00F046
:109C58007F0214BF6FF0FF030023134333607BE0E0
:109C6800012879D10C0144F06D04E4B2214628465C
:109C7800FFF7FFFB336820F4FE021B0403F4FE0326
:109C880065E050B9090141F06C0101F0FC0128467A
:109C9800FFF7EFFBC0F340406DE001285CD10C01F9
:109CA80044F06C04E4B221462846FFF7E2FB33682F
:109CB80020F400325B0403F4003348E000287FF40A
:109CC8001EAD090141F06F01C9B22846FFF7D1FB6B
:109CD800C0F304404FE020B9294B53F82130DB6929
:109CE800BCE7012838D120248C4064B244F011012B
:109CF80044F014041A68C9B22846E4B2FFF7A6FB78
:109D080021462846FFF7B5FB336820F480629B02A2
:109D180003F480631BE050B9090141F06C0101F0C4
:109D2800FC012846FFF7A5FBC0F3403023E00128DB
:109D380012D10C0144F06C04E4B221462846FFF726
:109D480098FB336820F400525B0303F40053214668
:109D58001A432846FFF77AFB0020BDE8F081002867
:109D68007FF4CDAC090141F06F01C9B22846FFF775
:109D780080FBC0F309003060EEE70420BDE8F08105
:109D88008000002007B50129019205D8024601ABE1
:109D98000120FFF713FC00E0082003B05DF804FB86
:109DA8000129134602D80246002007E4082070471C
:109DB800012838B504460D4610D80021FFF759FB95
:109DC800002140F006022046FFF740FB044B012229
:109DD80053F8243000201A76DD6038BD082038BDDD
:109DE800800000200021E3E74942E1E7E0E770B5A1
:109DF800554E564815F09EFAF568554C6B6803F1B8
:109E0800C802226103F59C72626203F5AA7222629B
:109E180003F5C672A26003F5D47203F5B8706260E8
:109E280003F5E27203F50D73A3622B68E260DB6849
:109E3800206098472B68A068DB6898472B686068A3
:109E4800DB6898472B68E068DB6898472B682069CF
:109E5800DB6898472B68A06ADB68984733693D4AF6
:109E680003F110011160A26A02205A613A4A3B4B81
:109E78003B4D1A6015F0B2F83A4920680B683A4A27
:109E88005862A068136098624B68384953606268EA
:109E980002205A62E26800249A62354BDA6FC2F8EF
:109EA800041234495470C2F8081201211170324A60
:109EB800C3F88820314AC3F88420314AC3F8802087
:109EC800304AC3F88C20304AC3F8A0202F4AC3F880
:109ED8009C202F4AC3F890202E4AC3F894202E4A7B
:109EE800C3F898202D4AC3F8B0202D4AC3F8AC20F7
:109EF8002C4AC3F8BC202C4AC3F8B8202B4AC3F814
:109F0800B4202B4AC3F8C8202A4AC3F8C4203222F6
:109F18005A674FF48C721A67274A83F87800C3F897
:109F2800C020FFF71BFA2B689847AB682046984774
:109F380021462046FFF79DFA214640F006022046BA
:109F4800BDE87040FFF782BA28660208383A002058
:109F5800E8130020283D00208C0F0020243D00201D
:109F6800B8090020640A002080000020B992000887
:109F780018390020AD920008B99D0008F59D000829
:109F8800F19D0008ED9D0008A99D00088D9D000821
:109F98006D950008A595000829950008719400089A
:109FA8001995000881920008259300080D93000870
:109FB8006593000875920008A593000828B9044B1A
:109FC80001221B681A76D96070470820704700BFC5
:109FD80088000020F2E74942F0E70021EEE730B9B7
:109FE800044B1B681961187683F84C0070470820E9
:109FF800704700BF88000020014B0846DB6B1847FC
:10A0080000000020034B10B51B6C0C4698472060DD
:10A0180010BD00BF0000002007B5034B68461B6B4E
:10A02800984703B05DF804FB0000002070B50020DD
:10A03800FFF7F2FF1E4B1F4CDD68206B2B689B68F7
:10A0480098472B68E06A9B6898472B68E0689B688C
:10A0580098472B68A0689B6898472B6860689B683E
:10A0680098472B6820689B6898472B68A0699B686D
:10A0780098472B68E0699B6898472B68A06A9B689B
:10A0880098472B6860699B6898472B68206A9B688B
:10A0980098472B68606A9B6898472B6820699B687B
:10A0A800984714F0FDFFBDE87040034B5B68184704
:10A0B8002866020820140020B809002038B9054B8A
:10A0C8001B689A680B6813440B60194687E70820D9
:10A0D800704700BF88000020062873B505460C4667
:10A0E8005CD8022903D901285AD10F2958DC2E4EF1
:10A0F8006846336B98473346052D4AD8DFE805F0A4
:10A1080003063E4144478DF8004042E0082C40D801
:10A11800DFE804F0050A11161B20252A2F00F27823
:10A128008DF80120327B03E032798DF80120727BB3
:10A138008DF802202DE072798DF80120B27BF7E7C7
:10A14800B2798DF80120F27BF2E7F2798DF80120DF
:10A15800327CEDE7727A8DF80120B27CE8E7B27ABA
:10A168008DF80120F27CE3E7327A8DF80120727CC9
:10A17800DEE7F27A8DF80120327DD9E78DF80340C9
:10A1880007E08DF8044004E08DF8054001E08DF803
:10A1980006406846DB6A9847002002E0042000E099
:10A1A800102002B070BD00BF0000002073B5054646
:10A1B800434E6846336B0C4698473346062D7AD88B
:10A1C800DFE805F076046A6D707376009DF801206B
:10A1D800F178914208D13A499DF80200097B8842FA
:10A1E80002D10020206069E01979914207D13449F1
:10A1F8009DF80200497B884201D101235AE0597930
:10A20800914207D12E499DF80200897B884201D1ED
:10A2180002234FE09979914207D129499DF802001C
:10A22800C97B884201D1032344E0D979914207D1FF
:10A2380023499DF80200097C884201D1042339E0B2
:10A24800597A914207D11E499DF80200897C8842BB
:10A2580001D105232EE0997A914207D118499DF83A
:10A268000200C97C884201D1062323E0197A914271
:10A2780007D113499DF80200497C884201D1072380
:10A2880018E0DB7A934218D10D4B9DF802201B7D14
:10A298009A4212D108230DE09DF803300AE09DF898
:10A2A800043007E09DF8053004E09DF8063001E031
:10A2B8009DF800302360002000E0102002B070BD3F
:10A2C8000000002030B585B001920C4600295CD111
:10A2D8000B2814D8062836D2022829D007D818B354
:10A2E800012854D12B4B1B689A601A614BE0042853
:10A2F80022D005284BD1274B1B685A6043E013280E
:10A3080006D80E2839D20C281FD00D282CD03EE0B4
:10A318008C283CD101A90120FFF748FF1E4B0446B9
:10A328009B6B02A898472EE01A4B1B681A612FE016
:10A33800184B1B68DA6026E0164B002A1B68B8BF6A
:10A3480052425A611FE0063818E01546134A144B6A
:10A35800D26812681DB15269D86A904713E0D86A6A
:10A3680092699047284613E042F210739A420ED839
:10A378000C4B90B29B68984705E00E381146C0B266
:10A38800FFF7AAFE04E0204602E0082000E00420CF
:10A3980005B030BD880000200000002028660208B3
:10A3A80020140020B809002010B51446002946D111
:10A3B800132846D8DFE800F00A0E12161A1E2222C9
:10A3C8002222222229303C3C3C3C3C3C1E4B1B6850
:10A3D8001B6918E01C4B1B689B6814E01A4B1B6830
:10A3E800DB6810E0184B1B681B680CE0164B1B68F9
:10A3F8005B6908E0144B1B685B6804E0082820D1FF
:10A40800114B1B685B7E236017E0104B104ADB681A
:10A41800D06A1B681B6A05E00C4B0D4ADB68106BA1
:10A428001B681B6A9847003018BF0120206004E0B1
:10A438000E381146C0B2FFF7B9FE002010BD082043
:10A4480010BD042010BD00BF880000202866020847
:10A4580020140020604B2DE9F041DF685F4C7868DC
:10A46800002500F5FE73236300F5F073E36200F541
:10A478002973E36000F53073A36000F5227363600D
:10A4880000F50D73236000F55A73A36100F553734B
:10A49800E36100F1C803A36200F5C673636100F5C8
:10A4A8006873236200F56F7363623B6800F5B870E8
:10A4B800DB68206198473B686069DB6898473B68C0
:10A4C800206BDB6898473B68E06ADB6898473B6825
:10A4D800206A1B6998473B68606A1B699847404B2C
:10A4E800E1681E465A6C11605A6CA16851605A6C3A
:10A4F800616891605A6C2168D1605A6CA1691161D8
:10A508005A6CE16951615A6CA16A9161726C3B683D
:10A518005059DB689847726C3B6850599B69043501
:10A5280098471C2DF2D12F4D0022EB6F01201A7095
:10A5380014F054FD2C4B22695B68DFF8E8805A62FE
:10A548006269C8F800309A62284B0220C5F8883042
:10A55800274BC5F88430274BC5F88030264BC5F803
:10A568008C30264BC5F8A030254BC5F89C30254BC0
:10A57800C5F89030244BC5F89430244BC5F8B0305A
:10A58800234BC5F8AC30234BC5F8C830012385F8F8
:10A598007830214BC5F8C030FFF73EFDD8F80030C1
:10A5A8001B6813B11D4B9B780BB1B36A9847236B9B
:10A5B8000222197C5A741868012217F0A5FD3B681D
:10A5C800206B174C1B68984723689847A36800209E
:10A5D800BDE8F041184700BF286602082014002093
:10A5E8000000002018390020640A0020C59F0008D8
:10A5F800DD9F0008DF9F0008E39F0008B1A3000863
:10A60800CDA20008E79F0008C5A0000801A0000827
:10A618000DA0000821A0000835A00008300A00207D
:10A62800B80900208800002028B9044B01221B68C3
:10A638001A76D96070470820704700BF8C00002048
:10A64800F2E74942F0E70021EEE730B9044B1B6816
:10A658001961187683F84C0070470820704700BFCE
:10A668008C00002010B5042804D8DFE800F005238A
:10A6780021333F00042010BD44F6206314689C4237
:10A688006AD842F21071354B354ADB688C421B6838
:10A69800106ADB6994BF00210121984742F21170CA
:10A6A800B4FBF0F300FB13402E4B80B29B68984735
:10A6B800002010BD294B1468DB6858681B6824B15A
:10A6C800DB69002100F506700EE09B6800F5067056
:10A6D8009847EDE7214B1168DB68214A1B68003178
:10A6E800DB69106918BF01219847E1E71468002069
:10A6F8001D4B032C20D8DFE804F002070E1553F891
:10A70800213083F84C00D3E7184A53F821301268F7
:10A7180092685A64CCE7154A53F821301268926857
:10A728009A64C5E753F82130012283F84C205A6C0B
:10A7380000201A61187610BD53F821300B4983F8B0
:10A748004C0009688968596412689A645A6C1A61DD
:10A75800012283F84C20ABE7102010BD28660208C0
:10A7680060140020B80900208C000020640A002032
:10A778001B4B70B5DD681B4C2B68A0685B6998475C
:10A788002B6820689B6898472B6860689B68984787
:10A798002B68206A9B6898472B68606A9B68984773
:10A7A8002B68E0689B6898472B6820699B689847E6
:10A7B8002B6860699B6898472B68A0699B689847D5
:10A7C8002B68E0699B6898472B68A0689B68984746
:10A7D80014F066FCBDE87040034B5B68184700BF87
:10A7E8002866020860140020B8090020014B186888
:10A7F80014F076BEB03F00200C4B10B51A681C460A
:10A80800126812B10A4B987878B10A4B186814F09C
:10A818005EFE012014F0E2FB074A084B11681B6832
:10A828005268236059629A62012010BD8C00002092
:10A83800300A0020B03F002060140020640A002085
:10A8480038B9054B1B689A680B6813440B601946A6
:10A85800FBE60820704700BF8C00002078B9094B40
:10A86800094A1B681268187683F84C0092685A6483
:10A878005A6C1A610122996483F84C2070470820A9
:10A88800704700BF8C000020640A002020B9034BE9
:10A898001B681B680B60704708207047640A00201B
:10A8A800022804BF0B4B93F8D00020B90A4BDB6891
:10A8B8001B685B690AE001280BD1064B93F8D0307E
:10A8C800012B06D1044BDB681B689B69034A90681F
:10A8D80018477047183900202866020860140020BD
:10A8E8002DE9F04788460446924699461A4D0021BC
:10A8F80055F8203048F080009B689DF820709DF83E
:10A908002460984755F8243000219B6850469847A2
:10A9180055F8243000219B684846984755F824305C
:10A9280000219B683846984755F8243030469B6884
:10A9380001219847094B49EA0A2953F8243047EA84
:10A94800092708F07F0803EB880846EA0726C8F8B5
:10A958000460BDE8F08700BFB43F0020B03F00208E
:10A9680007B5D3B20193C2F307230093C2F3074399
:10A97800120EFFF7B5FF03B05DF804FB0A46014667
:10A988000020FFF7EDBF2C4A4FF4217370B503FB8D
:10A99800002301F07F04234493F804320546DB07C3
:10A9A80006D4264B53F8203003EB8404606870BD4E
:10A9B800234E002156F8203020469B68984756F8C9
:10A9C800253000219B680846984756F82530002115
:10A9D8009B680846984756F8253000219B6808462A
:10A9E800984756F8253001219B680020984756F86B
:10A9F800253000219B682046984756F825300021CD
:10AA08009B680846984756F82530002104029B6841
:10AA18000846984756F825300021204304029B68D1
:10AA28000846984756F82530204304029B680121C0
:10AA380000209847204370BD2C3D0020B03F0020E7
:10AA4800B43F002038B5104B104C1B68104A014623
:10AA5800002014F035FD236893F8302002F0FF053C
:10AA680082B993F840306BB16F212846FFF78BFF0E
:10AA78006F212846FFF787FFC30142BF23680122E1
:10AA880083F8302038BD00BFB03F0020640A0020A2
:10AA98002C3D002010B50C4601460020FFF773FF3F
:10AAA800206010BDA62AF8B504460D461E4600F0E3
:10AAB8006A8251D8172A00F0308124D8042A00F07D
:10AAC800CE800CD8012A00F0A280C0F09280022A21
:10AAD80000F0AD80032A00F0B98000F064BC072ABA
:10AAE80000F0F48007D8052A00F0CB80062A00F091
:10AAF800D78000F058BC082A00F0FF80152A00F023
:10AB0800038100F050BC1D2A00F0658110D81A2A74
:10AB180000F0248104D8182A00F0148100F043BC06
:10AB28001B2A00F02C811C2A00F03F8100F03BBC5E
:10AB3800A32A00F0B78107D88C2A00F05381A22AF3
:10AB480000F09A8100F02FBCA42A00F0C781A52A42
:10AB580000F0DA8100F027BCB52A00F0268323D85C
:10AB6800AB2A00F0A1820CD8A82A00F05C82C0F0C1
:10AB78004A82A92A00F06C82AA2A00F07F8200F09B
:10AB880012BCAE2A00F0D18207D8AC2A00F0A2820B
:10AB9800AD2A00F0B48200F006BCB32A00F0E582CA
:10ABA800B42A00F0F882FEE3BB2A00F06E830ED8C8
:10ABB800B82A00F0228303D8B62A00F00B83F2E308
:10ABC800B92A00F02A83BA2A00F03783EBE3C02AB7
:10ABD80000F0AB8306D8BC2A00F07D83BF2A00F0C2
:10ABE8008C83E0E3CC2A00F0B883CE2A00F0D0832F
:10ABF800D9E320B9AF4B53F821301B69DAE20128B9
:10AC080040F0C483AB4B326853F821300DE020B9D3
:10AC1800A84B53F821309B68CCE2012840F0B6835A
:10AC2800A44B326853F821309A601A61AEE320B918
:10AC3800A04B53F82130DB68BCE2012840F0A68322
:10AC48009C4B326853F82130DA609FE318B9994B6E
:10AC580053F82130C4E0012C00F0A58396E320B915
:10AC6800944B53F821305B69A4E2012840F08E83AD
:10AC7800904B53F821203368002BB8BF5B425361D7
:10AC880084E320B98B4B53F821305B6892E20128AA
:10AC980040F07C83874B326853F821305A6075E363
:10ACA80030B910212846FFF76EFEC0F3042078E380
:10ACB800012840F06B8310212846FFF764FE3368B3
:10ACC80020F4F8521B0203F4F85313E030B91021B2
:10ACD8002846FFF758FE00F01F0062E3012840F005
:10ACE800558310212846FFF74EFE336820F01F02D7
:10ACF80003F01F031A43102145E30028ABD16D4B25
:10AD080053F821305B7E55E2002800F04C8301287F
:10AD180040F03C831A68112135E308B915218EE209
:10AD2800012840F033831B684FF08074002B08BF64
:10AD3800012394FBF3F4604B15219C42A8BF1C46E9
:10AD480022469DE220B933212846FFF71CFE28E35E
:10AD5800012840F01B831A68332114E308B96C21D9
:10AD6800E5E2012840F012836C212846FFF70BFE2C
:10AD7800336820F480229B0403F4802340E130B937
:10AD88006C212846FFF7FFFDC0F3C04009E3012806
:10AD980040F0FC826C212846FFF7F5FD336820F46B
:10ADA8000022DB0403F400232AE130B901462846D7
:10ADB800FFF7E9FDC0F34000F3E2012840F0E68226
:10ADC80000212846FFF7DFFD336820F002025B0010
:10ADD80003F002037CE200287FF43DAF374B1B6889
:10ADE8001B68E7E150B96C212846FFF7CCFD4FF40A
:10ADF8008073C0F3036043FA00F0D2E2012840F008
:10AE0800C5821B68102B1FD00CDC022B18D003DC6A
:10AE1800012B1FD108231FE0042B13D0082B19D1B5
:10AE2800052319E0402B11D003DC202B12D103237A
:10AE380012E0802B0CD0B3F5807F0BD100230BE000
:10AE4800072309E0062307E0042305E0022303E0C3
:10AE5800306002E04FF0FF3333603368013300F0B5
:10AE6800A4826C212846FFF78EFD336820F07062BB
:10AE78001B0603F07063C3E030B96C212846FFF766
:10AE880082FDC0F3C1308CE2012840F07F826C2142
:10AE98002846FFF778FD336820F4C032DB0303F45B
:10AEA800C033ADE060B96C212846FFF76CFDC0F3F4
:10AEB800803076E28C000020FFFF0F00640A00203B
:10AEC800012840F063826C212846FFF75CFD336857
:10AED80020F480429B0303F4804391E030B96C2155
:10AEE8002846FFF750FDC0F300305AE2012840F031
:10AEF8004D826C212846FFF746FD336820F48052C6
:10AF08001B0303F480537BE0D0B96C212846FFF77C
:10AF18003AFD10F4804F4FF06C01284604D0FFF73B
:10AF280032FDC0F3C3103CE2FFF72DFD6C2107464C
:10AF38002846FFF728FD17F4006FC0F302103DE024
:10AF4800012840F023826C212846FFF71CFD10F4ED
:10AF580080444FF06C0128464AD1FFF714FD6C215C
:10AF68002846FFF710FD336820F4006213F0080F3D
:10AF780018BF4FF400646C2128462243FFF7F0FC09
:10AF88006C2128462BE0E8B96C212846FFF7FBFC2A
:10AF980010F480474FF06C01284604D0FFF7F3FC0B
:10AFA800C0F30210FDE1FFF7EEFC6C2104462846D1
:10AFB800FFF7E9FC14F4006FC0F3C31018BF40F0AA
:10AFC8000800EEE1012840F0E1816C212846FFF7F6
:10AFD800DAFC10F480444FF06C01284608D0FFF7E3
:10AFE800D2FC336820F070021B0103F0700307E005
:10AFF800FFF7C9FC336820F4F062DB0103F4F06367
:10B008001A436C21BFE108B96C2165E0012840F0C2
:10B01800BD816C212846FFF7B6FC336820F00F028B
:10B0280003F00F03ECE730B96D212846FFF7ABFCBE
:10B03800C0F3C030B5E1012840F0A8816D21284651
:10B04800FFF7A1FC336820F40042DB039BB289E0E0
:10B0580030B96D212846FFF796FCC0F34130A0E1D6
:10B06800012840F093816D212846FFF78CFC336856
:10B0780020F4C0425B0303F4C04373E030B96D2190
:10B088002846FFF780FCC0F303208AE1012840F03E
:10B098007D816D212846FFF776FC336820F47062C5
:10B0A8001B0203F470635DE030B96D212846FFF799
:10B0B8006AFCC0F3411074E1012840F067816D21FA
:10B0C8002846FFF760FC336820F060025B0103F05C
:10B0D800600347E030B96D212846FFF754FC00F0C3
:10B0E8000F005EE1012840F051816D212846FFF7ED
:10B0F8004AFC336820F00F0203F00F0332E030B946
:10B108006D212846FFF73FFCC0F3006049E10128A4
:10B1180040F03C816D212846FFF735FC336820F06C
:10B1280080721B0603F080731CE070B96D212846FD
:10B13800FFF729FC001410F0400F00F07F0214BF45
:10B148006FF07F030023134334E0012840F01E8191
:10B158006D212846FFF717FC336820F4FE021B0414
:10B1680003F4FE031A436D210DE130B96C21284622
:10B17800FFF709FCC0F3404013E1012840F00681C5
:10B188006C212846FFF7FFFB336820F400325B048C
:10B1980003F4003334E700287FF45DAD6F212846BF
:10B1A800FFF7F1FBC0F30440FBE028B9804B53F8EC
:10B1B8002130DB693360E9E0012840F0E7807C4B0F
:10B1C800326853F821300024DA617A4B1B6883F81F
:10B1D8003040DBE008B9142131E0012840F0D68086
:10B1E8001A68754C32B14FF0807393FBF2F39C42AE
:10B1F800A8BF1C462246142142E030B96C212846DB
:10B20800FFF7C1FBC0F34030CBE0012840F0BE801F
:10B218001A68520302F40052F3E630B96C2128464A
:10B22800FFF7B1FBC0F30350BBE0012840F0AE804C
:10B238001A68120502F47002E3E680B91321284661
:10B24800FFF7A1FB002808BF01204FF0807393FB94
:10B25800F0F0594B9842D4BF3060336096E0012833
:10B2680040F094801B684FF08074002B08BF0123C6
:10B2780094FBF3F4504B13219C42A8BF1C46224672
:10B288002846FFF76DFB346080E030B9702128460E
:10B29800FFF779FBC0F3072083E0012876D17021FE
:10B2A8002846FFF770FB326820F47F40120292B202
:10B2B800024370212846FFF753FB00212846FFF779
:10B2C80062FB336820F00402002BCCBF0423002368
:10B2D8001A43002157E028B970212846FFF753FB8D
:10B2E800C0B25EE0012851D170212846FFF74BFB20
:10B2F800327820F0FF00024344E030B9702128463C
:10B30800FFF741FBC0F301404BE001283ED11B6829
:10B31800032B4AD870212846FFF735FB336820F401
:10B3280040321B0403F440332BE030B97021284627
:10B33800FFF729FBC0F3804033E0012826D11B68C2
:10B34800012B32D870212846FFF71DFB336820F403
:10B3580080229B0403F4802313E030B9702128462F
:10B36800FFF711FBC0F301501BE001280ED170213B
:10B378002846FFF708FB336820F440121B0503F446
:10B3880040131A4370212846FFF7EAFA0020F8BD57
:10B3980000287FF460AC6F212846FFF7F4FAC0F369
:10B3A80009003060F2E70420F8BD1020F8BD00BFA6
:10B3B8008C000020640A0020FFFF0F0007B50192EF
:10B3C80029B9024601AB0120FFF76CFB00E0082019
:10B3D80003B05DF804FB10B413460446084619B9D7
:10B3E800224610BCFFF75EBB082010BC70472DE951
:10B3F800F041674D674814F02FF8EE68664C7368A3
:10B40800012703F1C802A26003F5B872226003F5B0
:10B41800C672626003F5F072226203F5FE72626220
:10B4280003F55372E26003F55A7203F568702261FE
:10B4380003F5617203F56F73E361336862611B6939
:10B44800A06198473368E0691B6998473368606969
:10B458001B69984733682068DB68984733686068D9
:10B46800DB6898473368A068DB68984733682069C9
:10B47800DB6898473368E068DB6898473368606A38
:10B48800DB6898473368206ADB6898473368606AE6
:10B498009B6998473368206A9B6998473368606955
:10B4A8009B6998473368E0689B6998472A693B4BD2
:10B4B80002F1100119607368394D03F50D7353617A
:10B4C800EA6F384B01201A6013F088FD364B374A73
:10B4D8001B684FF000081360226802205A626268F5
:10B4E8009A62EB6F324A1F70C3F80422314A83F81C
:10B4F8000180C3F80822304B85F87870C5F8883089
:10B508002E4BC5F884302E4BC5F880302D4BC5F82E
:10B518008C302D4BC5F8A0302C4BC5F89C302C4BEB
:10B52800C5F890302B4BC5F894302B4BC5F89830A4
:10B538002A4BC5F8B0302A4BC5F8AC30294BC5F8B2
:10B54800BC30294BC5F8B830284BC5F8B430284B67
:10B55800C5F8C83032236B674FF4F0732B67254B5F
:10B56800C5F8C030FFF79CF9636A0222197C5A7447
:10B5780018683A4616F0C8FD3368606A1E4C1B68A6
:10B58800984723689847A3684046BDE8F0411847A4
:10B59800286602082C3D002060140020B43F0020DB
:10B5A80018390020B03F0020640A00208C000020D9
:10B5B80001A80008F5A7000831A6000849A6000858
:10B5C8004BA600084FA60008DFB30008C5B3000863
:10B5D80053A6000849A8000865A8000885A900081E
:10B5E8009DAA00084DAA00086DA6000895A80008A5
:10B5F800A9A8000879A70008B809002010B50B4CC5
:10B6080001440023884204D010F8012B5340E35C26
:10B61800F8E70822002003F0010101EB4000013A9D
:10B6280000F0FF004FEA5303F5D110BD1C64020877
:10B6380028B9044B01221B681A76D9607047082084
:10B64800704700BF90000020F2E74942F0E7002170
:10B65800EEE720B9034B1B6819611876704708207C
:10B66800704700BF90000020F7B505238DF8003023
:10B6780060F07F038DF802300B168DF803300B1441
:10B688008DF804308DF806100B1206460D4600247E
:10B69800072168468DF805308DF80140FFF7AEFFA9
:10B6A8000B4F8DF807003B689B6998473B681DF86E
:10B6B80004009B6801349847082CF7D1054B26F005
:10B6C80080061B6803EB8606756003B0F0BD00BFFB
:10B6D800BC3F0020B83F0020014B0022DA667047CB
:10B6E8001839002000207047F0B5314B00F07F0674
:10B6F800334493F80C3285B0DB070D4605D42D4B47
:10B708001B6803EB860673684EE0052303218DF85A
:10B71800043001A800238DF805308DF80660FFF786
:10B728006DFF254C8DF8070023689B6998472368AF
:10B7380004211B690DEB0100984710F027FC074610
:10B748002368DB699847072805D8384610F02EFC8F
:10B758000A28F5D929E0184B08211B680DEB0100D0
:10B768005B699847072102A8FFF748FF9DF80F403B
:10B7780084421AD19DF80830052B16D19DF809305E
:10B78800FF2B12D19DF80A30B3420ED19DF80C3030
:10B798009DF80B201B0443EA02639DF80E20134317
:10B7A8009DF80D2043EA02232B6005B0F0BD00BFD1
:10B7B800C03F0020B83F0020BC3F0020034B01469B
:10B7C8001B68034A002013F0CEBE00BFB83F00201C
:10B7D800C03F0020014B186813F0DDBEB83F0020C1
:10B7E800014B186813F0CEBEB83F002038B9054B9E
:10B7F8001B689A680B6813440B60194629E70820F0
:10B80800704700BF90000020022804BF0B4B93F83C
:10B81800D00020B90A4BDB681B685B690AE0012885
:10B828000BD1064B93F8D030012B06D1044BDB68C3
:10B838001B689B69034A106818477047183900202D
:10B84800286602089414002038B50020FFF7DCFFB2
:10B85800114B124CDD6820682B689B6898472B6851
:10B8680060689B6898472B68A0689B6898472B6816
:10B87800E0689B6898472B6820699B6898472B6805
:10B8880060699B6898472B68A0699B689847BDE8E2
:10B89800384013F005BC00BF286602089414002045
:10B8A80001BB052820D8DFE800F003070B0F1317AA
:10B8B8000E4B1B681B6912E00C4B1B689B680EE063
:10B8C8000A4B1B68DB680AE0084B1B681B6806E02C
:10B8D800064B1B685B6902E0044B1B685B681360DE
:10B8E800002070470820704704207047900000200F
:10B8F800F1B905281ED8DFE800F003060B1D101764
:10B908000D4B1B6802E00C4B1B689A601A6102E041
:10B91800094B1B68DA6000207047074B002A1B6838
:10B92800B8BF52425A61F6E7034B1B685A60F2E708
:10B9380008207047042070479000002094E6D3E662
:10B9480070B5484E484813F0D5FDF568474C6B680C
:10B9580003F5B872626003F5C672A26003F58E72D1
:10B96800E26003F59C7203F1C800226103F1E4026E
:10B9780003F58073A3612B686261DB6820609847D8
:10B988002B686068DB6898472B68A068DB68984775
:10B998002B68E068DB6898472B682069DB68984764
:10B9A8002B6860691B6998472B68A0691B699847D1
:10B9B800F56A2B6898472E4B2E491D602E4B0125A2
:10B9C800DA6F28460A602D491570C2F804122C490E
:10B9D800C2F80812002151702A4A83F87850C3F837
:10B9E8008820294AC3F88420284AC3F88020284A96
:10B9F800C3F88C20274AC3F8A020274AC3F89C2004
:10BA0800264AC3F89020264AC3F89420254AC3F84A
:10BA1800B020254AC3F8AC20244AC3F8B820244AE9
:10BA2800C3F8C820234AC3F8C42032225A674FF407
:10BA3800C3721A67204AC3F8C020204AC3F8BC2042
:10BA480013F0CCFA1E4B1F4A1B6828461360626825
:10BA58005A62A268BDE870409A624FF448425A613F
:10BA68005A60D1E628660208C03F002094140020DE
:10BA7800BC3F0020B83F002018390020E9B7000873
:10BA8800DDB7000839B6000851B6000853B60008FB
:10BA980057B60008A9B80008F9B800085BB600084E
:10BAA800F5B7000871B60008F1B60008EDB6000851
:10BAB80011B80008E1B6000851B80008C5B7000879
:10BAC800640A00209000002010B50B4C01440023AC
:10BAD800884204D010F8012B5340E35CF8E70822B1
:10BAE800002003F0010101EB4000013A00F0FF00E3
:10BAF8004FEA5303F5D110BD1C65020828B9044B61
:10BB080001221B681A76D96070470820704700BF69
:10BB180094000020F2E74942F0E70021EEE720B95F
:10BB2800034B1B681961187670470820704700BFDF
:10BB380094000020F7B505238DF8003060F07F03EE
:10BB48008DF802300B168DF803300B148DF8043085
:10BB58008DF806100B1206460D460024072168468C
:10BB68008DF805308DF80140FFF7AEFF0B4F8DF8CB
:10BB780007003B689B6998473B681DF804009B6871
:10BB880001349847082CF7D1054B26F080061B682E
:10BB980003EB8606756003B0F0BD00BFDC440020EF
:10BBA800E0440020014B0022DA6670471839002073
:10BBB80000207047F0B5314B00F07F06334493F80E
:10BBC8000C3285B0DB070D4605D42D4B1B6803EB03
:10BBD800860673684EE0052303218DF8043001A81A
:10BBE80000238DF805308DF80660FFF76DFF254CB2
:10BBF8008DF8070023689B699847236804211B690F
:10BC08000DEB0100984710F0C1F907462368DB697E
:10BC18009847072805D8384610F0C8F91428F5D9E8
:10BC280029E0184B08211B680DEB01005B69984758
:10BC3800072102A8FFF748FF9DF80F4084421AD158
:10BC48009DF80830052B16D19DF80930FF2B12D12D
:10BC58009DF80A30B3420ED19DF80C309DF80B20A8
:10BC68001B0443EA02639DF80E2013439DF80D2040
:10BC780043EA02232B6005B0F0BD00BF4C42002010
:10BC8800E0440020DC440020034B01461B68034AC3
:10BC9800002013F0C4BC00BFE04400204C42002048
:10BCA800014B186813F0D3BCE0440020014B18681E
:10BCB80013F0C4BCE044002038B9054B1B689A68EF
:10BCC8000B6813440B60194629E70820704700BF2A
:10BCD80094000020022804BF0B4B93F8D00020B931
:10BCE8000A4BDB681B685B690AE001280BD1064B2D
:10BCF80093F8D030012B06D1044BDB681B689B6995
:10BD0800034A106818477047183900202866020847
:10BD1800BC14002070B5144E0020FFF7DBFFF56857
:10BD2800124C2B6820689B6898472B6860689B6852
:10BD380098472B68A0689B6898472B68E0689B68C1
:10BD480098472B6820699B6898472B6860699B68AF
:10BD580098472B68A0699B689847F36A5B6898477F
:10BD6800BDE8704013F09CB928660208BC14002096
:10BD780001BB052820D8DFE800F003070B0F1317D5
:10BD88000E4B1B681B6912E00C4B1B689B680EE08E
:10BD98000A4B1B68DB680AE0084B1B681B6806E057
:10BDA800064B1B685B6902E0044B1B685B68136009
:10BDB8000020704708207047042070479400002036
:10BDC800F1B905281ED8DFE800F003070B1D10178E
:10BDD8000D4B1B681A6106E00B4B1B689A6002E06A
:10BDE800094B1B68DA6000207047074B002A1B6864
:10BDF800B8BF52425A61F6E7034B1B685A60F2E734
:10BE080008207047042070479400002092E6D1E68D
:10BE180070B5484E484813F0C7FBF568474C6B6847
:10BE280003F5B872626003F5C672A26003F58E72FC
:10BE3800E26003F59C7203F1C800226103F1E40299
:10BE480003F58073A3612B686261DB682060984703
:10BE58002B686068DB6898472B68A068DB689847A0
:10BE68002B68E068DB6898472B682069DB6898478F
:10BE78002B6860691B6998472B68A0691B699847FC
:10BE8800F56A2B6898472E4B2E491D602E4B0125CD
:10BE9800DA6F28460A602D491570C2F804122C4939
:10BEA800C2F80812002151702A4A83F87850C3F862
:10BEB8008820294AC3F88420284AC3F88020284AC1
:10BEC800C3F88C20274AC3F8A020274AC3F89C202F
:10BED800264AC3F89020264AC3F89420254AC3F876
:10BEE800B020254AC3F8AC20244AC3F8B820244A15
:10BEF800C3F8C820234AC3F8C42032225A674FF433
:10BF0800C3721A67204AC3F8C020204AC3F8BC206D
:10BF180013F064F81E4B1F4A1B68284613606268BA
:10BF28005A62A268BDE870409A624FF448425A616A
:10BF38005A60CFE6286602084C420020BC14002054
:10BF4800DC440020E044002018390020B5BC00087B
:10BF5800A9BC000805BB00081DBB00081FBB0008E2
:10BF680023BB000879BD0008C9BD000827BB00082D
:10BF7800C1BC00083DBB0008BDBB0008B9BB000838
:10BF8800DDBC0008ADBB00081DBD000891BC000861
:10BF9800640A00209400002048B101280ED11368DB
:10BFA800074AB3FA83F35B091360002070471368EC
:10BFB800044AB3FA83F35B0993727047042070470D
:10BFC80098000020E444002020B9034B5B68196105
:10BFD80018767047082070479800002010B50D4B60
:10BFE8000D4C1B6822460146002013F05AFB237AA9
:10BFF8000A4A1BB1D36E43F0010302E0D36E23F06B
:10C008000103617A11B143F0020301E023F0020356
:10C01800D36610BD28450020E444002018390020CC
:10C02800014B186813F0B1BB2845002040B9054BF7
:10C03800012258721872044B5B681A76D9607047EF
:10C0480008207047E444002098000020EEE74942A9
:10C05800ECE70021EAE738B9044B5B689A680B689B
:10C0680013440B601946AFE708207047980000207A
:10C0780020B9034B1B681B680B607047082070478A
:10C08800640A0020022804BF0B4B93F8D00020B9A3
:10C098000A4BDB681B685B690AE001280BD1064B79
:10C0A80093F8D030012B06D1044BDB681B689B69E1
:10C0B800034AD068184770471839002028660208D4
:10C0C800E414002038B50020FFF7DCFF0F4B104CBC
:10C0D800DD68E0682B685B6998472B6820689B6877
:10C0E80098472B68A0689B6898472B68E0689B680E
:10C0F80098472B6820699B6898472B6860689B68FD
:10C108009847BDE8384012F0CBBF00BF2866020848
:10C11800E414002038B50A4D6B681C6874B9094BE3
:10C128000948196813F014FB6B68022083F8304043
:10C1380001242C60FFF7A6FF204638BD002038BD3B
:10C148009800002028450020E44400202DE9F84309
:10C15800830C04460ED0C0F34243062B0AD1294B68
:10C1680020F01F045A7A0AB11B7800E0DB7A03F04A
:10C178001F031C43244F254E3B68254D9B68002117
:10C18800C4F30740D6F8008095F8189098472A7E9F
:10C19800336808EB8908C8F8040003EB82035A687F
:10C1A800002112025A603B68C4F307209B68984735
:10C1B80033682A7E012103EB820253681843000288
:10C1C8003B6850609B68E0B298473268297E02EB72
:10C1D80081014B6818430011A30C4860106107D017
:10C1E800C4F34243072B09D1C4F30111297605E0B2
:10C1F800082302EB83035C60BDE8F88343F008037F
:10C20800F7E700BFE444002024450020284500202B
:10C21800E4140020C2F31300830C0B4A05D0431426
:10C22800062B04BF00F01F03D372084B01F07701FF
:10C238001B6841F0080103EB81014860937A0BB950
:10C24800FFF784BF704700BFE44400202845002062
:10C258000A4601460020FFF7DDBF10B5074B01F085
:10C268007F049B7A23B90B0702D4204600F00AF812
:10C27800034B186800EB8400406810BDE4440020BC
:10C288002845002038B504460F210020FFF7E5FFB8
:10C298000323B4FBF3F3054603EB4303E41A240139
:10C2A80004F0300420F030002043FFF74FFF284609
:10C2B800BDE83840FFF74ABF10B50C4601460020DC
:10C2C800FFF7CBFF206010BDA82A38B504461D46ED
:10C2D80000F0738242D81D2A00F029811CD8042A54
:10C2E80000F0CA800BD8012A00F08F807AD3022A86
:10C2F80000F09E80032A00F0AF8000F06CBC062A94
:10C3080000F0E380C0F0CE80072A00F0F980082A08
:10C3180000F0048100F05FBCA32A00F0BD8110D8B2
:10C32800A02A00F05C8104D88C2A00F0098100F072
:10C3380052BCA12A00F07081A22A00F08B8100F083
:10C348004ABCA52A00F0E281C0F0C381A62A00F009
:10C35800FA81A72A00F0158200F03DBCB22A00F04D
:10C3680047831DD8AD2A00F0AB820CD8AA2A00F06A
:10C378005D82C0F03E82AB2A00F07582AC2A00F0E4
:10C38800908200F028BCAF2A00F0DB82C0F0B582B2
:10C39800B02A00F0F282B12A00F00D8300F01BBC35
:10C3A800B72A00F093830CD8B42A00F05B83C0F05E
:10C3B8003C83B52A00F06183B62A00F0748300F04C
:10C3C8000ABCCE2A50D006D8B82A00F09B83B92AD6
:10C3D80000F0B683FFE3D02A00F0E683D62A00F007
:10C3E800EE83F8E330B9AA4B03EB81014B681B6974
:10C3F8002B6038BD012840F0F083A54B2A6803EB79
:10C4080081014B6800201A6138BD30B9A04B03EB9D
:10C4180081014B689B682B6038BD012840F0DF83A1
:10C428009B4B2A6803EB81014B6800209A6038BD5A
:10C4380038B9974B002003EB81014B68DB682B6010
:10C4480038BD012840F0CD83914B2A6803EB810168
:10C458004B680020DA6038BD48B98D4B03EB810189
:10C468004B681B682B6038BD002800F08683012CC0
:10C4780014BF0020042038BD30B9854B03EB81017F
:10C488004B685B692B6038BD012840F0AC83804B5A
:10C49800002003EB81012B684A68002BB8BF5B4280
:10C4A800536138BD30B97A4B03EB81014B685B6847
:10C4B8002B6038BD012840F09883754B2A6803EB40
:10C4C80081014B6800205A6038BD18B9714BDB7A7E
:10C4D8002B6038BD012840F08A831A686D4B0E2105
:10C4E8000020DA72FFF7B9FE2B6820F01F0203F074
:10C4F8001F031A430E210020FFF78CFE002038BDD1
:10C5080020B9644B00201B782B6038BD012840F00F
:10C5180070831A685F4B00201A7038BD0028A6D1B6
:10C528005B4B03EB81014B685B7E2B6038BD0028B9
:10C538009DD1574B03EB81014B681B682B6038BDBD
:10C5480050B908210020FFF788FE00F00F00C0F165
:10C5580008002860002038BD012840F04C831B6883
:10C56800102B1FD00CDC022B18D003DC012B1FD1A1
:10C5780008231FE0042B13D0082B19D1052319E039
:10C58800402B11D003DC202B12D1032312E0802B87
:10C598000CD0B3F5807F0BD100230BE0072309E013
:10C5A800062307E0042305E0022303E0286002E0F5
:10C5B8004FF0FF332B602B68013300F01E830821F6
:10C5C8000020FFF74AFE2B6820F00F0203F00F034C
:10C5D8001A4308210020FFF71DFE002038BD38B996
:10C5E8000821FFF73AFEC0F340202860204638BDF6
:10C5F800012840F0048308210020FFF72EFE2B6855
:10C6080020F400725B0203F400731A43082100202F
:10C61800FFF700FE002038BD40B908210020FFF7D1
:10C628001CFEC0F300202860002038BD012840F01F
:10C63800E88208210020FFF710FE2B6820F48072A2
:10C648001B0203F480731A4308210020FFF7E2FD60
:10C65800002038BD38B90C21FFF7FFFDC0F3C13009
:10C668002860204638BD012840F0CD820C210020EA
:10C67800FFF7F3FD2B6820F4C032DB0303F4C0336B
:10C688001A430C210020FFF7C5FD002038BD00BF6C
:10C6980098000020E444002038B90C21FFF7DDFDA4
:10C6A800C0F380302860204638BD012840F0AD82B4
:10C6B8000C210020FFF7D1FD2B6820F480429B035A
:10C6C80003F480431A430C210020FFF7A3FD002048
:10C6D80038BD38B90C21FFF7C0FDC0F3C120286070
:10C6E800204638BD012840F092820C210020FFF737
:10C6F800B4FD2B6820F4C052DB0203F4C0531A4384
:10C708000C210020FFF786FD002038BD38B90C2128
:10C71800FFF7A3FDC0F3C3102860204638BD0128E9
:10C7280040F077820C210020FFF797FD2B6820F45A
:10C73800F062DB0103F4F0631A430C210020FFF7D9
:10C7480069FD002038BD40B90C210020FFF785FDA8
:10C75800C0F302102860002038BD012840F05B8239
:10C768000C210020FFF779FD2B6820F070021B01D7
:10C7780003F070031A430C210020FFF74BFD002043
:10C7880038BD38B90C21FFF768FD00F00F002860AC
:10C79800204638BD012840F040820C210020FFF7D8
:10C7A8005CFD2B6820F00F0203F00F031A430C21E5
:10C7B8000020FFF72FFD002038BD38B90521FFF70D
:10C7C8004CFDC0F3C0302860204638BD012840F039
:10C7D80026820D210020FFF740FD2B6820F400423F
:10C7E800DB039BB21A430D210020FFF713FD002045
:10C7F80038BD38B90521FFF730FDC0F34130286056
:10C80800204638BD012840F00C820D210020FFF79A
:10C8180024FD2B6820F4C0425B0303F4C0431A4391
:10C828000D210020FFF7F6FC002038BD38B905219E
:10C83800FFF713FDC0F303202860204638BD012808
:10C8480040F0F1810D210020FFF707FD2B6820F44F
:10C8580070621B0203F470631A430D210020FFF776
:10C86800D9FC002038BD40B905210020FFF7F5FCB0
:10C87800C0F341102860002038BD012840F0D58160
:10C888000D210020FFF7E9FC2B6820F060025B0116
:10C8980003F060031A430D210020FFF7BBFC0020C2
:10C8A80038BD20B9BE4B1B685B6B2B6038BD0128B7
:10C8B80040F0BD81BA4B2A681B6800205A6338BD16
:10C8C80038B90621FFF7C9FCC0F3004028602046AC
:10C8D80038BD012840F0AD810E210020FFF7BDFCD6
:10C8E8002B6820F480321B0403F480331A430E2192
:10C8F8000020FFF78FFC002038BD70B90621FFF734
:10C90800ACFC000A00F07F0310F0400018BF6FF085
:10C918007F0018432860204638BD012840F08B81ED
:10C928000E210020FFF799FC2B6820F4FE421B0221
:10C9380003F4FE431A430E210020FFF76BFC00208E
:10C9480038BD38B90721FFF788FCC0F3813028606B
:10C95800204638BD012840F070810F210020FFF7E4
:10C968007CFC2B6820F440429B039BB21A430F21A6
:10C978000020FFF74FFC002038BD40B907210020F8
:10C98800FFF76BFCC0F301302860002038BD012898
:10C9980040F055810F210020FFF75FFC2B6820F441
:10C9A80040521B0303F440531A430F210020FFF7A2
:10C9B80031FC002038BD38B90721FFF74EFCC0F321
:10C9C80080202860204638BD012840F03A810F2198
:10C9D8000020FFF742FC2B6820F480629B0203F4DE
:10C9E80080631A430F210020FFF714FC002038BD94
:10C9F80038B90721FFF731FCC0F301202860204631
:10CA080038BD012840F01F810F210020FFF725FCC9
:10CA18002B6820F440721B0203F440731A430F2161
:10CA28000020FFF7F7FB002038BD38B90721FFF7D2
:10CA380014FCC0F380102860204638BD012840F05F
:10CA480004810F210020FFF708FC2B6820F040022A
:10CA58009B0103F040031A430F210020FFF7DAFB84
:10CA6800002038BD00287FF402AD0221FFF7F5FB56
:10CA7800C0F384202860204638BD38B9494B0020CF
:10CA880003EB81014B68DB692B6038BD012840F05E
:10CA9800DE80444B2A6803EB81014B680020DA6191
:10CAA80083F8300038BD30B93E4B03EB81014B6849
:10CAB8001B6A2B6038BD012840F0CB80394B2A68AF
:10CAC80003EB81014B6800201A6238BD38B9072191
:10CAD800FFF7C3FBC0F3C0102860204638BD01280B
:10CAE80040F0B9800F210020FFF7B7FB2B6820F03A
:10CAF8008002DB01DBB21A430F210020FFF78AFB1B
:10CB0800002038BD40B904210020FFF7A6FBC0F380
:10CB180040302860002038BD012840F09E800C215C
:10CB28000020FFF79AFB2B6820F400525B0303F404
:10CB380000531A430C210020FFF76CFB002038BD7E
:10CB480038B90721FFF789FBC0F300402860204669
:10CB580038BD012840F083800F210020FFF77DFBBE
:10CB68002B6820F480321B0403F480331A430F210E
:10CB78000020FFF74FFB002038BD0A4B1B6833B17C
:10CB88000221FFF76AFB800A00F4787004E00121B3
:10CB9800FFF763FBC0F389202860002038BD00BF81
:10CBA800640A00209800002000287FF460AC03216C
:10CBB8000020FFF752FBC0B22860002038BD18B92A
:10CBC800294B5B682B6038BD01284AD11A68264B6F
:10CBD80000205A6038BD042038BD002038BD002030
:10CBE80038BD002038BD002038BD002038BD0020E9
:10CBF80038BD002038BD002038BD102038BD0020C9
:10CC080038BD002038BD002038BD002038BD0020C8
:10CC180038BD002038BD002038BD002038BD0020B8
:10CC280038BD002038BD002038BD002038BD0020A8
:10CC380038BD002038BD002038BD002038BD002098
:10CC480038BD002038BD002038BD002038BD002088
:10CC580038BD002038BD002038BD002038BD002078
:10CC680038BD002038BD00BFE444002007B501925C
:10CC780029B9024601AB0120FFF726FB00E0082096
:10CC880003B05DF804FB10B413460446084619B90E
:10CC9800224610BCFFF718BB082010BC704710B51F
:10CCA8000D2104460020FFF7D8FA04F00F0420F005
:10CCB8000F0222430D210020BDE81040FFF7AABA59
:10CCC8002DE9F8438B0C0C460ED0C1F34243062BDA
:10CCD8000AD1294B21F01F045A7A0AB11B7800E0C7
:10CCE800DB7A03F01F031C43244F254E3B68254D78
:10CCF8009B680021C4F30740D6F8008095F8199086
:10CD080098476A7E336808EB8908C8F8040003EB83
:10CD180082035A68002112025A603B68C4F3072054
:10CD28009B68984733686A7E012103EB8202536847
:10CD3800184300023B6850609B68E0B2984732682D
:10CD4800697E02EB81014B6818430011A30C48600F
:10CD5800106107D0C4F34243072B09D1C4F3011172
:10CD6800697605E0082302EB83035C60BDE8F8837D
:10CD780043F00803F7E700BFE444002024450020FF
:10CD880028450020E41400202DE9F8434C4FDFF833
:10CD98009081DFF8909101263846C8F8006012F0BB
:10CDA8005FFCD9F80C50474C6B6803F1C802E2608D
:10CDB80003F1E40203F5B870226103F5C67203F5C6
:10CDC8000D7323602B68A260DB68606098472B684E
:10CDD800A068DB6898472B68E068DB6898472B6891
:10CDE80020691B6998472B682068DB689847686842
:10CDF8002B6820309B6860619847D9F81030324A18
:10CE080003F110011160226830465A6105233B7016
:10CE18004FF47A737B6012F0E1F82C4B62681B6860
:10CE280000215A62A26899639A622269C8F804309C
:10CE3800DA62274A27481A65274BDA6F02602748C3
:10CE48001170C2F8080226485170C2F80402254A37
:10CE580083F87860C3F88820234A0220C3F8842026
:10CE6800224AC3F88020224AC3F88C20214AC3F8FA
:10CE7800A020214AC3F89C20204AC3F89020204AC9
:10CE8800C3F894201F4AC3F8B0201F4AC3F8AC2047
:10CE98001E4AC3F8BC201E4AC3F8B8201D4AC3F86E
:10CEA800B4201D4AC3F8C82032225A6740F225121E
:10CEB8001A671A4AC3F8C020BDE8F843FFF7E2B87A
:10CEC800E4440020E414002024450020640A0020E3
:10CED800A7CC0008284500201839002029C00008E0
:10CEE8001DC1000835C0000855C0000857C000081B
:10CEF8005BC000088FCC000875CC0008D1BF0008C3
:10CF08005FC0000859C20008C1C20008E5BF000898
:10CF1800A1BF000879C000088DC00008CDC0000876
:10CF28009800002028660208014B00225A607047CA
:10CF3800183900200128F8B5144633D00BD3FF2840
:10CF480043D1244CE36FD3F8043298476369D3F88C
:10CF5800043298472FE0136833F0030237D113F0F7
:10CF6800010F1D4D1D4E03D0F3681B681B6906E0B9
:10CF7800F76828693B68DB6898473B689B692869BC
:10CF88009847206810F0020403D0F3681B681B69F7
:10CF980006E0F66868693368DB68984733689B6918
:10CFA800686907E014680C4D0C4B34B1DB681B68EA
:10CFB8001B69E86898470020F8BDDE68E8683368B0
:10CFC800DB68984733689B69F3E70420F8BD1020B5
:10CFD800F8BD00BF183900200C150020286602088B
:10CFE80070B5144E144CF56860682B689B699847B7
:10CFF8002B6860699B6898472B6820699B689847ED
:10D008002B68E0689B6898472B68A0689B689847DE
:10D018002B68A0699B6898472B6820689B6898478D
:10D028002B6860689B6898473369BDE87040DB6986
:10D03800184700BF286602080C1500202DE9F843A0
:10D04800194C1E462368894607469B68002140F014
:10D05800800090469DF820509847144B002183F893
:10D06800E002236848469B689847236800219B682C
:10D0780040469847236800219B68304698472368B4
:10D0880028469B6801219847094B48EA09281B68EC
:10D0980046EA082607F07F0703EB870745EA0625D7
:10D0A8007D60BDE8F88300BF2C4500203445002092
:10D0B8003045002007B5CBB20093C1F30742C1F356
:10D0C8000723090EFFF7BAFF03B05DF804FBFFF76B
:10D0D800F1BF10B50F4C104A2368D268197812684E
:10D0E8000E4B31B9926958689047236801221A702B
:10D0F8000EE058685269904704211020FFF7DAFFC4
:10D10800236800221A70064BDB6FD3F80432984765
:10D11800012010BD30450020286602080C150020AB
:10D128001839002010B5064C0649226812F024FD73
:10D1380023681B7813B1BDE81040CAE710BD00BFD3
:10D14800304500203445002010B5002940F0888083
:10D15800122867D01AD805284CD007D8012837D00C
:10D1680033D3022837D0042835D07BE00F2847D0A6
:10D1780007D80E2876D1002A14BF022101212020C9
:10D188004CE010283FD0112843D06BE017285BD023
:10D1980009D814284FD048D315284FD0162861D164
:10D1A80011462D203AE01A2854D006D818284ED017
:10D1B800192857D11146302030E01B284DD0D628E9
:10D1C80050D12A491520514328E01146372025E03F
:10D1D8001146212022E082EAE271254BA1EBE2719F
:10D1E800994204DD234911EA220238BF1A46110286
:10D1F800242013E0940DA405B4BB910028200DE071
:10D20800114625200AE0940DA40574BB91002A203C
:10D2180004E0930D9B053BBB91002920FFF74AFFD3
:10D22800002010BD11462720F8E7940DA405DCB9AD
:10D2380091002B20F2E711462620EFE7940DA40574
:10D2480094B911462C20E9E711462E20E6E711464D
:10D258002F20E3E711463320E0E711463420DDE7CD
:10D26800082010BD042010BD102010BD0071020060
:10D2780000127A0000EE85FF70B5254E00F07F049D
:10D28800331993F80C32DB0705D4224B1B6803EBE8
:10D298008404606870BD204D00212B6820469B687F
:10D2A80098472B6800219B68084698472B680021FF
:10D2B8009B68084698472B6800219B680846984752
:10D2C8002B6801219B68002098472B6800219B68E8
:10D2D800204698472B6886F8E00200219B6808469C
:10D2E80098472B68002104029B68084698472B68DA
:10D2F8000021204304029B68084698472B68204376
:10D3080004029B68012100209847204370BD00BF9C
:10D3180034450020304500202C45002010B50C462F
:10D32800FFF7AAFF206010BD38B50D46044668B95E
:10D338002020FFF7A1FF40F004012020FFF7BAFEEC
:10D3480029463720FFF7B6FE204638BD082038BDED
:10D3580038B50C4605462120FFF78EFF2368C11813
:10D3680021602846BDE83840DEE738B515460C464A
:10D3780000296CD1112852D01ED8042841D008D8D1
:10D3880001283CD039D302283BD0032861D1222080
:10D3980058E00E283CD009D8052837D0082858D19D
:10D3A8000F20FFF769FF00F001004DE00F2834D08F
:10D3B80010284ED12A2036E017283CD00ED8142841
:10D3C80035D005D812282CD0132842D12B202AE09A
:10D3D80015282ED016283CD12D2033E01A282ED01F
:10D3E80005D8182829D0192833D130202AE01B283D
:10D3F80027D0D6282DD1152024E0372022E021205F
:10D4080020E02420FFF738FF00121DE028200AE062
:10D418002020FFF731FF400016E0252012E02920E8
:10D4280001E027200EE0FFF727FF80100CE0262000
:10D4380008E02C2006E02E2004E02F2002E0332014
:10D4480000E03420FFF718FF2860204638BD082088
:10D4580038BD042038BD10B50C46C8B92020FFF7E8
:10D468000BFF20F004012020FFF724FE84EAE47279
:10D47800084BA2EBE4729A4204DD074A12EA24043C
:10D4880038BF1C4621022420FFF714FE002010BDDF
:10D49800082010BD00127A0000EE85FF0021DAE7AF
:10D4A8004942D8E7D7E770B53F4E404812F07EFAB8
:10D4B800F5683F4C6B6803F5AA72A26103F55372D5
:10D4C800626103F55A72226103F5617203F57670A1
:10D4D800E26003F5687203F57D7323602B68A26030
:10D4E800DB68606098472B686069DB6898472B6841
:10D4F8002069DB6898472B68E068DB6898472B68E9
:10D50800A068DB6898472B6860685B6998472B6858
:10D5180060695B6998472B6820695B6998472B6845
:10D52800E0685B6998472B68A0685B6998472B6837
:10D53800A0691B6998472B6820681B69984732695E
:10D548001C4B1D4C1A606B68012103F5377353603F
:10D5580062691A4B20201A60FFF7ACFD6369184A0C
:10D56800C3F8042200225A7001221A70154B227443
:10D578002362154BE361154BA361154B6362154B91
:10D58800A363154B6363154BA362154BE362154BFD
:10D59800A364154B6364154B6365154B2365154BE5
:10D5A800E365154BA36570BD286602083445002065
:10D5B8000C1500202C45002018390020304500208B
:10D5C800DBD000085FD40008ADD40008A9D4000857
:10D5D800A5D4000873D3000851D1000831D300083E
:10D5E80059D30008D7D0000825D300082DD100084A
:10D5F8003DCF000831CF0008E9CF0008014B0022D9
:10D608005A607047183900200128F8B5144633D0FD
:10D618000BD3FF2843D1244CE36FD3F80432984747
:10D628006369D3F8043298472FE0136833F0030294
:10D6380037D113F0010F1D4D1D4E03D0F3681B6841
:10D648001B6906E0F76828693B68DB6898473B6810
:10D658009B6928699847206810F0020403D0F36892
:10D668001B681B6906E0F66868693368DB689847D9
:10D6780033689B69686907E014680C4D0C4B34B13A
:10D68800DB681B681B69E86898470020F8BDDE68FE
:10D69800E8683368DB68984733689B69F3E70420D8
:10D6A800F8BD1020F8BD00BF18390020381500203B
:10D6B8002866020870B5164E164CF56860682B6827
:10D6C8009B6998472B6860699B6898472B68206915
:10D6D8009B6898472B68E0689B6898472B68A06808
:10D6E8009B6898472B68E0699B6898472B68A069F6
:10D6F8009B6898472B6820689B6898472B686068E8
:10D708009B6898473369BDE87040DB69184700BFDC
:10D71800286602083815002038B50A4B0A4CDD681F
:10D7280060682B689B69984701200EF035FC2B68D0
:10D7380060685B699847054B186812F081FA012008
:10D7480038BD00BF28660208381500201848002098
:10D7580038B50A4B0A4CDD6860682B689B699847A6
:10D7680001200EF019FC2B6860685B699847054B2F
:10D77800186812F05CFA012038BD00BF286602085C
:10D7880038150020184800202DE9F8430E46194D99
:10D7980098462B6800219B6846F0800017469DF844
:10D7A80020909DF824409847134B002183F8E0020D
:10D7B8002B6838469B6898472B6800219B68404631
:10D7C80098472B6800219B68484698472B68012199
:10D7D8009B6820469847094B44EA09221B6806F0D3
:10D7E8007F0642EA084203EB860642EA0762726055
:10D7F800BDE8F8831C480020204800201848002075
:10D8080007B5D3B20193C2F307230093C2F30743CA
:10D81800120EFFF7B9FF03B05DF804FB70B5174CA3
:10D8280001462368164A1D78002012F0B3FA1DB38A
:10D8380023681A7802BB134C94F86830012B06D081
:10D84800032B0BBF002228220D230F2300E00B23FC
:10D8580043F0884343F0401343EA42320421002056
:10D86800FFF7CEFFE36F012D0CBFD3F80432D3F8D6
:10D878000832BDE87040184770BD00BF1848002046
:10D8880020480020183900200A4601460020FFF7EA
:10D89800B7BF38B514460D4600297ED1122863D08B
:10D8A8001AD8052848D007D8012834D031D30228FF
:10D8B80033D0042831D072E00F2843D007D80E287F
:10D8C8006DD1002A14BF02220122202163E0102812
:10D8D8003AD011283ED062E0172855D008D814282D
:10D8E8004AD043D3152849D0162858D12D2152E0C3
:10D8F8001A284DD005D8182848D019284FD13021DA
:10D9080049E01B2846D0D62849D1274A1521624329
:10D9180041E037213FE021213DE084EAE472234BD6
:10D92800A2EBE4729A4204DD214A12EA240438BFC9
:10D938001C462202242112E0950DAD058DBB9200F4
:10D94800282128E0252126E0950DAD0555BB92003C
:10D958002A2120E0930D9B051BBB92002921002062
:10D96800FFF74EFF002038BD272114E0950DAD05C7
:10D97800BDB992002B210EE026210CE0940DA405E0
:10D988007CB92C212046EBE72E2104E02F2102E070
:10D99800332100E034212846E2E7082038BD04207E
:10D9A80038BD102038BD00BF0071020000127A0097
:10D9B80000EE85FF70B5254E01F07F04331993F80A
:10D9C8000C32DB0705D4224B1B6803EB8404606828
:10D9D80070BD204D00212B6820469B6898472B6816
:10D9E80000219B68084698472B6800219B680846D9
:10D9F80098472B6800219B68084698472B680121A7
:10DA08009B68002098472B6800219B682046984710
:10DA18002B6886F8E00200219B68084698472B6827
:10DA2800002104029B68084698472B680021204380
:10DA380004029B68084698472B68204304029B68A9
:10DA4800012100209847204370BD00BF20480020D6
:10DA5800184800201C48002010B50C46014600203C
:10DA6800FFF7A8FF206010BD38B50D46044678B909
:10DA78002021FFF79FFF202140F004022046FFF7F6
:10DA8800BFFE20462A463721FFF7BAFE204638BD9A
:10DA9800082038BD38B50C4621210546FFF78AFF16
:10DAA8002168014421602846BDE83840DCE738B5E4
:10DAB80015460C46002975D1112859D01FD80428BD
:10DAC80042D008D801283DD03AD302283CD00328B8
:10DAD8006AD1222160E00E283ED00AD8052839D024
:10DAE800082861D10F212046FFF764FF00F00100EC
:10DAF80055E00F283AD0102856D12A213CE01728A3
:10DB080043D00ED814283CD005D8122832D0132878
:10DB18004AD12B2130E0152835D0162844D12D21A3
:10DB28003AE01A2835D005D8182830D019283BD122
:10DB3800302131E01B282ED0D62835D115212BE0F5
:10DB4800372129E0212127E024212046FFF732FF51
:10DB5800001224E028210FE020212046FFF72AFFA9
:10DB680000F00300831E5842584118E0252113E0B5
:10DB7800292101E027210FE02046FFF71BFF801035
:10DB88000DE0262108E02C2106E02E2104E02F21BB
:10DB980002E0332100E034212046FFF70BFF286024
:10DBA800204638BD082038BD042038BD38B50C469D
:10DBB8000546D8B92021FFF7FDFE202120F00402F8
:10DBC8002846FFF71DFE84EAE472094BA2EBE472D3
:10DBD8009A4204DD074A12EA240438BF1C4622028E
:10DBE80024210020FFF70CFE002038BD082038BD96
:10DBF80000127A0000EE85FF0021D7E74942D5E7F9
:10DC0800D4E7354B2DE9F0415E6A1A6A350245EAD8
:10DC180012651402C6B293F82820586B26430027D1
:10DC28001C6B2F430132050E000240EA1460D2B289
:10DC380024021C63C3E9086783F8282058631C463C
:10DC4800002945D0042A04D93A466D210020FFF75F
:10DC5800D7FD226A6C210020FFF7D2FD01200EF0CB
:10DC68009BF9226A6C210020FFF7CAFD01200EF003
:10DC780093F900230022C4E90C2394F82830DFF834
:10DC88005880042B0AD96F210020FFF793FED8E9AA
:10DC98000C23002632430343C8E90C236E210020DD
:10DCA800FFF788FED4E90C67034694F8282047EA72
:10DCB800E371C2F10802D200304317F039FB0023A8
:10DCC8000022C4E90C01C4E90823002384F82830A1
:10DCD8002846BDE8F08100BF3815002070B5464ED3
:10DCE800464811F05BFFF568454C6B6803F59C727C
:10DCF800E26103F5AA72A26103F55372626103F54A
:10DD08005A72226103F5617203F57670E26003F5D9
:10DD1800687203F57D7323602B68A260DB6860601E
:10DD280098472B686069DB6898472B682069DB682F
:10DD380098472B68E068DB6898472B68A068DB6821
:10DD480098472B6860685B6998472B6860695B69CE
:10DD580098472B6820695B6998472B68E0685B697E
:10DD680098472B68A0685B6998472B68E0691B692E
:10DD780098472B68A0691B6998472B6820681B691E
:10DD8800984732691F4B204C1A606B68202103F5B5
:10DD98003773536062691D4B00201A600122FFF738
:10DDA8002FFD63690021597019490122C3F8041233
:10DDB80018491A70C3F80812174B22746366174B78
:10DDC8002362174BE361174BA361174B6362174B31
:10DDD800A363174B6363174BA362174BE362174B9D
:10DDE800A364174B6364174B6365174B2365174B85
:10DDF800E365174BA36570BD28660208204800201C
:10DE0800381500201C480020183900201848002028
:10DE180059D7000821D700080BDC0008B5DB00083B
:10DE280009DC000805DC000801DC0008B7DA000896
:10DE38009BD8000871DA00089DDA000891D800081C
:10DE480061DA000825D8000811D6000805D60008B0
:10DE5800BDD60008014B00225A60704718390020CF
:10DE680070B5184E184CF56860682B689B69984720
:10DE78002B68A0699B6898472B6860699B689847DE
:10DE88002B6820699B6898472B68E0689B689847CF
:10DE98002B68A0689B6898472B68206A9B689847FE
:10DEA8002B68E0699B6898472B6820689B689847AF
:10DEB8002B6860689B6898473369BDE87040DB69E8
:10DEC800184700BF28660208801500200228F8B508
:10DED80014464CD003D880B1012835D060E003281F
:10DEE80056D0FF285CD12F4CE36FD3F80432984703
:10DEF8006369D3F8043298472FE0136833F00302BC
:10DF08002BD113F0010F284D284E03D0F3681B685E
:10DF18001B6906E0F76868693B68DB6898473B68F7
:10DF28009B6968699847206810F0020403D0F36879
:10DF38001B681B6906E0F668A8693368DB689847C0
:10DF480033689B69A86907E01468174D174B34B10B
:10DF5800DB681B681B69286998470020F8BDDE68E4
:10DF680028693368DB68984733689B69F3E7146866
:10DF78000D4D0E4B1CB1DB681B681B6906E0DE68A3
:10DF8800A8683368DB68984733689B69A868E3E743
:10DF9800012011F08DFF20600028DED12020F8BD7F
:10DFA8000420F8BD183900208015002028660208D2
:10DFB80038B50A4B0A4CDD6860682B689B6998473E
:10DFC80001200DF0E9FF2B6860685B699847054BF5
:10DFD800186811F043FF012038BD00BF2866020809
:10DFE80080150020044B002038B50A4B0A4CDD6828
:10DFF80060682B689B69984701200DF0CDFF2B685E
:10E0080060685B699847054B186811F01EFF01208E
:10E0180038BD00BF2866020880150020044B002088
:10E028002DE9F843194D99462B680F4606469B681B
:10E03800002140F0800090469DF820409847144BFE
:10E04800002183F8E0022B6838469B6898472B68C4
:10E0580000219B68404698472B6800219B684846EA
:10E0680098472B6801219B6820469847094B44EA4A
:10E0780009211B6806F07F0641EA084103EB860682
:10E0880041EA07617160BDE8F88300BF084B0020D2
:10E098000C4B0020044B002007B5CBB20093C1F312
:10E0A8000742C1F30723090EFFF7BAFF03B05DF873
:10E0B80004FB70B5154C16492268157811F062FFFB
:10E0C80015B323681978F9B9124C94F86830012B04
:10E0D80006D0032B0BBF002128210D230F2300E0BE
:10E0E8000B2343F0884343F0401343EA41310420B3
:10E0F800FFF7D2FFE36F012D0CBFD3F80432D3F83A
:10E108000832BDE87040184770BD00BF044B0020BE
:10E118000C4B002018390020FFF7BEBF70B5254E04
:10E1280000F07F04331993F80C32DB0705D4224B37
:10E138001B6803EB8404606870BD204D00212B68C8
:10E1480020469B6898472B6800219B68084698479B
:10E158002B6800219B68084698472B6800219B681C
:10E16800084698472B6801219B68002098472B6830
:10E1780000219B68204698472B6886F8E00200211A
:10E188009B68084698472B68002104029B6808464C
:10E1980098472B680021204304029B68084698474B
:10E1A8002B68204304029B680121002098472043E4
:10E1B80070BD00BF0C4B0020044B0020084B002012
:10E1C80010B50C46FFF7AAFF206010BD38B50D4604
:10E1D800044668B92020FFF7A1FF40F00401202081
:10E1E800FFF75AFF29463720FFF756FF204638BD6C
:10E1F800082038BD38B50C4605462120FFF78EFFAC
:10E208002368C11821602846BDE83840DEE76F2939
:10E2180070B50446154600F0BA8155D8122900F0A9
:10E228002A8127D8052900F0D88011D8022900F0C2
:10E23800B48006D8002900F09E80012900F0A4804F
:10E24800F0E2032900F0AF80042900F0A680E9E29B
:10E258000F2900F0E98006D8082900F0CD800E29A2
:10E2680000F0D280DEE2102900F0E780112900F0EA
:10E27800F380D7E2182900F0428111D8152900F05F
:10E288001E8106D8132900F0FF80142900F00E81A2
:10E29800C8E2162900F02181172900F02781C1E280
:10E2A8001B2900F0478106D8192900F031811A2965
:10E2B80000F03781B6E26D2900F04E8100F25581F9
:10E2C8006C2900F04081ADE27D2900F0048227D856
:10E2D800752900F0AF8111D8722900F0838106D822
:10E2E800702900F06581712900F06B819AE2732929
:10E2F80000F08A81742900F0928193E2782900F075
:10E30800D28106D8762900F0B181772900F0C3813F
:10E3180088E2792900F0CF817C2900F0D48181E25C
:10E32800882900F0218211D8842900F0058206D8B6
:10E338007E2900F0D881812900F0EC8172E28529DC
:10E3480000F0FF81862900F007826BE2C82900F0FF
:10E35800388106D8892900F019828A2900F02D828F
:10E3680060E2D42900F04682D62900F04E82D129F5
:10E3780040F0588234E208B9372033E2012840F0EF
:10E38800B981116837204AE208B921202AE2012818
:10E3980040F0B0811168212041E25CB92420FFF7E8
:10E3A800BDFE0012A5E108B922201BE2012C00F0F5
:10E3B80039829FE1012C40F09D812968A14B81EAB7
:10E3C800E172A2EBE1729A4204DD9F4A12EA21014E
:10E3D80038BF19460902242021E208B9282055E04F
:10E3E800012840F0878111688C0DA405002C40F0AD
:10E3F8001B828900282012E20028D7D10F20FFF7BE
:10E408008DFE00F0010074E120B92020FFF786FEA0
:10E4180040006EE1012840F06D8113682020002B38
:10E4280014BF02210121FAE108B92520DAE1012807
:10E4380040F0608111682520F1E108B92A2025E023
:10E44800012840F0578111688C0DA405002C40F07C
:10E45800EB8189002A20E2E108B9292016E0012889
:10E4680040F0488111688C0DA405002C40F0DC8137
:10E4780089002920D3E108B92720B3E1012840F019
:10E48800398111682720CAE120B92B20FFF746FE01
:10E4980080102EE1012840F02D8111688C0DA40513
:10E4A800002C40F0C18189002B20B8E108B9262052
:10E4B80098E1012840F01E8111682620AFE108B9D3
:10E4C8002C208FE1012840F0158111688B0D9B05E8
:10E4D800002B40F0A9812C20A1E108B92D2081E171
:10E4E800012840F0078111682D2098E108B92E20F5
:10E4F80078E1012840F0FE8011682E208FE108B9EC
:10E508002F206FE1012840F0F58011682F2086E167
:10E5180008B9302066E1012840F0EC80116830200D
:10E528007DE108B933205DE1012840F0E3801168FE
:10E53800332074E108B9342054E1012840F0DA802E
:10E54800116834206BE108B960204BE1012840F0E4
:10E55800D1801168602062E108B9612042E1012898
:10E5680040F0C8801168612059E120B91C20FFF7EC
:10E57800D5FD0014BDE0012840F0BC801C20FFF749
:10E58800CDFD2968C0F3080040EA01410EE008B952
:10E598001C2018E0012840F0AD801C20FFF7BEFDCC
:10E5A8002B6800F47F01C3F3080319431C2036E1EC
:10E5B80008B9592016E1012840F09C8011685920BB
:10E5C8002DE124B90620FFF7A9FDC0B291E0012C86
:10E5D80040F090800620FFF7A1FD297820F0FF0089
:10E5E800014395E028B90620FFF798FDC0F30720FE
:10E5F8007FE001287ED10620FFF790FD2B6820F4EC
:10E608007F411B029BB282E020B9104B1B68D3F8F4
:10E618006C3109E001286DD111685A20FFE028B952
:10E628000A4B1B68D3F870312B6063E0012861D175
:10E6380011682EE060B9054B1B68D3F87031C3F33D
:10E648000E03F1E700127A0000EE85FF044B00206C
:10E6580001284FD1754B11681B68C1F30E01D3F81F
:10E66800703123F4FF4323F07F0311E020B96F4B8F
:10E678001B6893F87231D7E701283BD16B4B1B68B5
:10E68800D3F87011136821F47F011B0403F47F038E
:10E6980019435B20C3E008B95E20A3E0012829D113
:10E6A80011685E20BBE008B918209BE0012821D141
:10E6B80011681820B3E008B9192093E0012819D18E
:10E6C80011681920ABE008B95C208BE0012811D152
:10E6D80011685C20A3E008B95F2083E0012809D114
:10E6E80011685F209BE038B90620FFF717FDC0F3DB
:10E6F80007402860002070BD0128FBD10620FFF7E5
:10E708000DFD2B6820F47F011B0403F47F031943DC
:10E71800062084E00128EDD1166836B111F0C8FB57
:10E7280028600028E6D1202070BD0720FFF7F6FCFE
:10E7380020F48001072072E000287FF437AE6520BE
:10E7480050E00028D6D10720FFF7E8FCC0F381503D
:10E75800431E58425841CCE708B9522042E00128EC
:10E76800C8D1116852205AE020B9304B1B6893F881
:10E77800903159E70128BDD12C4B11681B6801F075
:10E788000F01D3F8903123F0FF0313E030B9274B82
:10E798001B68D3F89031C3F3032345E70128A9D1B7
:10E7A800224B1B68D3F89011136821F470611B0287
:10E7B80003F470631943632031E020B91B4B1B68D5
:10E7C80093F8923130E7012894D1184B1B68D3F89D
:10E7D8009011136821F47F011B0403F47F03E9E718
:10E7E80018B95020FFF79AFC83E7012882D11168F5
:10E7F800502014E018B90D4B1B68DB6914E7012899
:10E808007FF478AF1168532009E008B91520E9E7CB
:10E8180001287FF46FAF1368054915205943FFF7A6
:10E828003BFC67E7042070BD102070BD044B00203E
:10E838000071020007B5019229B9014601AA012019
:10E84800FFF7E5FC00E0082003B05DF804FB0B4689
:10E8580011B901461846DAE40820704710B50C468D
:10E86800C8B92020FFF75AFC20F004012020FFF748
:10E8780013FC84EAE472094BA2EBE4729A4204DDC9
:10E88800074A12EA240438BF1C4621022420FFF755
:10E8980003FC002010BD082010BD00BF00127A0044
:10E8A80000EE85FF0021D9E74942D7E7D6E7324B8A
:10E8B8002DE9F041DE6A9A6A350245EA12651402CA
:10E8C800C6B293F83020D86B264300279C6B2F43A1
:10E8D8000132050E000240EA1460D2B224029C63A1
:10E8E800C3E90A6783F83020D8631C46002940D062
:10E8F800042A03D939466D20FFF7CEFBA16A6C20A4
:10E90800FFF7CAFB01200DF047FBA16A6C20FFF757
:10E91800C3FB01200DF040FB00230022C4E90E23B5
:10E9280094F83030DFF85080042B09D96F20FFF7B6
:10E93800F5FBD8E90E23002632430343C8E90E232A
:10E948006E20FFF7EBFBD4E90E67034694F83020FE
:10E9580047EAE371C2F10802D200304316F0E8FC3E
:10E9680000230022C4E90E01C4E90A23002384F825
:10E9780030302846BDE8F0818015002070B54B4E38
:10E988004B4811F019FAF5684A4C6B6803F59C720C
:10E99800226203F5AA72E26103F55372A26103F5DC
:10E9A8005A72626103F56172226103F5687203F5B8
:10E9B8007670E26003F56F7203F57D7323602B6850
:10E9C800A260DB68606098472B68A069DB6898479D
:10E9D8002B686069DB6898472B682069DB68984773
:10E9E8002B68E068DB6898472B68A068DB68984765
:10E9F8002B6860685B6998472B68A0695B699847D2
:10EA08002B6860695B6998472B6820695B69984740
:10EA18002B68E0685B6998472B68A0685B69984732
:10EA28002B68206A1B6998472B68E0691B6998471F
:10EA38002B6820681B69984732691F4B1F4C1A6066
:10EA48006B68012103F53773536062691C4B202002
:10EA58001A60FFF721FB63690021597019490122E7
:10EA6800C3F8041218491A70C3F80812174B227415
:10EA78006366174B2362174BE361174BA361174B70
:10EA88006362174BA363174B6363174BA362174B60
:10EA9800E362174BA364174B6364174B6365174B0B
:10EAA8002365174BE365174BA36570BD28660208FD
:10EAB8000C4B002080150020084B0020183900203E
:10EAC800044B0020F1DF0008B9DF0008B7E80008B0
:10EAD80065E80008B5E80008B1E80008ADE80008F6
:10EAE80057E800083DE80008D5E10008FDE1000806
:10EAF80021E10008C9E10008BBE00008D5DE0008F4
:10EB08005DDE000869DE0008014B00225A6070478C
:10EB18001839002070B5184E184CF56860682B68D5
:10EB28009B6998472B68A0699B6898472B68606920
:10EB38009B6898472B6820699B6898472B68E06812
:10EB48009B6898472B68A0689B6898472B68206A41
:10EB58009B6898472B68E0699B6898472B682068F2
:10EB68009B6898472B6860689B6898473369BDE83D
:10EB78007040DB69184700BF28660208D0150020DE
:10EB88000228F8B514464CD003D880B1012835D0F6
:10EB980060E0032856D0FF285CD12F4CE36FD3F8F0
:10EBA800043298476369D3F8043298472FE0136812
:10EBB80033F003022BD113F0010F284D284E03D058
:10EBC800F3681B681B6906E0F76868693B68DB68DF
:10EBD80098473B689B6968699847206810F0020469
:10EBE80003D0F3681B681B6906E0F668A8693368F8
:10EBF800DB68984733689B69A86907E01468174D74
:10EC0800174B34B1DB681B681B69286998470020DB
:10EC1800F8BDDE6828693368DB68984733689B6904
:10EC2800F3E714680D4D0E4B1CB1DB681B681B69BC
:10EC380006E0DE68A8683368DB68984733689B6934
:10EC4800A868E3E7012011F02BFA20600028DED144
:10EC58002020F8BD0420F8BD18390020D015002068
:10EC68002866020838B50A4B0A4CDD6860682B68CC
:10EC78009B69984701200DF08FF92B6860685B69E4
:10EC88009847054B186811F0E1F9012038BD00BF1D
:10EC980028660208D0150020D850002038B50A4B45
:10ECA8000A4CDD6860682B689B69984701200DF065
:10ECB80073F92B6860685B699847054B186811F011
:10ECC800BCF9012038BD00BF28660208D015002015
:10ECD800D85000202DE9F843194D99462B680F4666
:10ECE80006469B68002140F0800090469DF8204031
:10ECF8009847144B002183F8E0022B6838469B683C
:10ED080098472B6800219B68404698472B6800214C
:10ED18009B68484698472B6801219B68204698477E
:10ED2800094B44EA09211B6806F07F0641EA0841BD
:10ED380003EB860641EA07617160BDE8F88300BF0E
:10ED4800D4500020F04D0020D850002007B5CBB299
:10ED58000093C1F30742C1F30723090EFFF7BAFF77
:10ED680003B05DF804FB70B5154C16492268157898
:10ED780011F000FA15B323681978F9B9124C94F810
:10ED88006830012B06D0032B0BBF002128210D234F
:10ED98000F2300E00B2343F0884343F0401343EA7A
:10EDA80041310420FFF7D2FFE36F012D0CBFD3F8E8
:10EDB8000432D3F80832BDE87040184770BD00BF70
:10EDC800D8500020F04D002018390020FFF7BEBFB2
:10EDD80070B5254E00F07F04331993F80C32DB0729
:10EDE80005D4224B1B6803EB8404606870BD204D7A
:10EDF80000212B6820469B6898472B6800219B6858
:10EE0800084698472B6800219B68084698472B6856
:10EE180000219B68084698472B6801219B680020C1
:10EE280098472B6800219B68204698472B6886F8EE
:10EE3800E00200219B68084698472B6800210402DD
:10EE48009B68084698472B680021204304029B686A
:10EE5800084698472B68204304029B68012100203C
:10EE68009847204370BD00BFF04D0020D8500020C7
:10EE7800D450002010B50C46FFF7AAFF206010BD43
:10EE880038B50D46044668B92020FFF7A1FF40F0C9
:10EE980004012020FFF75AFF29463720FFF756FFC5
:10EEA800204638BD082038BD38B50C460546212017
:10EEB800FFF78EFF2368C11821602846BDE8384057
:10EEC800DEE76F2970B50446154600F0BA8155D8BB
:10EED800122900F02A8127D8052900F0D88011D8F6
:10EEE800022900F0B48006D8002900F09E8001298C
:10EEF80000F0A480F0E2032900F0AF80042900F0BC
:10EF0800A680E9E20F2900F0E98006D8082900F078
:10EF1800CD800E2900F0D280DEE2102900F0E780D3
:10EF2800112900F0F380D7E2182900F0428111D8A6
:10EF3800152900F01E8106D8132900F0FF80142936
:10EF480000F00E81C8E2162900F02181172900F08F
:10EF58002781C1E21B2900F0478106D8192900F052
:10EF680031811A2900F03781B6E26D2900F04E810F
:10EF780000F255816C2900F04081ADE27D2900F056
:10EF8800048227D8752900F0AF8111D8722900F0C2
:10EF9800838106D8702900F06581712900F06B81A2
:10EFA8009AE2732900F08A81742900F0928193E231
:10EFB800782900F0D28106D8762900F0B181772926
:10EFC80000F0C38188E2792900F0CF817C2900F024
:10EFD800D48181E2882900F0218211D8842900F0A7
:10EFE800058206D87E2900F0D881812900F0EC81BD
:10EFF80072E2852900F0FF81862900F007826BE222
:10F00800C82900F0388106D8892900F019828A2990
:10F0180000F02D8260E2D42900F04682D62900F063
:10F028004E82D12940F0588234E208B9372033E2C1
:10F03800012840F0B981116837204AE208B9212037
:10F048002AE2012840F0B0811168212041E25CB930
:10F058002420FFF7BDFE0012A5E108B922201BE21B
:10F06800012C00F039829FE1012C40F09D81296834
:10F07800A14B81EAE172A2EBE1729A4204DD9F4A58
:10F0880012EA210138BF19460902242021E208B9F1
:10F09800282055E0012840F0878111688C0DA405CF
:10F0A800002C40F01B828900282012E20028D7D1CA
:10F0B8000F20FFF78DFE00F0010074E120B9202039
:10F0C800FFF786FE40006EE1012840F06D8113686D
:10F0D8002020002B14BF02210121FAE108B92520C4
:10F0E800DAE1012840F0608111682520F1E108B9D2
:10F0F8002A2025E0012840F0578111688C0DA405CD
:10F10800002C40F0EB8189002A20E2E108B929208F
:10F1180016E0012840F0488111688C0DA405002CE8
:10F1280040F0DC8189002920D3E108B92720B3E128
:10F13800012840F0398111682720CAE120B92B2025
:10F14800FFF746FE80102EE1012840F02D8111685E
:10F158008C0DA405002C40F0C18189002B20B8E15A
:10F1680008B9262098E1012840F01E811168262060
:10F17800AFE108B92C208FE1012840F01581116812
:10F188008B0D9B05002B40F0A9812C20A1E108B92B
:10F198002D2081E1012840F0078111682D2098E198
:10F1A80008B92E2078E1012840F0FE8011682E2051
:10F1B8008FE108B92F206FE1012840F0F580116830
:10F1C8002F2086E108B9302066E1012840F0EC8064
:10F1D800116830207DE108B933205DE1012840F055
:10F1E800E3801168332074E108B9342054E1012820
:10F1F80040F0DA80116834206BE108B960204BE1F7
:10F20800012840F0D1801168602062E108B96120CE
:10F2180042E1012840F0C8801168612059E120B915
:10F228001C20FFF7D5FD0014BDE0012840F0BC808C
:10F238001C20FFF7CDFD2968C0F3080040EA014112
:10F248000EE008B91C2018E0012840F0AD801C2011
:10F25800FFF7BEFD2B6800F47F01C3F308031943D1
:10F268001C2036E108B9592016E1012840F09C809D
:10F27800116859202DE124B90620FFF7A9FDC0B275
:10F2880091E0012C40F090800620FFF7A1FD29783D
:10F2980020F0FF00014395E028B90620FFF798FD0C
:10F2A800C0F307207FE001287ED10620FFF790FDFC
:10F2B8002B6820F47F411B029BB282E020B9104BDF
:10F2C8001B68D3F86C3109E001286DD111685A2008
:10F2D800FFE028B90A4B1B68D3F870312B6063E054
:10F2E800012861D111682EE060B9054B1B68D3F87D
:10F2F8007031C3F30E03F1E700127A0000EE85FFC8
:10F30800D850002001284FD1754B11681B68C1F3F4
:10F318000E01D3F8703123F4FF4323F07F0311E08B
:10F3280020B96F4B1B6893F87231D7E701283BD19E
:10F338006B4B1B68D3F87011136821F47F011B0411
:10F3480003F47F0319435B20C3E008B95E20A3E000
:10F35800012829D111685E20BBE008B918209BE07C
:10F36800012821D111681820B3E008B9192093E0C9
:10F37800012819D111681920ABE008B95C208BE08D
:10F38800012811D111685C20A3E008B95F2083E04F
:10F39800012809D111685F209BE038B90620FFF7E2
:10F3A80017FDC0F307402860002070BD0128FBD17D
:10F3B8000620FFF70DFD2B6820F47F011B0403F4E2
:10F3C8007F031943062084E00128EDD1166836B181
:10F3D80010F066FE28600028E6D1202070BD0720C6
:10F3E800FFF7F6FC20F48001072072E000287FF484
:10F3F80037AE652050E00028D6D10720FFF7E8FC9B
:10F40800C0F38150431E58425841CCE708B95220F6
:10F4180042E00128C8D1116852205AE020B9304B87
:10F428001B6893F8903159E70128BDD12C4B11681E
:10F438001B6801F00F01D3F8903123F0FF0313E0AC
:10F4480030B9274B1B68D3F89031C3F3032345E742
:10F458000128A9D1224B1B68D3F89011136821F415
:10F4680070611B0203F470631943632031E020B913
:10F478001B4B1B6893F8923130E7012894D1184B45
:10F488001B68D3F89011136821F47F011B0403F45F
:10F498007F03E9E718B95020FFF79AFC83E70128B2
:10F4A80082D11168502014E018B90D4B1B68DB6934
:10F4B80014E701287FF478AF1168532009E008B9F0
:10F4C8001520E9E701287FF46FAF13680549152077
:10F4D8005943FFF73BFC67E7042070BD102070BD5F
:10F4E800D85000200071020007B5019229B90146E1
:10F4F80001AA0120FFF7E5FC00E0082003B05DF851
:10F5080004FB0B4611B901461846DAE40820704797
:10F5180010B50C46C8B92020FFF75AFC20F00401AA
:10F528002020FFF713FC84EAE472094BA2EBE47293
:10F538009A4204DD074A12EA240438BF1C46210215
:10F548002420FFF703FC002010BD082010BD00BFD9
:10F5580000127A0000EE85FF0021D9E74942D7E77B
:10F56800D6E7314B2DE9F041DE6A9A6A350245EA61
:10F5780012651402C6B293F83020D86B26430027D0
:10F588009C6B2F430132050E000240EA1460D2B290
:10F5980024029C63C3E90A6783F83020D8631C46B9
:10F5A80000293DD0042A03D939466D20FFF7CEFB48
:10F5B800A16A6C20FFF7CAFB01200CF0EDFCA16AE0
:10F5C8006C20FFF7C3FB00230022C4E90E2394F844
:10F5D8003030DFF85480042B09D96F20FFF7F8FB8F
:10F5E800D8E90E23002632430343C8E90E236E20D0
:10F5F800FFF7EEFBD4E90E67034694F8302047EA9C
:10F60800E371C2F10802D200304315F091FE0023E5
:10F618000022C4E90E01C4E90A23002384F830302B
:10F628002846BDE8F08100BFD015002070B54B4ECC
:10F638004B4810F0B9FCF5684A4C6B6803F59C72AE
:10F64800226203F5AA72E26103F55372A26103F51F
:10F658005A72626103F56172226103F5687203F5FB
:10F668007670E26003F56F7203F57D7323602B6893
:10F67800A260DB68606098472B68A069DB689847E0
:10F688002B686069DB6898472B682069DB689847B6
:10F698002B68E068DB6898472B68A068DB689847A8
:10F6A8002B6860685B6998472B68A0695B69984715
:10F6B8002B6860695B6998472B6820695B69984784
:10F6C8002B68E0685B6998472B68A0685B69984776
:10F6D8002B68206A1B6998472B68E0691B69984763
:10F6E8002B6820681B69984732691F4B1F4C1A60AA
:10F6F8006B68012103F53773536062691C4B202046
:10F708001A60FFF723FB6369002159701949012228
:10F71800C3F8041218491A70C3F80812174B227458
:10F728006366174B2362174BE361174BA361174BB3
:10F738006362174BA363174B6363174BA362174BA3
:10F74800E362174BA364174B6364174B6365174B4E
:10F758002365174BE365174BA36570BD2866020840
:10F76800F04D0020D0150020D4500020183900207A
:10F77800D8500020A5EC00086DEC00086BF50008D7
:10F7880019F5000869F5000865F5000861F5000835
:10F798000BF50008F1F4000889EE0008B1EE000846
:10F7A800D5ED00087DEE00086FED000889EB000834
:10F7B80011EB00081DEB000800207047012070477E
:10F7C800014B00225A6070471839002010B50C46CA
:10F7D8000CF048FF206010BD0CF070BF38B50D4626
:10F7E800044620B910F091FD2860204638BD082055
:10F7F80038BDF0B5074689B004AC374D102200215A
:10F80800204616F043FD2B68FB1A092B06D9AA6877
:10F81800642353436B600023AB602F60AB68002008
:10F828000133AB602D4B33F8081CA3F10806727A3C
:10F838000291B11D0191B1880091394610F080FE06
:10F848000FF0C4FC20B10022114610460FF04AFD0B
:10F858000FF0B6FC00283CD00FF032FD032838D852
:10F86800DFE800F0120A021D002010F071FD04907C
:10F87800002010F074FD10E0002010F03AFD049014
:10F88800002010F042FD08E07189002010F0C9FC4A
:10F8980071890490002010F0CEFC059015E0EB680B
:10F8A8005BB1012B11D164230493C82305934FF452
:10F8B800967306934FF4C87306E00A23049314233F
:10F8C80005931E2306932823079394E80F000FF04F
:10F8D80097FC09B0F0BD00BF1C160020E4500020C2
:10F8E80010B5044620B9096810F021FD204610BD66
:10F8F800082010BD10B5044618B910F00BFD2046BD
:10F9080010BD082010BD10B5044618B910F0E4FC6D
:10F91800204610BD082010BD0021F4E74942F2E757
:10F92800F1E7022804BF0C4B93F8D00020B90B4B29
:10F93800DB681B689B690AE001280BD1064B93F82A
:10F94800D030012B06D1054BDB681B685B69044A84
:10F9580010681847704700BF183900202866020849
:10F96800343A002010B50020FFF7DBFFBDE8104057
:10F97800034B044ADB6810681B689B69184700BF83
:10F9880028660208343A0020043A38B504461D4671
:10F998000846FB2A00F28E87DFE812F0FC008C078D
:10F9A8008C078C078C078C078C070C0113018C07BC
:10F9B80017018C078C078C078C078C078C078C0722
:10F9C8008C078C078C078C078C078C078C078C0797
:10F9D8008C078C078C078C078C078C078C078C0787
:10F9E8008C078C078C078C078C078C078C078C0777
:10F9F8008C078C078C078C071B012E018C07410193
:10FA080054018C078C078C078C078C078C078C0794
:10FA18008C078C078C078C078C078C078C078C0746
:10FA28008C078C078C078C078C078C078C078C0736
:10FA38008C078C078C078C078C078C078C078C0726
:10FA48008C078C078C078C078C078C078C078C0716
:10FA58008C078C078C078C078C078C07670178014B
:10FA6800850192019F01AC01B901C601D301E001F2
:10FA7800ED01FA01080216022402320240024B028A
:10FA880056028C0761026C02770282028D029C0288
:10FA9800AB02BA02C4028C078C078C07CE02D702CD
:10FAA800E002EB02F6028C078C078C07FF020803C2
:10FAB80011038C078C078C078C078C078C078C0725
:10FAC8001C03270332033D038C078C078C078C0724
:10FAD8008C078C07480353035E03690374038C0780
:10FAE8008C078C078C078C077F038A039D03B00360
:10FAF800B903C803D303DF03EA03F20300040D04C8
:10FB08001A042704340441044E045B048C07680477
:10FB180076048C049904A704B404C104CE04DB045D
:10FB2800E804F704060515052405330542055405C0
:10FB380063057205810590059F05AE05BD05CC05D9
:10FB4800DB05EA05F905080616068C078C078C07FD
:10FB58008C078C078C078C078C078C078C078C0705
:10FB6800240633064206510660066F067E068D0699
:10FB78009C06AA06B806C606D406E206F006FE06E5
:10FB88000C0719072607330740074D075E0771075B
:10FB98007A0784072CB960200CF064FD28602046A1
:10FBA80038BD012C40F08886296860200CF086FD5D
:10FBB800002038BD002C40F0818600242C602046AF
:10FBC80038BD002CF9D0002038BD002CF5D000201D
:10FBD80038BD3CB9214608200CF0CFFD00B22860A2
:10FBE800204638BD012C40F06B862A880021082069
:10FBF8000CF0F5FD002038BD3CB9214609200CF079
:10FC0800BCFD00B22860204638BD012C40F05A8661
:10FC18002A88002109200CF0E2FD002038BD3CB9FB
:10FC2800012108200CF0A9FD00B22860204638BD4B
:10FC3800012C40F049862A88214608200CF0CFFD87
:10FC4800002038BD3CB9012109200CF096FD00B216
:10FC58002860204638BD012C40F038862A88214685
:10FC680009200CF0BCFD002038BD54B90121032047
:10FC78000CF024FD214602200CF07FFD2860204670
:10FC880038BD012C14BF0020042038BD002CF8D149
:10FC9800012103200CF012FD012102200CF06DFD62
:10FCA8002860204638BD002CEBD1022103200CF03F
:10FCB80005FD214602200CF060FD2860204638BD75
:10FCC800002CDED1214603200CF0F8FC214602204E
:10FCD8000CF053FD2860204638BD002CD1D12146B8
:10FCE80003200CF0EBFC012102200CF046FD2860FB
:10FCF800204638BD002CC4D1032108460CF0DEFC98
:10FD0800214602200CF039FD2860204638BD002C21
:10FD1800B7D1042103200CF0D1FC214602200CF0BD
:10FD28002CFD2860204638BD002CAAD104210320D0
:10FD38000CF0C4FC012102200CF01FFD28602046B5
:10FD480038BD002C9DD1052103200CF0B7FC2146BD
:10FD580002200CF012FD2860204638BD002C90D1FE
:10FD6800052103200CF0AAFC012102200CF005FD5E
:10FD78002860204638BD002C83D1062103200CF0D2
:10FD88009DFC214602200CF0F8FC2860204638BD76
:10FD9800002C7FF476AF072103200CF08FFC21465E
:10FDA80002200CF0EAFC2860204638BD002C7FF4C5
:10FDB80068AF072103200CF081FC012102200CF020
:10FDC800DCFC2860204638BD002C7FF45AAF08219F
:10FDD80003200CF073FC214602200CF0CEFC2860B6
:10FDE800204638BD002C7FF44CAF082103200CF0CE
:10FDF80065FC012102200CF0C0FC2860204638BDBB
:10FE0800002C7FF43EAF092103200CF057FC21465B
:10FE180002200CF0B2FC2860204638BD002C7FF48C
:10FE280030AF214612200CF0A8FC00B22860204612
:10FE380038BD002C7FF425AF012112200CF09DFC69
:10FE480000B22860204638BD002C7FF41AAF214646
:10FE580013200CF092FC00B22860204638BD002C1C
:10FE68007FF40FAF214615200CF087FC00B2286004
:10FE7800204638BD002C7FF404AF012115200CF07A
:10FE88007CFC00B22860204638BD002C7FF4F9AE17
:10FE9800214616200CF071FC00B22860204638BDBF
:10FEA800002C7FF4EEAE012116200CF066FC00B2A7
:10FEB8002860204638BD002C7FF4E3AE0A210320D9
:10FEC8000CF0FCFB214602200CF057FC00B2286025
:10FED800204638BD002C7FF4D4AE0A2103200CF054
:10FEE800EDFB012102200CF048FC00B228602046FE
:10FEF80038BD002C7FF4C5AE0B2103200CF0DEFBCF
:10FF0800214602200CF039FC00B22860204638BD9A
:10FF1800002C7FF4B6AE214606200CF02EFC28609B
:10FF2800204638BD002C7FF4ACAE012106200CF031
:10FF380024FC2860204638BD002C7FF4A2AE412066
:10FF48000CF090FB2860204638BD002C7FF499AE59
:10FF580042200CF087FB2860204638BD002C7FF437
:10FF680090AE012146200CF008FC00B22860204623
:10FF780038BD002C7FF485AE214646200CF0FDFBF1
:10FF880000B22860204638BD002C7FF47AAE4720A6
:10FF98000CF068FB2860204638BD002C7FF471AE59
:10FFA80021200CF05FFB2860204638BD002C7FF430
:10FFB80068AE22200CF056FB2860204638BD002C85
:10FFC8007FF45FAE214623200CF0D7FB00B22860F7
:10FFD800204638BD002C7FF454AE27200CF042FB9D
:10FFE80020F07F402860204638BD002C7FF449AEC1
:08FFF80028200CF037FB20F07B
:020000040801F1
:100000007F402860204638BD002C7FF43EAE0121A1
:100010002A200CF0B6FB00B22860204638BD002C28
:100020007FF433AE21462A200CF0ABFB00B22860EF
:10003000204638BD002C7FF428AE214639200CF034
:10004000A0FB00B22860204638BD002C7FF41DAE16
:10005000012139200CF095FB00B22860204638BD04
:10006000002C7FF412AE21463D200CF08AFB00B23A
:100070002860204638BD002C7FF407AE21463F2083
:100080000CF07FFB00B22860204638BD002C7FF4C6
:10009000FCAD21463A200CF074FB00B228602046EB
:1000A00038BD002C7FF4F1AD214653200CF069FBE4
:1000B00000B22860204638BD3CB9012164200CF014
:1000C00060FB00B22860204638BD012C40F004845B
:1000D0002A88214664200CF086FB002038BD3CB9FC
:1000E000214664200CF04DFB00B22860204638BD4C
:1000F000012C40F0F3832A88002164200CF073FB6C
:10010000002038BD002C7FF4C0AD66200CF0AEFAA4
:100110002860204638BD2CB968200CF0A7FA28606A
:10012000204638BD012C40F0DB83296810F0F6F83A
:10013000002038BD002C7FF4A8AD012169200CF00F
:1001400020FB00B22860204638BD002C7FF49DAD16
:10015000BD4B03EB0113598910F071F8286020465C
:1001600038BD002C7FF491AD214669200CF009FBCD
:1001700000B22860204638BD002C7FF486AD10F018
:10018000C8F82860204638BD24B910F0ECF8286083
:10019000204638BD012C40F0A583296810F0DFF817
:1001A000002038BD002C7FF470AD21466D200CF08E
:1001B00089FA6C200CF05AFA2860204638BD002CD1
:1001C0007FF463AD01216D200CF07CFA6C200CF003
:1001D0004DFA2860204638BD002C7FF456AD022130
:1001E0006D200CF06FFA6C200CF040FA286020466D
:1001F00038BD002C7FF449AD03216D200CF062FA6C
:100200006C200CF033FA2860204638BD002C7FF4B7
:100210003CAD04216D200CF055FA6C200CF026FA50
:100220002860204638BD002C7FF42FAD05216D20BD
:100230000CF048FA6C200CF019FA2860204638BD02
:10024000002C7FF422AD06216D200CF03BFA6C20CF
:100250000CF00CFA2860204638BD002C7FF415AD58
:1002600007216D200CF02EFA6C200CF0FFF92860AD
:10027000204638BD24B90FF0B1FF2860204638BDB4
:10028000012C40F0318329680FF09AFF002038BD1F
:1002900044B96D4B03EB011359890FF0C6FF286079
:1002A000204638BD012C40F02183674B2A6803EBC0
:1002B000011359890FF0A7FF002038BD002C7FF4EF
:1002C000E4AC01216F200CF0FDF96E200CF0CEF9AA
:1002D0002860204638BD24B910F00FF82860204669
:1002E00038BD012C40F0048329680FF0F9FF00208D
:1002F00038BD002C7FF4C9AC03216F200CF0E2F96B
:100300006E200CF0B3F92860204638BD002C7FF435
:10031000BCAC04216F200CF0D5F96E200CF0A6F9CE
:100320002860204638BD002C7FF4AFAC05216F203B
:100330000CF0C8F96E200CF099F92860204638BD01
:10034000002C7FF4A2AC06216F200CF0BBF96E20CC
:100350000CF08CF92860204638BD002C7FF495AC59
:1003600007216F200CF0AEF96E200CF07FF92860A9
:10037000204638BD002C7FF488AC08216F200CF09B
:10038000A1F921466E200CF0FCF900B2286020464D
:1003900038BD002C7FF479AC08216F200CF092F965
:1003A00001216E200CF0EDF900B22860204638BD26
:1003B000002C7FF46AAC09216F200CF083F92146F0
:1003C0006E200CF0DEF900B22860204638BD002C0B
:1003D0007FF45BAC0A216F200CF074F921466E208B
:1003E0000CF0CFF900B22860204638BD002C7FF415
:1003F0004CAC0A216F200CF065F901216E200CF045
:10040000C0F900B22860204638BD002C7FF43DAC16
:100410000B216F200CF056F921466E200CF0B1F93B
:1004200000B22860204638BD002C7FF42EAC0B2192
:100430006F200CF047F901216E200CF0A2F900B2F8
:100440002860204638BD00BFDC500020002C7FF41F
:100450001CAC0C216F200CF035F921466E200CF0FD
:1004600090F900B22860204638BD002C7FF40DAC16
:100470000C216F200CF026F901216E200CF081F97F
:1004800000B22860204638BD002C7FF4FEAB0D2161
:100490006F200CF017F921466E200CF072F900B2B3
:1004A0002860204638BD002C7FF4EFAB0D216F2073
:1004B0000CF008F901216E200CF063F900B22860FD
:1004C000204638BD002C7FF4E0AB0E216F200CF0ED
:1004D000F9F821466E200CF054F900B2286020464D
:1004E00038BD002C7FF4D1AB0E216F200CF0EAF860
:1004F00001216E200CF045F900B22860204638BD7D
:10050000002C7FF4C2AB0F216F200CF0DBF82146EA
:100510006E200CF036F900B22860204638BD002C61
:100520007FF4B3AB0F216F200CF0CCF801216E20CB
:100530000CF027F900B22860204638BD002C7FF46B
:10054000A4AB10216F200CF0BDF821466E200CF0FA
:1005500018F900B22860204638BD002C7FF495AB16
:1005600011216F200CF0AEF821466E200CF009F935
:1005700000B22860204638BD002C7FF486AB1121E4
:100580006F200CF09FF801216E200CF0FAF800B2F9
:100590002860204638BD002C7FF477AB12216F20F5
:1005A0000CF090F821466E200CF0EBF800B22860B9
:1005B000204638BD002C7FF468AB13216F200CF06F
:1005C00081F821466E200CF0DCF82860204638BD0A
:1005D000002C7FF45AAB13216F200CF073F801212B
:1005E0006E200CF0CEF82860204638BD002C7FF439
:1005F0004CABC0216F200CF065F821466E200CF04A
:10060000C0F800B22860204638BD002C7FF43DAB16
:10061000C0216F200CF056F801216E200CF0B1F8CB
:1006200000B22860204638BD002C7FF42EABC121DB
:100630006F200CF047F821466E200CF0A2F800B2B3
:100640002860204638BD002C7FF41FABC1216F20ED
:100650000CF038F801216E200CF093F800B22860FD
:10066000204638BD002C7FF410ABC2216F200CF067
:1006700029F821466E200CF084F800B2286020464C
:1006800038BD002C7FF401ABC2216F200CF01AF8AA
:1006900001216E200CF075F800B22860204638BDAC
:1006A000002C7FF4F2AAC3216F200CF00BF8214636
:1006B0006E200CF066F800B22860204638BD002C91
:1006C0007FF4E3AAC3216F200BF0FCFF01216E2011
:1006D0000CF057F800B22860204638BD002C7FF49B
:1006E000D4AAC4216F200BF0EDFF21466E200CF040
:1006F00048F82860204638BD002C7FF4C6AAC421E3
:100700006F200BF0DFFF01216E200CF03AF828601B
:10071000204638BD002C7FF4B8AAC5216F200BF00D
:10072000D1FF21466E200CF02CF82860204638BD01
:10073000002C7FF4AAAAC5216F200BF0C3FF012172
:100740006E200CF01EF82860204638BD002C7FF487
:100750009CAAC6216F200BF0B5FF21466E200CF03D
:1007600010F82860204638BD002C7FF48EAAC621E0
:100770006F200BF0A7FF01216E200CF002F828601B
:10078000204638BD002C7FF480AAC7216F200BF0D3
:1007900099FF21466E200BF0F4FF2860204638BDFB
:1007A000002C7FF472AAC7216F200BF08BFF012170
:1007B0006E200BF0E6FF2860204638BD002C7FF449
:1007C00064AAC8216F200BF07DFF6E200BF04EFF56
:1007D0002860204638BD002C7FF457AAC9216F201D
:1007E0000BF070FF6E200BF041FF2860204638BDF3
:1007F000002C7FF44AAACA216F200BF063FF6E2001
:100800000BF034FF2860204638BD002C7FF43DAA51
:10081000CB216F200BF056FF6E200BF027FF2860D6
:10082000204638BD24B9374B2046DB682B6038BDE5
:10083000012C5FD12A68334B0020DA6038BD34B90F
:10084000314A02EB0110438920462B6038BD012C50
:1008500052D12D4A2B6802EB01104381002038BD94
:1008600034B9294A02EB0110437A20462B6038BD87
:10087000012C43D1254A287802EB0112511C0FF0BC
:100880006DFE002038BD002C3AD11F4A02EB01104A
:10089000037A20462B6038BD002C7FF4F6A91A4A53
:1008A00002EB0110C38820462B6038BD002C7FF47A
:1008B000ECA9144B20465B682B6038BD042038BD82
:1008C000002038BD002038BD002038BD002038BDD4
:1008D000002038BD002038BD002038BD002038BDC4
:1008E000002038BD002038BD002038BD002038BDB4
:1008F000002038BD002038BD002038BD002038BDA4
:10090000002038BD1C160020DC500020E4500020E0
:1009100010B413460446084619B9224610BCFFF726
:1009200037B8082010BC70470120704707B5019206
:1009300029B9024601AB0120FFF72AF800E00820A0
:1009400003B05DF804FB08460BF090BE0846114664
:100950000BF0B8BE084611460BF013BF084611460F
:100960001A460BF040BF38B5274B284DDC6860684D
:100970002368C8302860DB689847236828685B696B
:100980009847234B23495A6901200A602249C2F83B
:1009900004122249C2F80812002111705170204A35
:1009A00018741A621F4ADA611F4A9A611F4A5A6212
:1009B0001F4ADA641F4A9A631F4A5A631F4A9A629F
:1009C0001F4ADA621F4A9A641F4A5A641F4A5A65CC
:1009D0001F4A1A651F4A1A661F4ADA651F4A9A6536
:1009E0003222DA6040F28A229A601D4B4FF47A720A
:1009F0009A8041F2707259721A604FF480725A8173
:100A0000BDE83840FEF791BF28660208343A00205E
:100A100018390020EC50002029090108C5F700080A
:100A20000FF9000829F9000825F9000821F9000844
:100A3000E5F70008110901082D090108FDF8000873
:100A4000E9F80008E1F70008D5F70008FBF700080F
:100A5000C1F700082BF90008C9F700086DF9000874
:100A6000DC5000200020704701207047014B00221D
:100A70005A6070471839002010B50C460BF0F6FD8F
:100A8000206010BD0BF01EBE38B50D46044620B9DF
:100A90000FF0B0FE2860204638BD082038BD30B5C4
:100AA000054689B004AC10220021204615F0F2FB67
:100AB000374B1A68AA1A092A06D9996864224A4348
:100AC0005A6000229A601D609A6801329A60314B28
:100AD00033F8060C5A780290981E019033F8041CE3
:100AE0000020009129460FF0A1FF0EF073FB20B10A
:100AF0000022114610460EF0F9FB0EF065FB0028AF
:100B000044D00EF0E1FB032840D8DFE800F0120AE1
:100B1000022800200FF091FE049000200FF094FEB8
:100B20001BE000200FF063FE049000200FF062FE37
:100B300013E000216F200BF0C5FD6E200BF096FD39
:100B40000121049069200BF01CFE0021054669205C
:100B50000BF017FE2DB200B22844059012E076206B
:100B60000BF084FD6423C0F30222C0F302505A4309
:100B70004343A3F52F730593074B04920693A3F504
:100B8000FA63079394E80F000EF03EFB09B030BD06
:100B900038160020E2500020F0D8FFFF10B50446C0
:100BA00020B909680FF038FE204610BD082010BD9E
:100BB00010B5044618B90FF022FE204610BD0820DB
:100BC00010BD10B5044618B90FF004FE204610BD44
:100BD000082010BD0021F4E74942F2E7F1E70228BE
:100BE00004BF0C4B93F8D00020B90B4BDB681B689B
:100BF0009B690AE001280BD1064B93F8D030012BFA
:100C000006D1054BDB681B685B69044A106818470E
:100C1000704700BF1839002028660208343A0020C7
:100C200010B50020FFF7DBFFBDE81040034B044A7E
:100C3000DB6810681B689B69184700BF28660208BC
:100C4000343A0020043A38B504461D460846FB2ACB
:100C500001F21D80DFE812F0FC001B081B081B08D6
:100C60001B081B081B080C0113011B0817011B089C
:100C70001B081B081B081B081B081B081B081B085C
:100C80001B081B081B081B081B081B081B081B084C
:100C90001B081B081B081B081B081B081B081B083C
:100CA0001B081B081B081B081B081B081B081B082C
:100CB0001B081B081B012D011B083F0152011B08CB
:100CC0001B081B081B081B081B081B081B081B080C
:100CD0001B081B081B081B081B081B081B081B08FC
:100CE0001B081B081B081B081B081B081B081B08EC
:100CF0001B081B081B081B081B081B081B081B08DC
:100D00001B081B081B081B081B081B081B081B08CB
:100D10001B081B081B081B086501760183011B08C3
:100D20001B081B081B081B081B081B081B0890013D
:100D30009D01AA011B081B08B701C101CB011B08BB
:100D4000D501DF01E9011B08F30101021B080F02B5
:100D500019021B081B081B0823022C023502400243
:100D60004B021B081B081B0854025D0266021B088D
:100D70001B081B081B081B081B081B0871027C02B0
:100D8000870292029D02B502CD02E80203031E0310
:100D9000380343034E03590364031B081B081B0855
:100DA0001B081B086F037A038D03A003A903B2037A
:100DB000BD03CA03D503DD03EC03F90306041304E2
:100DC00020042D043A0447041B08540462047A04E6
:100DD00087049404A104AE04BB04C804D504E4044D
:100DE000F3040205110520052F0540054F055E059A
:100DF0006D057C058B059A05A905B805C705D605BF
:100E0000E505F40502061B081006280640065B06E9
:100E100076069106AC061B081B081B08B906C80617
:100E2000D706E606F50604071307220731073F0732
:100E30004D075B076907770785079307A107AE078B
:100E4000BB07C8071B08D507E807FE0708081308F3
:100E50002CB960200BF00AFC2860204638BD012C1C
:100E600040F01787296860200BF02CFC002038BD6B
:100E7000002C40F0108700242C60204638BD002C48
:100E8000F9D0002038BD002CF5D0002038BD34B991
:100E9000214608200BF075FC2860204638BD012C47
:100EA00040F0FB862A88002108200BF09CFC0020E3
:100EB00038BD34B9214609200BF063FC2860204678
:100EC00038BD012C40F0EB862A88002109200BF068
:100ED0008AFC002038BD3CB9012108200BF051FCF0
:100EE00000B22860204638BD012C40F0DA862A88FE
:100EF000214608200BF077FC002038BD3CB90121C9
:100F000009200BF03EFC00B22860204638BD012CC1
:100F100040F0C9862A88214609200BF064FC002095
:100F200038BD54B9012103200BF0CCFB214602202F
:100F30000BF027FC2860204638BD012C14BF002090
:100F4000042038BD002CF8D1012103200BF0BAFB9E
:100F5000012102200BF015FC2860204638BD002C32
:100F6000EBD1022103200BF0ADFB214602200BF058
:100F700008FC2860204638BD002CDED10221032069
:100F80000BF0A0FB012102200BF0FBFB28602046A8
:100F900038BD002CD1D1032108460BF093FB012171
:100FA00002200BF0EEFB2860204638BD002CC4D197
:100FB000032108460BF086FB214602200BF0E1FBE3
:100FC0002860204638BD002CB7D1214612200BF0F6
:100FD000D8FB00B22860204638BD002CADD10121DD
:100FE00012200BF0CEFB00B22860204638BD002C4A
:100FF000A3D1214613200BF0C4FB00B22860204689
:1010000038BD002C99D1214615200BF0BAFB00B257
:101010002860204638BD002C8FD1012115200BF00F
:10102000B0FB00B22860204638BD002C85D1214697
:1010300016200BF0A6FB00B22860204638BD002C1D
:101040007FF47BAF214603200BF03CFB21460220BE
:101050000BF097FB2860204638BD002C7FF46DAF65
:10106000214603200BF02EFB012102200BF089FB0F
:101070002860204638BD002C7FF45FAF21460B204E
:101080000BF07FFB2860204638BD002C7FF455AF65
:1010900001210B200BF075FB2860204638BD002C89
:1010A0007FF44BAF41200BF0E1FA2860204638BDB9
:1010B000002C7FF442AF42200BF0D8FA2860204683
:1010C00038BD002C7FF439AF012146200BF059FBCD
:1010D00000B22860204638BD002C7FF42EAF214698
:1010E00046200BF04EFB00B22860204638BD002C95
:1010F0007FF423AF47200BF0B9FA2860204638BDB3
:10110000002C7FF41AAF21200BF0B0FA28602046A3
:1011100038BD002C7FF411AF22200BF0A7FA286015
:10112000204638BD002C7FF408AF214623200BF069
:1011300028FB00B22860204638BD002C7FF4FDAEAD
:1011400027200BF093FA20F07F402860204638BD1E
:10115000002C7FF4F2AE28200BF088FA20F07F40BC
:101160002860204638BD002C7FF4E7AE01212A20FC
:101170000BF007FB00B22860204638BD002C7FF43E
:10118000DCAE21462A200BF0FCFA00B22860204693
:1011900038BD4CB9D4216F200BF094FA6E200BF0BF
:1011A00065FA2860204638BD012C40F07E85D421A8
:1011B0006F200BF087FA29686E200BF083FA00206D
:1011C00038BD4CB9D5216F200BF07CFA6E200BF0A6
:1011D0004DFA2860204638BD012C40F06885D521A5
:1011E0006F200BF06FFA29686E200BF06BFA00206D
:1011F00038BD5CB9D6216F200BF064FA21466E2011
:101200000BF0BFFA00B22860204638BD012C40F038
:101210005085D6216F200BF055FA2A8800216E20C8
:101220000BF0E1FA002038BD5CB9D6216F200BF03D
:1012300049FA01216E200BF0A4FA00B22860204682
:1012400038BD012C40F03785D6216F200BF03AFADB
:101250002A8821466E200BF0C6FA002038BD5CB902
:10126000D7216F200BF02EFA21466E200BF089FA61
:1012700000B22860204638BD012C40F01E85D721E1
:101280006F200BF01FFA2A8800216E200BF0ABFABA
:10129000002038BD54B9D7216F200BF013FA01217B
:1012A0006E200BF06EFA2860204638BD012C40F00D
:1012B0000685D7216F200BF005FA2A8821466E207B
:1012C0000BF091FA002038BD002C7FF436AE214699
:1012D00039200BF056FA00B22860204638BD002CA9
:1012E0007FF42BAE012139200BF04BFA00B22860BD
:1012F000204638BD002C7FF420AE21463D200BF067
:1013000040FA00B22860204638BD002C7FF415AEAC
:1013100021463F200BF035FA00B22860204638BD48
:10132000002C7FF40AAE21463A200BF02AFA00B2D4
:101330002860204638BD002C7FF4FFAD21465320A5
:101340000BF01FFA00B22860204638BD3CB90121DD
:1013500064200BF016FA00B22860204638BD012C3C
:1013600040F0AF842A88214664200BF03CFA00202C
:1013700038BD3CB9214664200BF003FA00B2286066
:10138000204638BD012C40F09E842A88002164202C
:101390000BF029FA002038BD002C7FF4CEAD66207A
:1013A0000BF064F92860204638BD002C7FF4C5ADF1
:1013B00068200BF05BF92860204638BD002C7FF4D4
:1013C000BCAD012169200BF0DCF900B22860204699
:1013D00038BD002C7FF4B1ADBE4A0C2303FB0123C2
:1013E00019890FF0A6F92860204638BD002C7FF43B
:1013F000A4AD214669200BF0C4F900B22860204654
:1014000038BD002C7FF499AD0FF0F4F92860204628
:1014100038BD24B90FF018FA2860204638BD012CD9
:1014200040F0538429686B200BF04CF9002038BD44
:10143000002C7FF482AD21466D200BF043F96C2027
:101440000BF014F92860204638BD002C7FF475ADF0
:1014500001216D200BF036F96C200BF007F92860A4
:10146000204638BD002C7FF468AD02216D200BF0C2
:1014700029F96C200BF0FAF82860204638BD002CC2
:101480007FF45BAD03216D200BF01CF96C200BF099
:10149000EDF82860204638BD002C7FF44EAD0421C5
:1014A0006D200BF00FF96C200BF0E0F8286020465F
:1014B00038BD002C7FF441AD05216D200BF002F901
:1014C0006C200BF0D3F82860204638BD002C7FF448
:1014D00034AD06216D200BF0F5F86C200BF0C6F84A
:1014E0002860204638BD002C7FF427AD07216D20F1
:1014F0000BF0E8F86C200BF0B9F82860204638BDF6
:1015000024B90FF0E5F82860204638BD012C40F0E2
:10151000DE8329680FF0CEF8002038BD4CB96D4A43
:101520000C2303FB012319890FF0F9F828602046EA
:1015300038BD012C40F0CD83664A0C2303FB012308
:101540002A6819890FF0D9F8002038BD002C7FF4E3
:10155000F4AC01216F200BF0B5F86E200BF086F88B
:101560002860204638BD002C7FF4E7AC02216F20B4
:101570000BF0A8F86E200BF079F82860204638BDF3
:10158000002C7FF4DAAC03216F200BF09BF86E2067
:101590000BF06CF82860204638BD002C7FF4CDACF1
:1015A00004216F200BF08EF86E200BF05FF828609E
:1015B000204638BD002C7FF4C0AC05216F200BF015
:1015C00081F86E200BF052F82860204638BD002CC0
:1015D0007FF4B3AC06216F200BF074F86E200BF093
:1015E00045F82860204638BD002C7FF4A6AC0721C2
:1015F0006F200BF067F86E200BF038F8286020465B
:1016000038BD002C7FF499AC08216F200BF05AF8FC
:1016100021466E200BF0B5F800B22860204638BD98
:10162000002C7FF48AAC08216F200BF04BF80121CD
:101630006E200BF0A6F800B22860204638BD002CC2
:101640007FF47BAC09216F200BF03CF821466E2023
:101650000BF097F800B22860204638BD002C7FF4CC
:101660006CAC0A216F200BF02DF821466E200BF098
:1016700088F800B22860204638BD002C7FF45DACAD
:101680000A216F200BF01EF801216E200BF079F873
:1016900000B22860204638BD002C7FF44EAC0B21F0
:1016A0006F200BF00FF821466E200BF06AF800B2A5
:1016B0002860204638BD002C7FF43FAC0B216F2002
:1016C0000BF000F801216E200BF05BF800B22860EF
:1016D000204638BDDC500020002C7FF42EAC0C21BD
:1016E0006F200AF0EFFF21466E200BF04AF800B29F
:1016F0002860204638BD002C7FF41FAC0C216F20E1
:101700000AF0E0FF01216E200BF03BF800B22860E8
:10171000204638BD002C7FF410AC0D216F200AF05C
:10172000D1FF21466E200BF02CF800B22860204635
:1017300038BD002C7FF401AC0D216F200AF0C2FFF0
:1017400001216E200BF01DF800B22860204638BD44
:10175000002C7FF4F2AB0E216F200AF0B3FF21467C
:101760006E200BF00EF800B22860204638BD002C29
:101770007FF4E3AB0E216F200AF0A4FF01216E205D
:101780000AF0FFFF00B22860204638BD002C7FF42D
:10179000D4AB0F216F200AF095FF21466E200AF08E
:1017A000F0FF00B22860204638BD002C7FF4C5ABA6
:1017B0000F216F200AF086FF01216E200AF0E1FF61
:1017C00000B22860204638BD002C7FF4B6AB102153
:1017D0006F200AF077FF21466E200AF0D2FF00B298
:1017E0002860204638BD002C7FF4A7AB11216F2064
:1017F0000AF068FF21466E200AF0C3FF00B228609D
:10180000204638BD002C7FF498AB11216F200AF0E0
:1018100059FF01216E200AF0B4FF00B22860204673
:1018200038BD002C7FF489AB12216F200AF04AFFEB
:1018300021466E200AF0A5FF00B22860204638BD80
:10184000002C7FF47AAB13216F200AF03BFF214676
:101850006E200AF096FF2860204638BD002C7FF4E9
:101860006CAB13216F200AF02DFF01216E200AF0CE
:1018700088FF2860204638BD4CB9D0216F200AF07F
:1018800021FF6E200AF0F2FE2860204638BD012CB0
:1018900040F02182D0216F200AF014FF29686E20C9
:1018A0000AF010FF002038BD4CB9D1216F200AF09A
:1018B00009FF6E200AF0DAFE2860204638BD012CB0
:1018C00040F00B82D1216F200AF0FCFE29686E20C7
:1018D0000AF0F8FE002038BD5CB9D2216F200AF072
:1018E000F1FE21466E200AF04CFF00B2286020462F
:1018F00038BD012C40F0F381D2216F200AF0E2FEC6
:101900002A8800216E200AF06EFF002038BD5CB9E5
:10191000D2216F200AF0D6FE01216E200AF031FF9D
:1019200000B22860204638BD012C40F0DA81D22177
:101930006F200AF0C7FE2A8821466E200AF053FF66
:10194000002038BD5CB9D3216F200AF0BBFE2146D0
:101950006E200AF016FF00B22860204638BD012C28
:1019600040F0C181D3216F200AF0ACFE2A8800210B
:101970006E200AF038FF002038BD5CB9D3216F20FB
:101980000AF0A0FE01216E200AF0FBFE00B22860E2
:10199000204638BD012C40F0A881D3216F200AF0E9
:1019A00091FE2A8821466E200AF01DFF002038BDD6
:1019B000002C7FF4C2AA1D216F200AF083FE6E2046
:1019C0000AF054FE2860204638BD002C7FF4B5AAEA
:1019D000C0216F200AF076FE21466E200AF0D1FE6B
:1019E00000B22860204638BD002C7FF4A6AAC02192
:1019F0006F200AF067FE01216E200AF0C2FE00B2DD
:101A00002860204638BD002C7FF497AAC1216F20A2
:101A10000AF058FE21466E200AF0B3FE00B228609C
:101A2000204638BD002C7FF488AAC1216F200AF01F
:101A300049FE01216E200AF0A4FE00B22860204673
:101A400038BD002C7FF479AAC2216F200AF03AFE3B
:101A500021466E200AF095FE00B22860204638BD6F
:101A6000002C7FF46AAAC2216F200AF02BFE01210C
:101A70006E200AF086FE00B22860204638BD002C99
:101A80007FF45BAAC3216F200AF01CFE21466E2062
:101A90000AF077FE00B22860204638BD002C7FF4A3
:101AA0004CAAC3216F200AF00DFE01216E200AF01E
:101AB00068FE00B22860204638BD002C7FF43DAAA5
:101AC000C4216F200AF0FEFD21466E200AF059FE67
:101AD0002860204638BD002C7FF42FAAC4216F2037
:101AE0000AF0F0FD01216E200AF04BFE286020462E
:101AF00038BD002C7FF421AAC5216F200AF0E2FD39
:101B000021466E200AF03DFE2860204638BD002C9C
:101B10007FF413AAC5216F200AF0D4FD01216E20A5
:101B20000AF02FFE2860204638BD002C7FF405AA5D
:101B3000C6216F200AF0C6FD21466E200AF021FE64
:101B40002860204638BD002C7FF4F7A9C6216F20FD
:101B50000AF0B8FD01216E200AF013FE286020462D
:101B600038BD002C7FF4E9A9C7216F200AF0AAFD37
:101B700021466E200AF005FE2860204638BD002C64
:101B80007FF4DBA9C7216F200AF09CFD01216E20A4
:101B90000AF0F7FD2860204638BD002C7FF4CDA95F
:101BA000C8216F200AF08EFD6E200AF05FFD2860CC
:101BB000204638BD002C7FF4C0A9C9216F200AF04F
:101BC00081FD6E200AF052FD2860204638BD002CB1
:101BD0007FF4B3A9CA216F200AF074FD6E200AF0C9
:101BE00045FD2860204638BD002C7FF4A6A9CB21F6
:101BF0006F200AF067FD6E200AF038FD286020464D
:101C000038BD3CB93D490C2303FB00100389204635
:101C10002B6038BD012C6AD138490C2303FB00101E
:101C20002B680381002038BD3CB934490C2303FBE9
:101C30000010C37920462B6038BD012C59D12F49A3
:101C40000C2303FB001128788A1D07310EF0F8FEE3
:101C5000002038BD002C4ED128490C2303FB001076
:101C6000837920462B6038BD002C7FF466A9234B76
:101C70000C2101FB0030838820462B6038BD002CEE
:101C80007FF45BA91E4B20465B682B6038BD0420A7
:101C900038BD002038BD002038BD002038BD0020F0
:101CA00038BD002038BD002038BD002038BD0020E0
:101CB00038BD002038BD002038BD002038BD0020D0
:101CC00038BD002038BD002038BD002038BD0020C0
:101CD00038BD002038BD002038BD002038BD0020B0
:101CE00038BD002038BD002038BD002038BD0020A0
:101CF00038BD002038BD002038BD00BFDC500020BA
:101D00003816002010B413460446084619B9224676
:101D100010BCFEF797BF082010BC70470120704729
:101D200007B5019229B9024601AB0120FEF78AFFEF
:101D300000E0082003B05DF804FB08460AF096BCFA
:101D4000084611460AF0BEBC084611460AF019BD05
:101D5000084611461A460AF046BD38B5274B284DAD
:101D6000DC6860682368C8302860DB6898472368AF
:101D700028685B699847234B23495A6901200A6008
:101D800022491070C2F804122149C2F80812002139
:101D90005170204A18741A621F4ADA611F4A9A6108
:101DA0001F4A5A621F4ADA641F4A9A631F4A5A63DB
:101DB0001F4A9A621F4ADA621F4A9A641F4A5A648B
:101DC0001F4A5A651F4A1A651F4A1A661F4ADA6572
:101DD0001F4A9A653222DA6040F28A229A601D4BCD
:101DE0004FF47A725A8041F27072D9711A804FF4AE
:101DF00080721A81BDE83840FEF7F1BE28660208FD
:101E0000343A002018390020F05000201D1D010830
:101E1000690A0108C30B0108DD0B0108D90B010891
:101E2000D50B0108890A0108051D0108211D0108BB
:101E3000B10B01089D0B0108850A0108790A010808
:101E40009F0A0108650A0108DF0B01086D0A0108F5
:101E5000210C0108DC500020002070470120704751
:101E6000014B00225A6070471839002010B50C460B
:101E70000AF0FCFB206010BD0AF024BC38B50D460A
:101E8000044620B90EF03CFF2860204638BD0820EB
:101E900038BD30B5054689B004AC1022002120467B
:101EA00014F0F8F9374B1A68AA1A092A06D9996862
:101EB00064224A435A6000229A601D609A68013287
:101EC0009A60314B33F8060C5A780290981E0190B4
:101ED00033F8041C0020009129460FF02DF80DF076
:101EE00079F920B10022114610460DF0FFF90DF0EE
:101EF0006BF9002844D00DF0E7F9032840D8DFE85B
:101F000000F0120A022800200EF01DFF04900020AD
:101F10000EF020FF1BE000200EF0EFFE04900020EA
:101F20000EF0EEFE13E000216F200AF0CBFB6E20D6
:101F30000AF09CFB0121049069200AF022FC002198
:101F4000054669200AF01DFC2DB200B22844059018
:101F500012E076200AF08AFB6423C0F30222C0F369
:101F600002505A434343A3F52F730593074B049242
:101F70000693A3F5FA63079394E80F000DF044F974
:101F800009B030BD50160020E2500020F0D8FFFF0D
:101F900010B5044620B909680EF0C4FE204610BDF5
:101FA000082010BD10B5044618B90EF0AEFE20464C
:101FB00010BD082010BD10B5044618B90EF090FEF3
:101FC000204610BD082010BD0021F4E74942F2E789
:101FD000F1E7022804BF0C4B93F8D00020B90B4B5B
:101FE000DB681B689B690AE001280BD1064B93F85C
:101FF000D030012B06D1054BDB681B685B69044AB6
:1020000010681847704700BF18390020286602087A
:10201000343A002010B50020FFF7DBFFBDE8104088
:10202000034B044ADB6810681B689B69184700BFB4
:1020300028660208343A0020043A38B504461D46A2
:102040000846FB2A01F21D80DFE812F0FC001B08A5
:102050001B081B081B081B081B080C0113011B088D
:1020600017011B081B081B081B081B081B081B0863
:102070001B081B081B081B081B081B081B081B0848
:102080001B081B081B081B081B081B081B081B0838
:102090001B081B081B081B081B081B081B081B0828
:1020A0001B081B081B081B081B012D011B083F01F7
:1020B00052011B081B081B081B081B081B081B08D8
:1020C0001B081B081B081B081B081B081B081B08F8
:1020D0001B081B081B081B081B081B081B081B08E8
:1020E0001B081B081B081B081B081B081B081B08D8
:1020F0001B081B081B081B081B081B081B081B08C8
:102100001B081B081B081B081B081B086501760120
:1021100083011B081B081B081B081B081B081B0846
:102120001B0890019D01AA011B081B08B701C101F2
:10213000CB011B08D501DF01E9011B08F3010102F6
:102140001B080F0219021B081B081B0823022C0284
:10215000350240024B021B081B081B0854025D029B
:1021600066021B081B081B081B081B081B081B0812
:1021700071027C02870292029D02B502CD02E80242
:1021800003031E03380343034E03590364031B0870
:102190001B081B081B081B086F037A038D03A00391
:1021A000A903B203BD03CA03D503DD03EC03F9039E
:1021B0000604130420042D043A0447041B085404A5
:1021C00062047A0487049404A104AE04BB04C80426
:1021D000D504E404F3040205110520052F0540058C
:1021E0004F055E056D057C058B059A05A905B805AB
:1021F000C705D605E505F40502061B0810062806E6
:1022000040065B0676069106AC061B081B081B08F9
:10221000B906C806D706E606F5060407130722071F
:1022200031073F074D075B07690777078507930766
:10223000A107AE07BB07C8071B08D507E807FE07BD
:10224000080813082CB960200AF010FA286020460C
:1022500038BD012C40F01787296860200AF032FA57
:10226000002038BD002C40F0108700242C60204650
:1022700038BD002CF9D0002038BD002CF5D000204E
:1022800038BD34B9214608200AF07BFA2860204680
:1022900038BD012C40F0FB862A88002108200AF076
:1022A000A2FA002038BD34B9214609200AF069FAA3
:1022B0002860204638BD012C40F0EB862A8800219A
:1022C00009200AF090FA002038BD3CB9012108200D
:1022D0000AF057FA00B22860204638BD012C40F0C1
:1022E000DA862A88214608200AF07DFA002038BDC7
:1022F0003CB9012109200AF044FA00B228602046C6
:1023000038BD012C40F0C9862A88214609200AF0F0
:102310006AFA002038BD54B9012103200AF0D2F92D
:10232000214602200AF02DFA2860204638BD012CF3
:1023300014BF0020042038BD002CF8D10121032057
:102340000AF0C0F9012102200AF01BFA2860204699
:1023500038BD002CEBD1022103200AF0B3F921464D
:1023600002200AF00EFA2860204638BD002CDED18B
:10237000032108460AF0A6F9214602200AF001FAD4
:102380002860204638BD002CD1D1042103200AF05A
:1023900099F9012102200AF0F4F92860204638BD9D
:1023A000002CC4D1042103200AF08CF9214602201C
:1023B0000AF0E7F92860204638BD002CB7D1214645
:1023C00012200AF0DEF900B22860204638BD002C49
:1023D000ADD1012112200AF0D4F900B228602046C4
:1023E00038BD002CA3D1214613200AF0CAF900B24F
:1023F0002860204638BD002C99D1214615200AF0CE
:10240000C0F900B22860204638BD002C8FD10121D0
:1024100015200AF0B6F900B22860204638BD002C1D
:1024200085D1214616200AF0ACF900B2286020467A
:1024300038BD002C7FF47BAF214603200AF042F91F
:10244000214602200AF09DF92860204638BD002C64
:102450007FF46DAF214603200AF034F901210220F8
:102460000AF08FF92860204638BD002C7FF45FAF5A
:1024700021460B200AF085F92860204638BD002C43
:102480007FF455AF01210B200AF07BF9286020462C
:1024900038BD002C7FF44BAF41200AF0E7F82860EC
:1024A000204638BD002C7FF442AF42200AF0DEF80F
:1024B0002860204638BD002C7FF439AF012146202A
:1024C0000AF05FF900B22860204638BD002C7FF486
:1024D0002EAF214646200AF054F900B2286020466B
:1024E00038BD002C7FF423AF47200AF0BFF82860E6
:1024F000204638BD002C7FF41AAF21200AF0B6F830
:102500002860204638BD002C7FF411AF22200AF04D
:10251000ADF82860204638BD002C7FF408AF214676
:1025200023200AF02EF900B22860204638BD002C86
:102530007FF4FDAE27200AF099F820F07F40286054
:10254000204638BD002C7FF4F2AE28200AF08EF829
:1025500020F07F402860204638BD002C7FF4E7AE95
:1025600001212A200AF00DF900B22860204638BD6A
:10257000002C7FF4DCAE21462A200AF002F900B2DA
:102580002860204638BD4CB9D4216F200AF09AF853
:102590006E200AF06BF82860204638BD012C40F010
:1025A0007E85D4216F200AF08DF829686E200AF00C
:1025B00089F8002038BD4CB9D5216F200AF082F887
:1025C0006E200AF053F82860204638BD012C40F0F8
:1025D0006885D5216F200AF075F829686E200AF009
:1025E00071F8002038BD5CB9D6216F200AF06AF876
:1025F00021466E200AF0C5F800B22860204638BD9A
:10260000012C40F05085D6216F200AF05BF82A8813
:1026100000216E200AF0E7F8002038BD5CB9D62111
:102620006F200AF04FF801216E200AF0AAF800B2DC
:102630002860204638BD012C40F03785D6216F2018
:102640000AF040F82A8821466E200AF0CCF80020D3
:1026500038BD5CB9D7216F200AF034F821466E20CE
:102660000AF08FF800B22860204638BD012C40F0F7
:102670001E85D7216F200AF025F82A8800216E20B8
:102680000AF0B1F8002038BD54B9D7216F200AF004
:1026900019F801216E200AF074F82860204638BD30
:1026A000012C40F00685D7216F200AF00BF82A880C
:1026B00021466E200AF097F8002038BD002C7FF4E8
:1026C00036AE214639200AF05CF800B22860204678
:1026D00038BD002C7FF42BAE012139200AF051F8CF
:1026E00000B22860204638BD002C7FF420AE214681
:1026F0003D200AF046F800B22860204638BD002C84
:102700007FF415AE21463F200AF03BF800B2286066
:10271000204638BD002C7FF40AAE21463A200AF04C
:1027200030F800B22860204638BD002C7FF4FFADA1
:10273000214653200AF025F800B22860204638BD13
:102740003CB9012164200AF01CF800B22860204640
:1027500038BD012C40F0AF842A88214664200AF05D
:1027600042F8002038BD3CB9214664200AF009F83F
:1027700000B22860204638BD012C40F09E842A8893
:10278000002164200AF02FF8002038BD002C7FF4CF
:10279000CEAD662009F06AFF2860204638BD002CC7
:1027A0007FF4C5AD682009F061FF2860204638BD80
:1027B000002C7FF4BCAD0121692009F0E2FF00B2DA
:1027C0002860204638BD002C7FF4B1ADBE4A0C23F2
:1027D00003FB012319890EF032FA2860204638BD28
:1027E000002C7FF4A4AD2146692009F0CAFF00B295
:1027F0002860204638BD002C7FF499AD0EF080FA99
:102800002860204638BD24B90EF0A4FA286020467E
:1028100038BD012C40F0538429686B2009F052FF29
:10282000002038BD002C7FF482AD21466D2009F0D8
:1028300049FF6C2009F01AFF2860204638BD002CA3
:102840007FF475AD01216D2009F03CFF6C2009F08B
:102850000DFF2860204638BD002C7FF468AD0221B2
:102860006D2009F02FFF6C2009F000FF2860204642
:1028700038BD002C7FF45BAD03216D2009F022FFF1
:102880006C2009F0F3FE2860204638BD002C7FF450
:102890004EAD04216D2009F015FF6C2009F0E6FE15
:1028A0002860204638BD002C7FF441AD05216D2005
:1028B00009F008FF6C2009F0D9FE2860204638BDD9
:1028C000002C7FF434AD06216D2009F0FBFE6C2056
:1028D00009F0CCFE2860204638BD002C7FF427ADDF
:1028E00007216D2009F0EEFE6C2009F0BFFE286084
:1028F000204638BD24B90EF071F92860204638BD55
:10290000012C40F0DE8329680EF05AF9002038BD12
:102910004CB96D4A0C2303FB012319890EF085F98C
:102920002860204638BD012C40F0CD83664A0C2338
:1029300003FB01232A6819890EF065F9002038BDD0
:10294000002C7FF4F4AC01216F2009F0BBFE6E2057
:1029500009F08CFE2860204638BD002C7FF4E7ACDF
:1029600002216F2009F0AEFE6E2009F07FFE286084
:10297000204638BD002C7FF4DAAC03216F2009F02B
:10298000A1FE6E2009F072FE2860204638BD002CA2
:102990007FF4CDAC04216F2009F094FE6E2009F085
:1029A00065FE2860204638BD002C7FF4C0AC0521B0
:1029B0006F2009F087FE6E2009F058FE286020463F
:1029C00038BD002C7FF4B3AC06216F2009F07AFEED
:1029D0006E2009F04BFE2860204638BD002C7FF4A5
:1029E000A6AC07216F2009F06DFE6E2009F03EFEB7
:1029F0002860204638BD002C7FF499AC08216F2058
:102A000009F060FE21466E2009F0BBFE00B228608E
:102A1000204638BD002C7FF48AAC08216F2009F0D5
:102A200051FE01216E2009F0ACFE00B22860204664
:102A300038BD002C7FF47BAC09216F2009F042FEE9
:102A400021466E2009F09DFE00B22860204638BD68
:102A5000002C7FF46CAC0A216F2009F033FE214674
:102A60006E2009F08EFE00B22860204638BD002C92
:102A70007FF45DAC0A216F2009F024FE01216E2055
:102A800009F07FFE00B22860204638BD002C7FF49C
:102A90004EAC0B216F2009F015FE21466E2009F087
:102AA00070FE00B22860204638BD002C7FF43FAC99
:102AB0000B216F2009F006FE01216E2009F061FE56
:102AC00000B22860204638BDDC500020002C7FF486
:102AD0002EAC0C216F2009F0F5FD21466E2009F087
:102AE00050FE00B22860204638BD002C7FF41FAC99
:102AF0000C216F2009F0E6FD01216E2009F041FE56
:102B000000B22860204638BD002C7FF410AC0D21A7
:102B10006F2009F0D7FD21466E2009F032FE00B289
:102B20002860204638BD002C7FF401AC0D216F20B9
:102B300009F0C8FD01216E2009F023FE00B22860D3
:102B4000204638BD002C7FF4F2AB0E216F2009F037
:102B5000B9FD21466E2009F014FE00B2286020461F
:102B600038BD002C7FF4E3AB0E216F2009F0AAFDE5
:102B700001216E2009F005FE00B22860204638BD14
:102B8000002C7FF4D4AB0F216F2009F09BFD214670
:102B90006E2009F0F6FD00B22860204638BD002CFA
:102BA0007FF4C5AB0F216F2009F08CFD01216E2051
:102BB00009F0E7FD00B22860204638BD002C7FF404
:102BC000B6AB10216F2009F07DFD21466E2009F083
:102BD000D8FD00B22860204638BD002C7FF4A7AB9A
:102BE00011216F2009F06EFD21466E2009F0C9FD0C
:102BF00000B22860204638BD002C7FF498AB11212C
:102C00006F2009F05FFD01216E2009F0BAFD00B2CE
:102C10002860204638BD002C7FF489AB12216F203C
:102C200009F050FD21466E2009F0ABFD00B228608E
:102C3000204638BD002C7FF47AAB13216F2009F0B9
:102C400041FD21466E2009F09CFD2860204638BDDC
:102C5000002C7FF46CAB13216F2009F033FD0121B0
:102C60006E2009F08EFD2860204638BD4CB9D02179
:102C70006F2009F027FD6E2009F0F8FC286020463F
:102C800038BD012C40F02182D0216F2009F01AFDBF
:102C900029686E2009F016FD002038BD4CB9D121FD
:102CA0006F2009F00FFD6E2009F0E0FC286020463F
:102CB00038BD012C40F00B82D1216F2009F002FDBC
:102CC00029686E2009F0FEFC002038BD5CB9D221D5
:102CD0006F2009F0F7FC21466E2009F052FD00B28A
:102CE0002860204638BD012C40F0F381D2216F20AE
:102CF00009F0E8FC2A8800216E2009F074FD00200C
:102D000038BD5CB9D2216F2009F0DCFC01216E20B6
:102D100009F037FD00B22860204638BD012C40F094
:102D2000DA81D2216F2009F0CDFC2A8821466E205D
:102D300009F059FD002038BD5CB9D3216F2009F09E
:102D4000C1FC21466E2009F01CFD00B2286020461F
:102D500038BD012C40F0C181D3216F2009F0B2FCB5
:102D60002A8800216E2009F03EFD002038BD5CB9A4
:102D7000D3216F2009F0A6FC01216E2009F001FD8E
:102D800000B22860204638BD012C40F0A881D32134
:102D90006F2009F097FC2A8821466E2009F023FD58
:102DA000002038BD002C7FF4C2AA1D216F2009F03D
:102DB00089FC6E2009F05AFC2860204638BD002CA2
:102DC0007FF4B5AAC0216F2009F07CFC21466E205B
:102DD00009F0D7FC00B22860204638BD002C7FF4F3
:102DE000A6AAC0216F2009F06DFC01216E2009F018
:102DF000C8FC00B22860204638BD002C7FF497AA9A
:102E0000C1216F2009F05EFC21466E2009F0B9FC5B
:102E100000B22860204638BD002C7FF488AAC1216A
:102E20006F2009F04FFC01216E2009F0AAFC00B2CE
:102E30002860204638BD002C7FF479AAC2216F207B
:102E400009F040FC21466E2009F09BFC00B228608E
:102E5000204638BD002C7FF46AAAC2216F2009F0F9
:102E600031FC01216E2009F08CFC00B22860204664
:102E700038BD002C7FF45BAAC3216F2009F022FC2F
:102E800021466E2009F07DFC00B22860204638BD46
:102E9000002C7FF44CAAC3216F2009F013FC012100
:102EA0006E2009F06EFC00B22860204638BD002C70
:102EB0007FF43DAAC4216F2009F004FC21466E2056
:102EC00009F05FFC2860204638BD002C7FF42FAA53
:102ED000C4216F2009F0F6FB01216E2009F051FC9E
:102EE0002860204638BD002C7FF421AAC5216F2020
:102EF00009F0E8FB21466E2009F043FC28602046DB
:102F000038BD002C7FF413AAC5216F2009F0DAFB2D
:102F100001216E2009F035FC2860204638BD002CC8
:102F20007FF405AAC6216F2009F0CCFB21466E2054
:102F300009F027FC2860204638BD002C7FF4F7A953
:102F4000C6216F2009F0BEFB01216E2009F019FC9B
:102F50002860204638BD002C7FF4E9A9C7216F20E6
:102F600009F0B0FB21466E2009F00BFC28602046DA
:102F700038BD002C7FF4DBA9C7216F2009F0A2FB2C
:102F800001216E2009F0FDFB2860204638BD002C91
:102F90007FF4CDA9C8216F2009F094FB6E2009F0C1
:102FA00065FB2860204638BD002C7FF4C0A9C921EC
:102FB0006F2009F087FB6E2009F058FB286020463F
:102FC00038BD002C7FF4B3A9CA216F2009F07AFB29
:102FD0006E2009F04BFB2860204638BD002C7FF4A2
:102FE000A6A9CB216F2009F06DFB6E2009F03EFBF6
:102FF0002860204638BD3CB93D490C2303FB001036
:10300000038920462B6038BD012C6AD138490C2336
:1030100003FB00102B680381002038BD3CB9344904
:103020000C2303FB0010C37920462B6038BD012C14
:1030300059D12F490C2303FB001128788A1D073131
:103040000DF084FF002038BD002C4ED128490C2300
:1030500003FB0010837920462B6038BD002C7FF4E1
:1030600066A9234B0C2101FB0030838820462B608E
:1030700038BD002C7FF45BA91E4B20465B682B609B
:1030800038BD042038BD002038BD002038BD0020E8
:1030900038BD002038BD002038BD002038BD0020DC
:1030A00038BD002038BD002038BD002038BD0020CC
:1030B00038BD002038BD002038BD002038BD0020BC
:1030C00038BD002038BD002038BD002038BD0020AC
:1030D00038BD002038BD002038BD002038BD00209C
:1030E00038BD002038BD002038BD002038BD00BFED
:1030F000DC5000205016002010B413460446084649
:1031000019B9224610BCFEF797BF082010BC7047C3
:103110000120704707B5019229B9024601AB012091
:10312000FEF78AFF00E0082003B05DF804FB0846C4
:1031300009F09CBA0846114609F0C4BA084611467F
:1031400009F01FBB084611461A4609F04CBB38B5BA
:10315000274B284DDC6860682368C8302860DB682E
:103160009847236828685B699847234B23495A6925
:1031700001200A6022491070C2F804122149C2F8E5
:10318000081200215170204A18741A621F4ADA612D
:103190001F4A9A611F4A5A621F4ADA641F4A9A6399
:1031A0001F4A5A631F4A9A621F4ADA621F4A9A6488
:1031B0001F4A5A641F4A5A651F4A1A651F4A1A66EF
:1031C0001F4ADA651F4A9A653222DA6040F28A2283
:1031D0009A601D4B4FF47A725A8041F27072D97125
:1031E0001A804FF480721A81BDE83840FEF7F1BEB4
:1031F00028660208343A002018390020F4500020D4
:10320000113101085D1E0108B71F0108D11F010817
:10321000CD1F0108C91F01087D1E0108F9300108F2
:1032200015310108A51F0108911F0108791E010829
:103230006D1E0108931E0108591E0108D31F0108C5
:10324000611E010815200108DC500020014B0022FE
:103250005A6070471839002070B50446074E084D73
:1032600033682A46014600200DF0DBFF33682A460A
:103270002146BDE8704001200DF0D3BF94530020DB
:10328000F8500020014B18680EF02BB89453002022
:1032900001280CD8074B1A68202303FA00F040F0ED
:1032A000020002EB8000436800200B60704708209A
:1032B000704700BF94530020012810B5144616D063
:1032C00008D302281FD1114B114ADB6890681B6894
:1032D0001B6A12E014680D4A0D4BD268126824B1C3
:1032E0005269D8689047002010BD9269F9E7074BF2
:1032F000074ADB6850681B681B6A9847003018BF94
:1033000001202060EFE7042010BD00BF28660208FE
:1033100068160020022804BF0B4B93F8D00020B998
:103320000A4BDB681B685B690AE001280BD1064B7E
:1033300093F8D030012B06D1044BDB681B689B69E6
:10334000034A106818477047183900202866020899
:103350006816002070B50020FFF7DCFF104B114C01
:10336000DD6820682B689B6898472B6860689B68BD
:1033700098472B68A0689B6898472B68A0699B6852
:1033800098472B6820699B6898472B6860699B6801
:1033900098472B68E0689B68BDE87040184700BFFD
:1033A00028660208681600202DE9F8430F4691466A
:1033B0009846174C0021236847F080009B689DF8D1
:1033C00020609DF824509847236800219B68484658
:1033D0009847236800219B6840469847236800214E
:1033E0009B6830469847236828469B680121984788
:1033F000084B48EA09281B6846EA082607F07F07B9
:1034000003EB870745EA06257D60BDE8F88300BF2A
:10341000905300209453002007B5D3B20193C2F318
:1034200007230093C2F30743120EFFF7BDFF03B05B
:103430005DF804FB0A4601460020FFF7EDBF0128B6
:1034400073B505460C4623D8134E335C63B1134B5A
:103450002021814003EB800341F00701DA69C9B202
:10346000FFF7DAFF002373552026AE4046F00D012A
:103470002246C9B200242846FFF7CEFF2846019411
:10348000009423462246F1B2FFF78EFF204600E06B
:10349000082002B070BD00BFA00000206816002008
:1034A000012873B505460E461BD82024844044F0FD
:1034B000070186EAE672A2EBE672C9B2FFF7ACFF3B
:1034C000094A0123002E5355E1B2B8BF022300245C
:1034D00001932846009423462246FFF765FF2046C5
:1034E00000E0082002B070BDA00000200021D7E756
:1034F0004942D5E7D4E738B5234B01F07F04234494
:1035000093F81432DB0705D4204B1B6803EB8404CB
:10351000606838BD1E4D00212B6820469B68984787
:103520002B6800219B68084698472B6800219B6800
:10353000084698472B6800219B68084698472B68E7
:1035400001219B68002098472B6800219B6820463A
:1035500098472B6800219B68084698472B680021F4
:1035600004029B68084698472B6800212043040208
:103570009B68084698472B68204304029B680121FA
:1035800000209847204338BDF85000209453002075
:103590009053002010B50C4601460020FFF7ABFF0A
:1035A000206010BD38B50D462021814041F0010159
:1035B000C9B20446FFF79FFF2968014429602046ED
:1035C000BDE838403BE71C2A2DE9F84304460E4687
:1035D0001F4600F088835DD80C2A00F0F8812BD8B4
:1035E000052A00F0508113D8022A00F0EA8007D89B
:1035F000002A00F0AD80012A00F0C88000F0C3BFAF
:10360000032A00F0FE80042A00F0138100F0BBBF03
:10361000082A00F0A58107D8062A00F05081072A61
:1036200000F0768100F0AFBF0A2A00F0AA810B2AD1
:1036300000F0BA8100F0A7BF122A00F0908213D8E0
:103640000F2A00F0348207D80D2A00F0EA810E2AF2
:1036500000F0118200F097BF102A00F04482112A76
:1036600000F0618200F08FBF152A00F0CC8207D8ED
:10367000132A00F09082142A00F0A98200F083BF80
:10368000172A00F0F882C0F0DA82182A00F00F83BF
:1036900000F079BFAC2A00F09E852AD8A52A00F058
:1036A0003D8413D8A22A00F0C18307D81D2A00F058
:1036B00042838C2A00F04F8300F065BFA32A00F0FC
:1036C000DD83A42A00F0028400F05DBFA82A00F088
:1036D000E38407D8A62A00F07084A72A00F0B384F8
:1036E00000F051BFAA2A00F0268540F2FC8400F0C9
:1036F0004ABDB62A00F0A38213D8B32A00F0EA85A7
:1037000007D8AD2A00F08E85AE2A00F0B38500F010
:103710003ABFB42A00F00686B52A00F0138600F0FE
:1037200032BFCE2A00F0968607D8B82A00F042862B
:10373000B92A00F0678600F026BFD22A00F0B686CC
:10374000D32A00F0CF86D12A40F01D8700F092BE28
:1037500058B92021B14041F00D01C9B23046FFF700
:10376000CAFE38600020BDE8F883012802D000209E
:10377000BDE8F8832021B14041F00D0130461A68C0
:10378000C9B2FFF749FE0020BDE8F88358B92021EF
:10379000B14041F00101C9B23046FFF7ACFE3860DC
:1037A0002046BDE8F8830128E1D12021B14041F055
:1037B000010130461A68C9B2FFF72EFE0020BDE8AD
:1037C000F88358B92021B14041F00701C9B2304611
:1037D000FFF791FE38602046BDE8F8830128C6D186
:1037E0003A682021C64BB140002A41F007019855A4
:1037F000B8BF52423046C9B2FFF70EFE0020BDE806
:10380000F88388B92021B14041F00201C9B23046A5
:10381000FFF771FE10F4000318BF4FF07F4303431E
:103820003B600020BDE8F883012CA0D10420BDE856
:10383000F88338B9B34800EB8100C36920463B6088
:10384000BDE8F883012892D13A68AE4B2024002AC3
:1038500004FA01F403EB8103B8BF5242E1B23046EF
:10386000DA61FFF748FE0546002880D13A6844F047
:103870000701002A3046B8BF5242C9B2FFF7CCFD5B
:103880002846BDE8F88358B92021B14041F006012F
:10389000C9B23046FFF72FFE38602046BDE8F883F6
:1038A00001287FF464AF2021B14041F00601304689
:1038B0001A68C9B2FFF7B0FD0020BDE8F88368B907
:1038C0002021B14041F01001C9B23046FFF713FE8C
:1038D000C0F3042038600020BDE8F88301287FF49D
:1038E00046AF20248C4044F01004E4B22146304618
:1038F000FFF701FE3B6820F4F8521B0203F4F85373
:1039000030461A432146FFF787FD0020BDE8F883C3
:1039100068B92021B14041F01001C9B23046FFF72B
:10392000EAFD00F01F0038602046BDE8F88301285A
:103930007FF41DAF20248C4044F01004E4B22146F3
:103940003046FFF7D8FD3B6820F01F0203F01F034D
:1039500030461A432146FFF75FFD0020BDE8F8839B
:1039600000287FF461AF2021B14041F01501C9B2B8
:103970003046FFF7C0FDC0F3402038602046BDE868
:10398000F88300287FF450AF2021B14041F01501A9
:10399000C9B23046FFF7AFFDC0F3400080F0010030
:1039A00038600020BDE8F88300287FF43DAF202177
:1039B000B14041F01501C9B23046FFF79CFD00F05F
:1039C000010080F0010038602046BDE8F88368B946
:1039D0002021B14041F01401C9B23046FFF78BFD00
:1039E000C0F3400038602046BDE8F88301287FF42A
:1039F000BEAE20248C4044F01404E4B2214630468C
:103A0000FFF779FD3B6820F00202002B0CBF022378
:103A1000002330461A432146FFF7FEFC0020BDE894
:103A2000F88368B92021B14041F01401C9B2304691
:103A3000FFF761FD00F0010038600020BDE8F88369
:103A400001287FF494AE20248C4044F01404E4B2A6
:103A500021463046FFF74FFD3A6820F00100002A6A
:103A600014BF024640F0010221463046FFF7D4FC65
:103A70000020BDE8F88358B92021B14041F014017D
:103A8000C9B23046FFF737FD38602046BDE8F883FD
:103A900001287FF46CAE2021B14041F01401304682
:103AA0001A68C9B2FFF7B8FC0020BDE8F88358B91E
:103AB0002021B14041F00401C9B23046FFF71BFD9F
:103AC00038602046BDE8F88301287FF450AE2021FD
:103AD000B14041F0040130461A68C9B2FFF79CFCBE
:103AE0000020BDE8F88378B92021B14041F00501FC
:103AF000C9B23046FFF7FFFC38600020BDE8F8830C
:103B0000A00000206816002001287FF430AE20219C
:103B1000B14041F0050130461A68C9B2FFF77CFC9C
:103B20000020BDE8F88358B92021B14041F00801D8
:103B3000C9B23046FFF7DFFC38602046BDE8F883A5
:103B400001287FF414AE2021B14041F00801304635
:103B50001A68C9B2FFF760FC0020BDE8F88358B9C5
:103B60002021B14041F00A01C9B23046FFF7C3FC41
:103B700038602046BDE8F88301287FF4F8AD2021A5
:103B8000B14041F00A0130461A68C9B2FFF744FC5F
:103B90000020BDE8F88358B92021B14041F003016D
:103BA000C9B23046FFF7A7FC38600020BDE8F883B3
:103BB00001287FF4DCAD2021B14041F00301304603
:103BC0001A68C9B2FFF728FC0020BDE8F88358B98D
:103BD0002021B14041F00B01C9B23046FFF78BFC08
:103BE00038602046BDE8F88301287FF4C0AD20216D
:103BF000B14041F00B0130461A68C9B2FFF70CFC26
:103C00000020BDE8F88358B92021B14041F00C01F3
:103C1000C9B23046FFF76FFC38602046BDE8F88334
:103C200001287FF4A4AD2021B14041F00C013046C1
:103C30001A68C9B2FFF7F0FB0020BDE8F8835CB951
:103C40002021B14041F01101C9B23046FFF753FCC9
:103C500038600020BDE8F883012C7FF488AD202176
:103C6000B14041F0110130463A68C9B2FFF7D4FBC8
:103C70000020BDE8F88358B92021B14041F012017D
:103C8000C9B23046FFF737FC38600020BDE8F88342
:103C900001287FF46CAD2021B14041F01201304683
:103CA0001A68C9B2FFF7B8FB0020BDE8F88358B91D
:103CB0002021B14041F01301C9B23046FFF71BFC8F
:103CC00038602046BDE8F88301287FF450AD2021FC
:103CD000B14041F0130130461A68C9B2FFF79CFBAE
:103CE0000020BDE8F88368B9090141F06C0101F0DA
:103CF000FC013046FFF7FFFBC0F3804038602046F0
:103D0000BDE8F88301287FF432AD0C0144F06C0467
:103D1000E4B221463046FFF7EEFB3B6820F48022F8
:103D20009B0403F4802330461A432146FFF774FBBB
:103D30000020BDE8F88300287FF476ADC94B202031
:103D40001B68884040F0020003EB800043680020BD
:103D50003B60BDE8F88388B9090141F06C0101F0CE
:103D6000FC013046FFF7C7FB4FF48073C0F30360DC
:103D700043FA00F038602046BDE8F88301287FF45C
:103D8000F6AC1B68102B1FD00CDC022B18D003DC08
:103D9000012B1FD108231FE0042B13D0082B19D1AE
:103DA000052319E0402B11D003DC202B12D1032373
:103DB00012E0802B0CD0B3F5807F0BD100230BE0F9
:103DC000072309E0062307E0042305E0022303E0BC
:103DD000386002E04FF0FF333B603B6801333FF453
:103DE000C6AC340144F06C04E4B221463046FFF71F
:103DF00082FB3B6820F070621B0603F070631A437D
:103E000021463046FFF708FB21463046FFF773FB9B
:103E10003B6820F070621B0603F0706330461A4363
:103E20002146FFF7F9FA0020BDE8F88368B90901D7
:103E300041F06C0101F0FC013046FFF75CFBC0F380
:103E4000C13038602046BDE8F88301287FF48FAC8C
:103E50000C0144F06C04E4B221463046FFF74BFB02
:103E60003B6820F4C032DB0303F4C03330461A430E
:103E70002146FFF7D1FA0020BDE8F88368B90901AF
:103E800041F06C0101F0FC013046FFF734FBC0F358
:103E9000803038600020BDE8F88301287FF467ACEB
:103EA0000C0144F06C04E4B221463046FFF723FBDA
:103EB0003B6820F480429B0303F4804330461A435E
:103EC0002146FFF7A9FA0020BDE8F88368B9090187
:103ED00041F06C0101F0FC013046FFF70CFBC0F330
:103EE000003038602046BDE8F88301287FF43FACFD
:103EF0000C0144F06C04E4B221463046FFF7FBFAB3
:103F00003B6820F480521B0303F4805330461A436D
:103F10002146FFF781FA0020BDE8F8834FEA011837
:103F200048F06C085FFA88F841463046FFF7E3FA3C
:103F30000546D4B915F480494146304607D0FFF70D
:103F4000DAFAC0F3C31038602046BDE8F883FFF703
:103F5000D2FA2C05C0F3021001D4386007E440F017
:103F6000080038604846BDE8F883012C7FF4FFABB9
:103F700015F48045414630460FD0FFF7BCFA3B6848
:103F800020F4F062DB0103F4F06330461A4341464B
:103F9000FFF742FA0020BDE8F883FFF7ACFA3B6870
:103FA00020F070021B0103F0700330461A434146B3
:103FB000FFF732FA2846BDE8F8830D0145F06C059D
:103FC000EDB229463046FFF796FAA4B910F48044C2
:103FD0002946304607D0FFF78EFAC0F3021038604A
:103FE0000020BDE8F883FFF786FAC0F3C3103860FD
:103FF0002046BDE8F883012C7FF4B9AB10F480446F
:10400000294630460FD0FFF776FA3B6820F0700261
:104010001B0103F0700330461A432946FFF7FCF9F1
:104020000020BDE8F883FFF766FA3B6820F4F062F1
:10403000DB0103F4F06330461A432946FFF7ECF93D
:104040002046BDE8F88378B9090141F06C0101F020
:10405000FC013046FFF74FFA00F00F0038602046B1
:10406000BDE8F8839453002001287FF480AB0C0155
:1040700044F06C04E4B221463046FFF73CFA3B685A
:1040800020F00F0203F00F0330461A432146FFF7DA
:10409000C3F90020BDE8F88368B9090141F06D015A
:1040A00001F0FD013046FFF726FAC0F3C03038605A
:1040B0002046BDE8F88301287FF459AB0C0144F099
:1040C0006D04E4B221463046FFF715FA3B6820F450
:1040D0000042DB039BB230461A432146FFF79CF9AE
:1040E0000020BDE8F88368B9090141F06D0101F0D5
:1040F000FD013046FFF7FFF9C0F34130386020463C
:10410000BDE8F88301287FF432AB0C0144F06D0464
:10411000E4B221463046FFF7EEF93B6820F4C04296
:104120005B0303F4C04330461A432146FFF774F99A
:104130000020BDE8F88368B9090141F06D0101F084
:10414000FD013046FFF7D7F9C0F3032038600020A7
:10415000BDE8F88301287FF40AAB0C0144F06D043C
:10416000E4B221463046FFF7C6F93B6820F470629E
:104170001B0203F4706330461A432146FFF74CF9E3
:104180000020BDE8F88368B9090141F06D0101F034
:10419000FD013046FFF7AFF9C0F34110386020460B
:1041A000BDE8F88301287FF4E2AA0C0144F06D0415
:1041B000E4B221463046FFF79EF93B6820F06002EA
:1041C0005B0103F0600330461A432146FFF724F9F0
:1041D0000020BDE8F88368B9090141F06D0101F0E4
:1041E000FD013046FFF787F900F00F0038602046E8
:1041F000BDE8F88301287FF4BAAA0C0144F06D04ED
:10420000E4B221463046FFF776F93B6820F00F0212
:1042100003F00F0330461A432146FFF7FDF8002054
:10422000BDE8F88368B9090141F06D0101F0FD01B5
:104230003046FFF760F9C0F3006038600020BDE849
:10424000F88301287FF493AA0C0144F06D04E4B2D2
:1042500021463046FFF74FF93B6820F080721B067D
:1042600003F0807330461A432146FFF7D5F800204B
:10427000BDE8F883A8B9090141F06D0101F0FD0125
:104280003046FFF738F9001410F0400F00F07F02BD
:1042900014BF6FF07F03002313433B602046BDE84B
:1042A000F88301287FF463AA0C0144F06D04E4B2A2
:1042B00021463046FFF71FF93B6820F4FE021B043D
:1042C00003F4FE0330461A432146FFF7A5F8002009
:1042D000BDE8F88368B9090141F06C0101F0FC0107
:1042E0003046FFF708F9C0F3404038602046BDE88B
:1042F000F88301287FF43BAA0C0144F06C04E4B27B
:1043000021463046FFF7F7F83B6820F400325B04A3
:1043100003F4003330461A432146FFF77DF80020AE
:10432000BDE8F88300287FF47FAA090141F06F01FE
:10433000C9B23046FFF7DFF8C0F304403860002010
:10434000BDE8F88320258D406DB245F014085FFA72
:1043500088F841463046FFF7CEF87CB9410509D5CB
:1043600045F01101C9B23046FFF7C5F83860204664
:10437000BDE8F8833C602046BDE8F883012C7FF45B
:10438000F6A945F011013A683046C9B2FFF744F882
:1043900041463046FFF7AFF83B6820F480629B024D
:1043A00003F4806330461A434146FFF735F8002096
:1043B000BDE8F88368B9090141F06C0101F0FC0126
:1043C0003046FFF798F8C0F3403038600020BDE871
:1043D000F88301287FF4CBA90C0144F06C04E4B20B
:1043E00021463046FFF787F83B6820F400525B0314
:1043F00003F4005330461A432146FFF70DF800201E
:10440000BDE8F88368B9090141F06C0101F0FC01D5
:104410003046FFF770F8C0F3035038602046BDE81F
:10442000F88301287FF4A3A90C0144F06C04E4B2E2
:1044300021463046FFF75FF83B6820F470021B0509
:1044400003F4700330461A432146FEF7E5FF0020CF
:10445000BDE8F88300287FF4E7A9090141F06F0166
:10446000C9B23046FFF747F8C0F30900386020466C
:10447000BDE8F88358B92021B14041F01901C9B213
:104480003046FFF738F838602046BDE8F883012849
:104490007FF46DA92021B14041F0190130461A681E
:1044A000C9B2FEF7B9FF0020BDE8F88358B9202152
:1044B000B14041F01A01C9B23046FFF71CF838602C
:1044C0000020BDE8F88301287FF451A92021B140E4
:1044D00041F01A0130461A68C9B2FEF79DFF00206C
:1044E000BDE8F883E8B979B101294FD101463046DA
:1044F000FFF701F800F06000A0F120035842584196
:1045000038602046BDE8F8830846FEF7F4FF00F067
:104510001800A0F110025042504138603046BDE80A
:10452000F88301287FF423A911B1012915D02FE0C8
:104530000846FEF7E0FF3B6823B120F0080242F096
:10454000100203E020F0100242F0080200210846A9
:10455000FEF762FF0020BDE8F88300213046FEF739
:10456000CAFF3B6823B120F0400242F0200203E082
:1045700020F0200242F0400200210120FEF74CFF13
:104580000020BDE8F8830420BDE8F883BDE8F88387
:104590000020BDE8F88307B50129019205D802463D
:1045A00001AB0120FFF70FF800E0082003B05DF831
:1045B00004FB0129134603D802460020FFF703B885
:1045C0000820704708B522210020FEF794FF50B95B
:1045D00042210120FEF78FFF28B9044B1868BDE87F
:1045E00008400CF077BE002008BD00BF94530020A7
:1045F00070B53D4E3D480CF0D5FDF5683C4C6B6800
:1046000003F5AA72626003F5B872A26003F56F72D7
:10461000E26003F5767203F1C800226103F57D7252
:1046200003F58263A3612B686261DB6820609847B1
:104630002B68E068DB6898472B68E0689B699847BF
:104640002B6860681B6998472B68A0681B699847AE
:104650002B68A0691B6998472B6820691B699847DC
:104660002B6860691B6998473269224B22491A609E
:104670006B68012003F537735360204B5A690A6059
:104680001F491070C2F804121E49C2F80812002116
:1046900051701D4A1A621D4ADA611D4A9A611D4A0B
:1046A0005A621D4A9A631D4A5A631D4A9A621D4AFC
:1046B000DA621D4A9A641D4A5A641D4A5A651D4AA7
:1046C0001A651D4ADA641D4A1A661D4ADA65022215
:1046D0001A743222DA60B6229A601A4A9A65BDE8E4
:1046E0007040FEF717BE00BF28660208F850002091
:1046F00068160020905300209453002018390020A1
:10470000C545010885320108A1340108F5340108C6
:10471000F1340108ED340108B3450108974501085B
:104720003F340108A53501083534010895350108E5
:1047300059320108B93201089132010815330108D4
:104740004D3201085533010801289FBF034B53F830
:10475000203000200B6088BF08207047A053002045
:10476000014B00225A6070471839002070B504468A
:10477000074E084D33682A46014600200CF0F9FD2B
:1047800033682A462146BDE8704001200CF0F1BD97
:1047900098530020A0530020014B18680CF033BE42
:1047A00098530020012810B5144608D0022813D1D0
:1047B0000A4B0B4ADB6890681B681B6A05E0074BD5
:1047C000074ADB6850681B681B6A9847003018BFAF
:1047D00001202060002010BD042010BD28660208C2
:1047E00098160020022804BF0B4B93F8D00020B984
:1047F0000A4BDB681B685B690AE001280BD1064B9A
:1048000093F8D030012B06D1044BDB681B689B6901
:10481000034A1068184770471839002028660208B4
:104820009816002070B50020FFF7DCFF084B094CFC
:10483000DD6820682B689B6898472B6860689B68D8
:1048400098472B68A0689B68BDE87040184700BF78
:1048500028660208981600202DE9F8430F46914675
:104860009846174C0021236847F080009B689DF80C
:1048700020609DF824509847236800219B68484693
:104880009847236800219B68404698472368002189
:104890009B6830469847236828469B6801219847C3
:1048A000084B48EA09281B6846EA082607F07F07F4
:1048B00003EB870745EA06257D60BDE8F88300BF66
:1048C0009C5300209853002007B5D3B20193C2F344
:1048D00007230093C2F30743120EFFF7BDFF03B097
:1048E0005DF804FB0A4601460020FFF7EDBF0128F2
:1048F000F7B505460F4627D8154C044494F8943272
:1049000073B1144B202181401B6841F0070103EB78
:1049100081035A68C9B2FFF7D7FF002384F89432A5
:104920002026AE4046F00D0100243A46C9B2284682
:10493000FFF7CAFF28460194009423462246F1B2AD
:10494000FFF78AFF204600E0082003B0F0BD00BF5B
:10495000A053002098530020012873B505460C464B
:1049600021D82026864084EAE47246F00701A2EBB3
:10497000E472C9B2FFF7A8FF0C4B002C2B444FF098
:10498000010283F89422A8BF13464FF00004B8BF79
:10499000022301932846009423462246F1B2FFF7F2
:1049A0005BFF204600E0082002B070BDA05300204D
:1049B0000021D1E74942CFE7CEE738B5234B01F0DC
:1049C0007F04234493F81432DB0705D4204B1B6883
:1049D00003EB8404606838BD1E4D00212B6820461F
:1049E0009B6898472B6800219B68084698472B686E
:1049F00000219B68084698472B6800219B68084661
:104A000098472B6801219B68002098472B6800215C
:104A10009B68204698472B6800219B68084698476A
:104A20002B68002104029B68084698472B680021E8
:104A3000204304029B68084698472B6820430402E1
:104A40009B68012100209847204338BDA0530020D7
:104A5000985300209C53002010B50C4601460020BE
:104A6000FFF7ABFF206010BD38B50D462021814017
:104A700041F00101C9B20446FFF79FFF29680144D4
:104A800029602046BDE8384031E71C2A2DE9F8436B
:104A900004460E461F4600F039835DD80C2A00F00C
:104AA000D8812BD8052A00F0458113D8022A00F0BE
:104AB000E08007D8002A00F0AE80012A00F0C5800F
:104AC00000F09BBE032A00F0F480042A00F0088165
:104AD00000F093BE082A00F08C8107D8062A00F067
:104AE0003D81072A00F0618100F087BE0A2A00F0AC
:104AF0008E810B2A00F09D8100F07FBE122A00F00B
:104B0000718213D80F2A00F0268207D80D2A00F0F0
:104B1000D6810E2A00F00B8200F06FBE102A00F042
:104B20002E82112A00F04A8200F067BE152A00F09A
:104B3000978207D8132A00F06882142A00F07D8239
:104B400000F05BBE172A00F0B682C0F09C82182AE3
:104B500000F0C98200F051BEAB2A00F0EF842BD8E0
:104B6000A52A00F0BF8313D8A22A00F0518307D8EA
:104B70001D2A00F0EE828C2A00F0F38200F03DBE88
:104B8000A32A00F06883A42A00F0898300F035BED0
:104B9000A82A00F0678407D8A62A00F0F883A72A7D
:104BA00000F0438400F029BEA92A00F07F84AA2ADD
:104BB00000F0A08400F021BEB52A00F0858513D84E
:104BC000AE2A00F0248507D8AC2A00F0DA84AD2A9A
:104BD00000F0FA8400F011BEB32A00F04485B42A34
:104BE00000F0658500F009BECE2A00F0B48507D834
:104BF000B62A00F04882B82A00F08B8500F0FDBD8F
:104C0000D12AC0F0FA85D22A40F2FD85D32A00F0DD
:104C1000AF8500F0F2BD50B92021B14041F00D0147
:104C2000C9B23046FFF7C9FE386000F0ECBD01287C
:104C300040F0E9852021B14041F00D011A68C9B268
:104C40003046FFF741FE00F0DEBD20B92021B14023
:104C500041F0010112E0012840F0D5852021B1404A
:104C600041F001011A68C9B23046FFF72DFE00F08D
:104C7000CABD48B92021B14041F00701C9B2304650
:104C8000FFF79BFE00F041BC012840F0BC85C94BFA
:104C90000B4483F894023A682021B140002A41F085
:104CA0000701B8BF5242C9B23046FFF70DFE00F00F
:104CB000AABD80B92021B14041F00201C9B23046FD
:104CC000FFF77BFE10F4000318BF4FF07F43034350
:104CD0003B6000F098BD012C00F08F8500F093BD83
:104CE00050B9B54B20201B68884040F0070003EB0B
:104CF0008000436800F09EBC012840F08485AE4BE4
:104D00003A682021B1401B6841F00704002A03EBF8
:104D10008403B8BF52425A60C9B23046FFF74DFE15
:104D20000546002840F06F853A68E1B2002AB8BF16
:104D3000524274E320B92021B14041F006019DE7C1
:104D4000012840F060852021B14041F006011A6839
:104D5000C9B23046FFF7B8FD00F055BD60B920215B
:104D6000B14041F01001C9B23046FFF726FEC0F352
:104D70000420386000F047BD012840F0448520241D
:104D80008C4044F01004E4B221463046FFF715FE93
:104D90003B6820F4F8521B0203F4F8531A432146EF
:104DA0003046FFF791FD00F02EBD50B92021B140F3
:104DB00041F01001C9B23046FFF7FFFD00F01F00BF
:104DC000A3E3012840F01F8520248C4044F0100408
:104DD000E4B221463046FFF7F0FD3B6820F01F02A9
:104DE00003F01F031A4321463046FFF76DFD00F024
:104DF0000ABD00287FF46FAF2021B14041F01501BA
:104E0000C9B23046FFF7D9FDC0F340207DE300284A
:104E10007FF461AF2021B14041F01501C9B23046A5
:104E2000FFF7CBFDC0F3400080F00100386000F0D8
:104E3000EABC00287FF44FAF2021B14041F01501BA
:104E4000C9B23046FFF7B9FD00F0010080F0010063
:104E50005BE350B92021B14041F01401C9B23046A2
:104E6000FFF7ABFDC0F340004FE3012840F0CB84D7
:104E700020248C4044F01404E4B221463046FFF76D
:104E80009CFD3B6820F00202002B14BF022300238C
:104E90001A4321463046FFF717FD21463046FFF7FB
:104EA0008CFD3B6820F00802022B0CBF0823002376
:104EB0001A4321463046FFF707FD00F0A4BC60B955
:104EC0002021B14041F01401C9B23046FFF775FD11
:104ED00000F00100386000F096BC012840F0938497
:104EE00020248C4044F01404E4B221463046FFF7FD
:104EF00064FD3A6820F00100002A0CBF024640F031
:104F0000010221463046FFF7DFFC21463046FFF71D
:104F100054FD3B6820F00402022B0CBF0423002345
:104F20001A4321463046FFF7CFFC00F06CBC20B995
:104F30002021B14041F01401A0E6012840F0638433
:104F40002021B14041F014011A68C9B23046FFF780
:104F5000BBFC00F058BC20B92021B14041F0040155
:104F60008CE6012840F04F842021B14041F004013B
:104F70001A68C9B23046FFF7A7FC00F044BC50B92C
:104F80002021B14041F00501C9B23046FFF715FDBF
:104F9000386000F038BC012840F035842021B14051
:104FA00041F005011A68C9B23046FFF78DFC00F0E8
:104FB0002ABC00BFA05300209853002020B9202114
:104FC000B14041F0080159E6012840F01C8420213D
:104FD000B14041F008011A68C9B23046FFF774FCCD
:104FE00000F011BC20B92021B14041F00A0145E692
:104FF000012840F008842021B14041F00A011A68DC
:10500000C9B23046FFF760FCFDE348B92021B1404A
:1050100041F00301C9B23046FFF7CFFC3860F2E33C
:10502000012840F0F0832021B14041F003011A68CB
:10503000C9B23046FFF748FCE5E320B92021B14072
:1050400041F00B011AE6012840F0DD832021B14038
:1050500041F00B011A68C9B23046FFF735FCD2E3C4
:1050600020B92021B14041F00C0107E6012840F0B1
:10507000CA832021B14041F00C011A68C9B2304600
:10508000FFF722FCBFE34CB92021B14041F01101F0
:10509000C9B23046FFF791FC3860B4E3012C40F010
:1050A000B2832021B14041F011013A68C9B23046C3
:1050B000FFF70AFCA7E348B92021B14041F01201F3
:1050C000C9B23046FFF779FC38609CE3012840F014
:1050D0009A832021B14041F012011A68C9B23046CA
:1050E000FFF7F2FB8FE320B92021B14041F013011B
:1050F000C4E5012840F087832021B14041F013012D
:105100001A68C9B23046FFF7DFFB7CE350B90901EA
:1051100041F06C0101F0FC013046FFF74EFCC0F39A
:105120008040F2E1012840F06E830C0144F06C04F1
:10513000E4B221463046FFF740FC3B6820F4802271
:105140009B0403F480231A4321463046FFF7BCFB3F
:1051500059E300287FF4BFADC84B53F821303B60C2
:1051600051E370B9090141F06C0101F0FC013046D6
:10517000FFF723FC4FF48073C0F3036043FA00F0A1
:10518000C3E1012840F03F831B68102B1FD00CDCCB
:10519000022B18D003DC012B1FD108231FE0042BA6
:1051A00013D0082B19D1052319E0402B11D003DCB3
:1051B000202B12D1032312E0802B0CD0B3F5807F7B
:1051C0000BD100230BE0072309E0062307E00423AB
:1051D00005E0022303E0386002E04FF0FF333B605C
:1051E0003B68013300F00F83340144F06C04E4B2F7
:1051F00021463046FFF7E1FB3B6820F070621B065A
:1052000003F070631A4321463046FFF75DFBFAE274
:1052100050B9090141F06C0101F0FC013046FFF783
:10522000CCFBC0F3C13070E1012840F0EC820C01EE
:1052300044F06C04E4B221463046FFF7BEFB3B6805
:1052400020F4C032DB0303F4C0331A432146304656
:10525000FFF73AFBD7E258B9090141F06C0101F0C0
:10526000FC013046FFF7A9FBC0F380303860CAE28A
:10527000012840F0C8820C0144F06C04E4B22146DD
:105280003046FFF79AFB3B6820F480429B0303F40F
:1052900080431A4321463046FFF716FBB3E250B96C
:1052A000090141F06C0101F0FC013046FFF785FB7C
:1052B000C0F3003029E1012840F0A5820C0144F040
:1052C0006C04E4B221463046FFF777FB3B6820F4DC
:1052D00080521B0303F480531A4321463046FFF7E4
:1052E000F3FA90E20D0145F06C05EDB22946304627
:1052F000FFF763FBB4B910F4804206D0294630466C
:10530000FFF75BFBC0F3C310FFE00311010503F0DF
:10531000700301D43B6076E243F008033B60104623
:10532000BDE8F883012C40F06E8210F480442946D9
:1053300030460DD0FFF741FB3B6820F4F062DB0103
:1053400003F4F0631A4329463046FFF7BDFA5AE2E8
:10535000FFF733FB3B6820F4006213F0080F18BF1F
:105360004FF40064224329463046FFF7ADFA294640
:105370003046FFF722FB3B6820F070021B0103F070
:1053800070031A4329463046FFF79EFA3BE24FEA84
:10539000011848F06C085FFA88F841463046FFF77C
:1053A0000CFB8146BCB919F480454146304605D016
:1053B000FFF703FBC0F30210386024E2FFF7FDFAA9
:1053C00019F4006FC0F3C31001D138601BE240F044
:1053D0000800386026E0012C40F015824146304636
:1053E000FFF7EBFA10F48045414630460DD0FFF749
:1053F000E4FA3B6820F070021B0103F070031A43CB
:1054000041463046FFF760FAFDE1FFF7D6FA414624
:105410003B6820F4F062DB0103F4F0631A4330468A
:10542000FFF752FA2846BDE8F88348B9090141F070
:105430006C0101F0FC013046FFF7BFFA3C60DFE190
:10544000012840F0E0810C0144F06C04E4B22146F4
:105450003046FFF7B2FA214620F00F023046FFF740
:1054600033FAD0E160B9090141F06D0101F0FD01AD
:105470003046FFF7A2FAC0F3C03046E0A053002048
:10548000012840F0C0810C0144F06D04E4B22146D3
:105490003046FFF792FA3B6820F40042DB039BB2F0
:1054A0001A4321463046FFF70FFAACE158B909011B
:1054B00041F06D0101F0FD013046FFF77EFAC0F3C7
:1054C000413038609FE1012840F09D810C0144F09B
:1054D0006D04E4B221463046FFF76FFA3B6820F4D2
:1054E000C0425B0303F4C0431A4321463046FFF732
:1054F000EBF988E158B9090141F06D0101F0FD01B6
:105500003046FFF75AFAC0F30320386078E10128EB
:1055100040F079810C0144F06D04E4B2214630463C
:10552000FFF74BFA3B6820F470621B0203F47063D0
:105530001A4321463046FFF7C7F964E150B9090123
:1055400041F06D0101F0FD013046FFF736FAC0F37E
:105550004110DAE7012840F056810C0144F06D0457
:10556000E4B221463046FFF728FA3B6820F060029B
:105570005B0103F060031A4321463046FFF7A4F9AC
:1055800041E158B9090141F06D0101F0FD013046DA
:10559000FFF713FA00F00F00386034E1012840F003
:1055A00032810C0144F06D04E4B221463046FFF72D
:1055B00004FA3B6820F00F0203F00F031A43214660
:1055C0003046FFF781F91EE150B9090141F06D0144
:1055D00001F0FD013046FFF7F0F9C0F3006094E7F9
:1055E000012840F010810C0144F06D04E4B2214622
:1055F0003046FFF7E2F93B6820F080721B0603F0AB
:1056000080731A4321463046FFF75EF9FBE098B9F4
:10561000090141F06D0101F0FD013046FFF7CDF9C0
:10562000001410F0400F00F07F0214BF6FF07F03F2
:10563000002313433B60E3E0012840F0E4800C01C9
:1056400044F06D04E4B221463046FFF7B6F93B68FA
:1056500020F4FE021B0403F4FE031A4321463046E5
:10566000FFF732F9CFE058B9090141F06C0101F0C0
:10567000FC013046FFF7A1F9C0F340403860C2E0BA
:10568000012840F0C0800C0144F06C04E4B22146D3
:105690003046FFF792F93B6820F400325B0403F4D4
:1056A00000331A4321463046FFF70EF9ABE00028DD
:1056B0007FF411AB090141F06F01C9B23046FFF729
:1056C0007CF9C0F3044020E700283FF4DDAC01285A
:1056D00040F0998020248C4064B244F0110144F0E1
:1056E00014041A683046E4B2C9B2FFF7EDF8214657
:1056F0003046FFF762F93B6820F48062002B14BF4C
:105700004FF4806300231A4321463046FFF7DCF84C
:1057100079E050B9090141F06C0101F0FC0130461B
:10572000FFF74BF9C0F34030EFE601286BD10C01D5
:1057300044F06C04E4B221463046FFF73EF93B6882
:1057400020F400525B0303F400531A432146304611
:10575000FFF7BAF857E000287FF4BDAA090141F02D
:105760006F01C9B23046FFF728F9C0F30900CCE653
:10577000D0B961B1012943D101463046FFF71DF987
:1057800000F06000A0F1200358425841BDE60846F1
:10579000FFF713F900F01800A0F110025042504139
:1057A00038603046BDE8F88301282CD111B10129B9
:1057B00011D028E00846FFF700F93B6820F01800F8
:1057C00013B140F0100201E040F008020021084649
:1057D000FFF77AF817E000213046FFF7EEF83B6854
:1057E00020F0600013B140F0200201E040F04002E0
:1057F00000210120FFF768F805E00420BDE8F883E8
:105800002046BDE8F8830020BDE8F88307B50129EC
:10581000019205D8024601AB0120FFF736F900E0FE
:10582000082003B05DF804FB0129134603D80246A3
:105830000020FFF72AB90820704708B52221002070
:10584000FFF7BBF850B942210120FFF7B6F828B99D
:10585000034B1868BDE808400BF0CCBD002008BD24
:105860009853002070B52D4E2D480BF043FDF46881
:105870002C4D636803F5AA7203F1C80003F5B873F1
:10588000AB6023686A60DB682860984723686868B3
:105890001B6998472368A8681B6998473269224B9F
:1058A00022491A606368022003F537735360204B66
:1058B0005A690A601F49C2F804121F49C2F8081247
:1058C00001211170002151701C4A18741A621C4A7F
:1058D000DA611C4A9A611C4A5A621C4A9A631C4A41
:1058E0005A631C4A9A621C4ADA621C4A9A641C4A2D
:1058F0005A641C4A5A651C4A1A651C4ADA641C4AD6
:105900001A661C4ADA653222DA604FF48C729A60A9
:10591000194A9A65BDE87040FEF764BF2866020820
:10592000A0530020981600209C530020985300207C
:10593000183900203B5801089947010859490108C6
:10594000B9490108B5490108B149010829580108B8
:105950000D580108EF480108694A0108E5480108A7
:10596000594A01086D470108A54701084947010840
:10597000E5470108614701082548010801289FBF44
:10598000034B53F8203000200B6088BF082070477D
:105990003C560020014B00225A6070471839002005
:1059A00070B50446074E084D33682A46014600206C
:1059B0000BF071FD33682A462146BDE87040012096
:1059C0000BF069BD385600203C560020014B18688A
:1059D0000BF0C3BD38560020012810B5144616D070
:1059E00008D302281FD1114B114ADB6890681B684D
:1059F0001B6A12E014680D4A0D4BD268126824B17C
:105A00005269D8689047002010BD9269F9E7074BAA
:105A1000074ADB6850681B681B6A9847003018BF4C
:105A200001202060EFE7042010BD00BF28660208B7
:105A3000B0160020022804BF0B4B93F8D00020B909
:105A40000A4BDB681B685B690AE001280BD1064B37
:105A500093F8D030012B06D1044BDB681B689B699F
:105A6000034A106818477047183900202866020852
:105A7000B016002070B50020FFF7DCFF104B114C72
:105A8000DD6820682B689B6898472B6860689B6876
:105A900098472B68A0689B6898472B68A0699B680B
:105AA00098472B6820699B6898472B6860699B68BA
:105AB00098472B68E0689B68BDE87040184700BFB6
:105AC00028660208B01600202DE9F8430F469146DB
:105AD0009846174C0021236847F080009B689DF88A
:105AE00020609DF824509847236800219B68484611
:105AF0009847236800219B68404698472368002107
:105B00009B6830469847236828469B680121984740
:105B1000084B48EA09281B6846EA082607F07F0771
:105B200003EB870745EA06257D60BDE8F88300BFE3
:105B3000D45800203856002007B5D3B20193C2F3E1
:105B400007230093C2F30743120EFFF7BDFF03B014
:105B50005DF804FB0A4601460020FFF7EDBF01286F
:105B6000F7B505460F4627D8154C044494F89432EF
:105B700073B1144B202181401B6841F0070103EBF6
:105B800081035A68C9B2FFF7D7FF002384F8943223
:105B90002026AE4046F00D0100243A46C9B2284600
:105BA000FFF7CAFF28460194009423462246F1B22B
:105BB000FFF78AFF204600E0082003B0F0BD00BFD9
:105BC0003C56002038560020012873B505460C4687
:105BD00021D82026864084EAE47246F00701A2EB31
:105BE000E472C9B2FFF7A8FF0C4B002C2B444FF016
:105BF000010283F89422A8BF13464FF00004B8BFF7
:105C0000022301932846009423462246F1B2FFF76F
:105C10005BFF204600E0082002B070BD3C5600202B
:105C20000021D1E74942CFE7CEE738B5234B01F059
:105C30007F04234493F81432DB0705D4204B1B6800
:105C400003EB8404606838BD1E4D00212B6820469C
:105C50009B6898472B6800219B68084698472B68EB
:105C600000219B68084698472B6800219B680846DE
:105C700098472B6801219B68002098472B680021DA
:105C80009B68204698472B6800219B6808469847E8
:105C90002B68002104029B68084698472B68002166
:105CA000204304029B68084698472B68204304025F
:105CB0009B68012100209847204338BD3C560020B6
:105CC00038560020D458002010B50C46014600205C
:105CD000FFF7ABFF206010BD38B50D462021814095
:105CE00041F00101C9B20446FFF79FFF2968014452
:105CF00029602046BDE8384031E71C2A2DE9F041F3
:105D000004460E461F4600F08E835DD80C2A00F034
:105D100000822BD8052A00F0588113D8022A00F0FF
:105D2000EA8007D8002A00F0AD80012A00F0C88080
:105D300000F0E3BF032A00F00081042A00F015817F
:105D400000F0DBBF082A00F0AD8107D8062A00F07A
:105D50005881072A00F07E8100F0CFBF0A2A00F0A8
:105D6000B2810B2A00F0C28100F0C7BF122A00F0F6
:105D7000968213D80F2A00F0398207D80D2A00F036
:105D8000F1810E2A00F0168200F0B7BF102A00F051
:105D90004982112A00F0678200F0AFBF152A00F097
:105DA000D28207D8132A00F09682142A00F0AF821C
:105DB00000F0A3BF172A00F0FE82C0F0E082182A8C
:105DC00000F0158300F099BFAC2A00F0BF852AD8F7
:105DD000A52A00F02E8413D8A22A00F0B28307D897
:105DE0001D2A00F048838C2A00F04F8300F085BF05
:105DF000A32A00F0CE83A42A00F0F38300F07DBF35
:105E0000A82A00F0048507D8A62A00F07E84A72AD5
:105E100000F0D68400F071BFAA2A00F0478540F256
:105E20001D8500F06BBDB62A00F0A98213D8B32AF5
:105E300000F00B8607D8AD2A00F0AF85AE2A00F03F
:105E4000D48500F05ABFB42A00F02786B52A00F0A6
:105E5000348600F052BFCE2A00F0BA8607D8B82A9E
:105E600000F06686B92A00F08B8600F046BFD22A81
:105E700000F0DA86D32A00F0F386D12A40F03D877D
:105E800000F0B6BE58B92021B14041F00D01C9B2B1
:105E90003046FFF7CAFE38600020BDE8F0810128D7
:105EA00002D00020BDE8F0812021B14041F00D0179
:105EB00030461A68C9B2FFF73FFE0020BDE8F08106
:105EC00058B92021B14041F00101C9B23046FFF775
:105ED000ACFE38602046BDE8F0810128E1D12021E8
:105EE000B14041F0010130461A68C9B2FFF724FE03
:105EF0000020BDE8F08158B92021B14041F00701F0
:105F0000C9B23046FFF791FE38602046BDE8F08107
:105F10000128C6D1CA4B0B4483F894023A68202169
:105F2000B140002A41F007013046B8BF5242C9B221
:105F3000FFF702FE0020BDE8F08188B92021B140C2
:105F400041F00201C9B23046FFF76FFE10F40003C2
:105F500018BF4FF07F4303433B600020BDE8F08152
:105F6000012C9ED10420BDE8F08160B9B54B202002
:105F70001B68884040F0070003EB80004368204620
:105F80003B60BDE8F08101288BD1AE4B3A682021FF
:105F9000B1401B6841F00704002A03EB8403B8BF3B
:105FA00052425A60C9B23046FFF73FFE054600280C
:105FB0007FF477AF3A683046002AB8BF5242E1B268
:105FC000FFF7BAFD2846BDE8F08158B92021B1405D
:105FD00041F00601C9B23046FFF727FE386020467F
:105FE000BDE8F08101287FF45CAF2021B14041F091
:105FF000060130461A68C9B2FFF79EFD0020BDE8D1
:10600000F08168B92021B14041F01001C9B2304699
:10601000FFF70BFEC0F3042038600020BDE8F081DC
:1060200001287FF43EAF20248C4044F01004E4B2F9
:1060300021463046FFF7F9FD3B6820F4F8521B0279
:1060400003F4F85330461A432146FFF775FD00204C
:10605000BDE8F08168B92021B14041F01001C9B21A
:106060003046FFF7E2FD00F01F0038602046BDE833
:10607000F08101287FF415AF20248C4044F01004F7
:10608000E4B221463046FFF7D0FD3B6820F01F0206
:1060900003F01F0330461A432146FFF74DFD002051
:1060A000BDE8F08100287FF45BAF2021B14041F0D2
:1060B0001501C9B23046FFF7B8FDC0F34020386083
:1060C0002046BDE8F08100287FF44AAF2021B1408E
:1060D00041F01501C9B23046FFF7A7FDC0F34000FB
:1060E00080F0010038600020BDE8F08100287FF4D6
:1060F00037AF2021B14041F01501C9B23046FFF75A
:1061000094FD00F0010080F0010038602046BDE8F9
:10611000F08168B92021B14041F01401C9B2304684
:10612000FFF783FDC0F3400038602046BDE8F081F2
:1061300001287FF4B6AE20248C4044F01404E4B26D
:1061400021463046FFF771FD3B6820F002025B00FC
:1061500003F0020330461A432146FFF7EDFC00200E
:10616000BDE8F08168B92021B14041F01401C9B205
:106170003046FFF75AFD00F0010038600020BDE80E
:10618000F08101287FF48DAE20248C4044F014046B
:10619000E4B221463046FFF748FD3B6820F001029B
:1061A00003F0010330461A432146FFF7C5FC0020E7
:1061B000BDE8F08158B92021B14041F01401C9B2C5
:1061C0003046FFF732FD38602046BDE8F0810128F7
:1061D0007FF467AE2021B14041F0140130461A68C7
:1061E000C9B2FFF7A9FC0020BDE8F08158B9202111
:1061F000B14041F00401C9B23046FFF716FD3860E6
:106200002046BDE8F08101287FF44BAE2021B1404B
:1062100041F0040130461A68C9B2FFF78DFC002036
:10622000BDE8F08180B92021B14041F00501C9B23B
:106230003046FFF7FAFC38600020BDE8F08100BF6F
:106240003C5600203856002001287FF42AAE202139
:10625000B14041F0050130461A68C9B2FFF76CFC45
:106260000020BDE8F08158B92021B14041F008017B
:10627000C9B23046FFF7D9FC38602046BDE8F0814E
:1062800001287FF40EAE2021B14041F008013046D4
:106290001A68C9B2FFF750FC0020BDE8F08158B978
:1062A0002021B14041F00A01C9B23046FFF7BDFCE0
:1062B00038602046BDE8F08101287FF4F2AD20214E
:1062C000B14041F00A0130461A68C9B2FFF734FC08
:1062D0000020BDE8F08158B92021B14041F0030110
:1062E000C9B23046FFF7A1FC38600020BDE8F0815C
:1062F00001287FF4D6AD2021B14041F003013046A2
:106300001A68C9B2FFF718FC0020BDE8F08158B93F
:106310002021B14041F00B01C9B23046FFF785FCA6
:1063200038602046BDE8F08101287FF4BAAD202115
:10633000B14041F00B0130461A68C9B2FFF7FCFBCF
:106340000020BDE8F08158B92021B14041F00C0196
:10635000C9B23046FFF769FC38602046BDE8F081DD
:1063600001287FF49EAD2021B14041F00C01304660
:106370001A68C9B2FFF7E0FB0020BDE8F0815CB904
:106380002021B14041F01101C9B23046FFF74DFC68
:1063900038600020BDE8F081012C7FF482AD20211F
:1063A000B14041F0110130463A68C9B2FFF7C4FB71
:1063B0000020BDE8F08158B92021B14041F0120120
:1063C000C9B23046FFF731FC38600020BDE8F081EB
:1063D00001287FF466AD2021B14041F01201304622
:1063E0001A68C9B2FFF7A8FB0020BDE8F08158B9D0
:1063F0002021B14041F01301C9B23046FFF715FC2E
:1064000038602046BDE8F08101287FF44AAD2021A4
:10641000B14041F0130130461A68C9B2FFF78CFB56
:106420000020BDE8F08168B9090141F06C0101F07C
:10643000FC013046FFF7F9FBC0F38040386020468E
:10644000BDE8F08101287FF42CAD0C0144F06C0410
:10645000E4B221463046FFF7E8FB3B6820F4802297
:106460009B0403F4802330461A432146FFF764FB64
:106470000020BDE8F08100287FF472ADCF4B0020F2
:1064800053F821303B60BDE8F08188B9090141F043
:106490006C0101F0FC013046FFF7C7FB4FF480733D
:1064A000C0F3036043FA00F038602046BDE8F08195
:1064B00001287FF4F6AC1B68102B1FD00CDC022BDC
:1064C00018D003DC012B1FD108231FE0042B13D0AD
:1064D000082B19D1052319E0402B11D003DC202B08
:1064E00012D1032312E0802B0CD0B3F5807F0BD1A7
:1064F00000230BE0072309E0062307E0042305E05F
:10650000022303E0386002E04FF0FF333B603B685A
:1065100001333FF4C6AC340144F06C04E4B22146CC
:106520003046FFF782FB3B6820F070621B0603F0E9
:10653000706330461A432146FFF7FEFA0020BDE89B
:10654000F08168B9090141F06C0101F0FC013046AD
:10655000FFF76BFBC0F3C13038602046BDE8F08127
:1065600001287FF49EAC0C0144F06C04E4B2214697
:106570003046FFF75AFB3B6820F4C032DB0303F4DC
:10658000C03330461A432146FFF7D6FA0020BDE853
:10659000F08168B9090141F06C0101F0FC0130465D
:1065A000FFF743FBC0F3803038600020BDE8F08186
:1065B00001287FF476AC0C0144F06C04E4B221466F
:1065C0003046FFF732FB3B6820F480429B0303F424
:1065D000804330461A432146FFF7AEFA0020BDE85B
:1065E000F08168B9090141F06C0101F0FC0130460D
:1065F000FFF71BFBC0F3003038602046BDE8F08198
:1066000001287FF44EAC0C0144F06C04E4B2214646
:106610003046FFF70AFB3B6820F480521B0303F46B
:10662000805330461A432146FFF786FA0020BDE822
:10663000F08148BB0D0145F06C05EDB229463046AE
:10664000FFF7F3FAC0F3803829463046B8F1000F5F
:1066500007D0FFF7EAFAC0F3C31038602046BDE860
:10666000F081FFF7E2FAC0F30210386029463046A5
:10667000FFF7DBFA04057FF514AC3B68404643F0B6
:1066800008033B60BDE8F08101287FF40AAC0C01EF
:1066900044F06C04E4B221463046FFF7C6FA10F429
:1066A0008045214630460FD0FFF7BFFA3B6820F403
:1066B000F062DB0103F4F06330461A432146FFF732
:1066C0003BFA0020BDE8F081FFF7AFFA3B6820F409
:1066D000006213F0080F18BF4FF400652A432146EB
:1066E0003046FFF729FA21463046FFF79EFA3B680D
:1066F00020F070021B0103F0700330461A4321465C
:10670000FFF71AFA0020BDE8F08138BB0C0144F015
:106710006C04E4B221463046FFF787FA10F4804556
:106720002146304607D0FFF780FAC0F302103860E8
:106730000020BDE8F081FFF778FAC0F3C31038609D
:1067400021463046FFF771FA00057FF5AAAB3B689A
:10675000284643F008033B60BDE8F08101287FF440
:10676000A0AB0C0144F06C04E4B221463046FFF7C4
:106770005CFA10F48045214630460FD0FFF755FAF9
:106780003B6820F070021B0103F0700330461A438F
:106790002146FFF7D1F90020BDE8F081FFF745FA67
:1067A0003B6820F4F062DB0103F4F06330461A43E7
:1067B0002146FFF7C1F92846BDE8F0813C5600208C
:1067C00068B9090141F06C0101F0FC013046FFF7A6
:1067D0002CFA00F00F0038602046BDE8F081012857
:1067E0007FF45FAB0C0144F06C04E4B22146304608
:1067F000FFF71BFA3B6820F00F0203F00F0330464F
:106800001A432146FFF798F90020BDE8F08168B9E6
:10681000090141F06D0101F0FD013046FFF705FA75
:10682000C0F3C03038602046BDE8F08101287FF415
:1068300038AB0C0144F06D04E4B221463046FFF75A
:10684000F4F93B6820F40042DB039BB230461A4364
:106850002146FFF771F90020BDE8F08168B9090110
:1068600041F06D0101F0FD013046FFF7DEF9C0F3A4
:10687000413038602046BDE8F08101287FF411AB3B
:106880000C0144F06D04E4B221463046FFF7CDF927
:106890003B6820F4C0425B0303F4C04330461A4314
:1068A0002146FFF749F90020BDE8F08168B90901E8
:1068B00041F06D0101F0FD013046FFF7B6F9C0F37C
:1068C000032038600020BDE8F08101287FF4E9AAA8
:1068D0000C0144F06D04E4B221463046FFF7A5F9FF
:1068E0003B6820F470621B0203F4706330461A4365
:1068F0002146FFF721F90020BDE8F08168B90901C0
:1069000041F06D0101F0FD013046FFF78EF9C0F353
:10691000411038602046BDE8F08101287FF4C1AA0B
:106920000C0144F06D04E4B221463046FFF77DF9D6
:106930003B6820F060025B0103F0600330461A43BD
:106940002146FFF7F9F80020BDE8F08168B9090198
:1069500041F06D0101F0FD013046FFF766F900F0EE
:106960000F0038602046BDE8F08101287FF499AA25
:106970000C0144F06D04E4B221463046FFF755F9AE
:106980003B6820F00F0203F00F0330461A43214604
:10699000FFF7D2F80020BDE8F08168B9090141F0A5
:1069A0006D0101F0FD013046FFF73FF9C0F30060D3
:1069B00038600020BDE8F08101287FF472AA0C0144
:1069C00044F06D04E4B221463046FFF72EF93B68EF
:1069D00020F080721B0603F0807330461A43214674
:1069E000FFF7AAF80020BDE8F081A8B9090141F03D
:1069F0006D0101F0FD013046FFF717F9001410F0AA
:106A0000400F00F07F0214BF6FF07F030023134399
:106A10003B602046BDE8F08101287FF442AA0C01CA
:106A200044F06D04E4B221463046FFF7FEF83B68BF
:106A300020F4FE021B0403F4FE0330461A432146F1
:106A4000FFF77AF80020BDE8F08168B9090141F04C
:106A50006C0101F0FC013046FFF7E7F8C0F340405D
:106A600038602046BDE8F08101287FF41AAA0C01A5
:106A700044F06C04E4B221463046FFF7D6F83B6898
:106A800020F400325B0403F4003330461A432146FD
:106A9000FFF752F80020BDE8F08100287FF460AADB
:106AA000090141F06F01C9B23046FFF7BEF8C0F3EB
:106AB000044038600020BDE8F081A8B920258D4051
:106AC0006DB245F01401C9B23046FFF7AEF841058A
:106AD0007FF5E7A945F01101C9B23046FFF7A5F8E7
:106AE00038602046BDE8F08101287FF4DAA920242F
:106AF0008C4064B244F0110144F014041A6830462A
:106B0000E4B2C9B2FFF718F821463046FFF78DF816
:106B10003B6820F48062002B14BF4FF48063002395
:106B200030461A432146FFF707F80020BDE8F08100
:106B300068B9090141F06C0101F0FC013046FFF732
:106B400074F8C0F3403038600020BDE8F0810128BF
:106B50007FF4A7A90C0144F06C04E4B2214630464E
:106B6000FFF763F83B6820F400525B0303F4005323
:106B700030461A432146FEF7DFFF0020BDE8F081D2
:106B800068B9090141F06C0101F0FC013046FFF7E2
:106B90004CF8C0F3035038602046BDE8F08101286E
:106BA0007FF47FA90C0144F06C04E4B22146304626
:106BB000FFF73BF83B6820F470021B0503F47003F9
:106BC00030461A432146FEF7B7FF0020BDE8F081AA
:106BD00000287FF4C5A9090141F06F01C9B2304610
:106BE000FFF723F8C0F3090038602046BDE8F081C4
:106BF00058B92021B14041F01901C9B23046FFF720
:106C000014F838602046BDE8F08101287FF449A9D6
:106C10002021B14041F0190130461A68C9B2FEF78F
:106C20008BFF0020BDE8F08158B92021B14041F030
:106C30001A01C9B23046FEF7F8FF38600020BDE8FF
:106C4000F08101287FF42DA92021B14041F01A01E3
:106C500030461A68C9B2FEF76FFF0020BDE8F08128
:106C6000E8B979B101294BD101463046FEF7DDFF85
:106C700000F06000A0F120035842584138602046DF
:106C8000BDE8F0810846FEF7D0FF00F01800A0F143
:106C900010025042504138603046BDE8F081012872
:106CA0007FF4FFA811B1012913D02BE00846FEF7AD
:106CB000BCFF3B6820F0180013B140F0100201E067
:106CC00040F0080200210846FEF736FF0020BDE82C
:106CD000F08100213046FEF7A8FF3B6820F06000FD
:106CE00013B140F0200201E040F0400200210120F9
:106CF000FEF722FF0020BDE8F0810420BDE8F0810E
:106D0000BDE8F0810020BDE8F08107B501290192BE
:106D100005D8024601AB0120FEF7EFFF00E0082096
:106D200003B05DF804FB0129134603D80246002096
:106D3000FEF7E3BF0820704708B522210020FEF7C8
:106D400074FF50B942210120FEF76FFF28B9044BB0
:106D50001868BDE808400AF0F7BB002008BD00BF76
:106D60003856002070B53D4E3D480AF055FBF56899
:106D70003C4C6B6803F5AA72626003F5B872A260BE
:106D800003F56F72E26003F5767203F1C8002261C9
:106D900003F57D7203F58263A3612B686261DB6892
:106DA000206098472B68E068DB6898472B68E068AC
:106DB0009B6998472B6860681B6998472B68A06897
:106DC0001B6998472B68A0691B6998472B68206945
:106DD0001B6998472B6860691B6998473269224B89
:106DE00022491A606B68012003F537735360204B0A
:106DF0005A690A601F491070C2F804121E49C2F88D
:106E00000812002151701D4A1A621D4ADA611D4A9A
:106E10009A611D4A5A621D4A9A631D4A5A631D4A65
:106E20009A621D4ADA621D4A9A641D4A5A641D4AD2
:106E30005A651D4A1A651D4ADA641D4A1A661D4ABA
:106E4000DA6502221A743222DA60DE229A601A4A65
:106E50009A65BDE87040FEF7EDBD00BF28660208E8
:106E60003C560020B0160020D45800203856002090
:106E700018390020396D0108CD590108C95B010896
:106E8000295C0108255C0108215C0108276D0108C7
:106E90000B6D01085F5B0108D95C0108555B0108B7
:106EA000C95C0108A1590108D95901087D59010897
:106EB000355A010895590108755A010801289FBFE4
:106EC000034B53F8203000200B6088BF0820704728
:106ED000DC580020014B00225A607047183900200E
:106EE00070B50446074E084D33682A460146002017
:106EF0000AF07BFB33682A462146BDE8704001203A
:106F00000AF073BBD8580020DC580020014B1868E9
:106F10000AF0B5BBD8580020012810B5144616D089
:106F200008D302281FD1114B114ADB6890681B68F7
:106F30001B6A12E014680D4A0D4BD268126824B126
:106F40005269D8689047002010BD9269F9E7074B55
:106F5000074ADB6850681B681B6A9847003018BFF7
:106F600001202060EFE7042010BD00BF2866020862
:106F7000D8160020022804BF0B4B93F8D00020B98C
:106F80000A4BDB681B685B690AE001280BD1064BE2
:106F900093F8D030012B06D1044BDB681B689B694A
:106FA000034A1068184770471839002028660208FD
:106FB000D816002070B50020FFF7DCFF104B114CF5
:106FC000DD6820682B689B6898472B6860689B6821
:106FD00098472B68A0689B6898472B68A0699B68B6
:106FE00098472B6820699B6898472B6860699B6865
:106FF00098472B68E0689B68BDE87040184700BF61
:1070000028660208D81600202DE9F8430F4691465D
:107010009846174C0021236847F080009B689DF834
:1070200020609DF824509847236800219B684846BB
:107030009847236800219B684046984723680021B1
:107040009B6830469847236828469B6801219847EB
:10705000084B48EA09281B6846EA082607F07F071C
:1070600003EB870745EA06257D60BDE8F88300BF8E
:10707000745B0020D858002007B5D3B20193C2F347
:1070800007230093C2F30743120EFFF7BDFF03B0BF
:107090005DF804FB0A4601460020FFF7EDBF01281A
:1070A000F7B505460F4627D8154C044494F894329A
:1070B00073B1144B202181401B6841F0070103EBA1
:1070C00081035A68C9B2FFF7D7FF002384F89432CE
:1070D0002026AE4046F00D0100243A46C9B22846AB
:1070E000FFF7CAFF28460194009423462246F1B2D6
:1070F000FFF78AFF204600E0082003B0F0BD00BF84
:10710000DC580020D8580020012873B505460C46ED
:1071100021D82026864084EAE47246F00701A2EBDB
:10712000E472C9B2FFF7A8FF0C4B002C2B444FF0C0
:10713000010283F89422A8BF13464FF00004B8BFA1
:10714000022301932846009423462246F1B2FFF71A
:107150005BFF204600E0082002B070BDDC58002034
:107160000021D1E74942CFE7CEE738B5234B01F004
:107170007F04234493F81432DB0705D4204B1B68AB
:1071800003EB8404606838BD1E4D00212B68204647
:107190009B6898472B6800219B68084698472B6896
:1071A00000219B68084698472B6800219B68084689
:1071B00098472B6801219B68002098472B68002185
:1071C0009B68204698472B6800219B680846984793
:1071D0002B68002104029B68084698472B68002111
:1071E000204304029B68084698472B68204304020A
:1071F0009B68012100209847204338BDDC580020BF
:10720000D8580020745B002010B50C4601460020C1
:10721000FFF7ABFF206010BD38B50D46202181403F
:1072200041F00101C9B20446FFF79FFF29680144FC
:1072300029602046BDE8384031E71C2A2DE9F3419A
:1072400004460E461F4600F03C835DD80C2A00F031
:10725000D6812BD8052A00F0428113D8022A00F0EB
:10726000E18007D8002A00F0AE80012A00F0C58036
:1072700000F0CABE032A00F0F180042A00F0058164
:1072800000F0C2BE082A00F08C8107D8062A00F060
:107290003B81072A00F05F8100F0B6BE0A2A00F0A9
:1072A0008F810B2A00F09C8100F0AEBE122A00F004
:1072B000718213D80F2A00F0268207D80D2A00F019
:1072C000D5810E2A00F00A8200F09EBE102A00F03E
:1072D0002E82112A00F04A8200F096BE152A00F094
:1072E0009A8207D8132A00F06982142A00F080825B
:1072F00000F08ABE172A00F0B982C0F09F82182AD7
:1073000000F0CC8200F080BEAB2A00F0EA842BD8DB
:10731000A52A00F0C28313D8A22A00F0548307D80C
:107320001D2A00F0F1828C2A00F0F68200F06CBE7B
:10733000A32A00F06B83A42A00F08C8300F064BEC3
:10734000A82A00F0628407D8A62A00F0F183A72AB1
:1073500000F0398400F058BEA92A00F07B84AA2AE4
:1073600000F09C8400F050BEB52A00F0808513D850
:10737000AE2A00F01F8507D8AC2A00F0D584AD2ACC
:1073800000F0F58400F040BEB32A00F03F85B42A37
:1073900000F0608500F038BECE2A00F09C8507D84A
:1073A000B62A00F04B82B82A00F0308300F02CBEE1
:1073B000D22A00F0B585D32A00F0C985D12A40F041
:1073C000238600F095BD50B92021B14041F00D0158
:1073D000C9B23046FFF7C9FE386000F017BE012879
:1073E00040F014862021B14041F00D011A68C9B265
:1073F0003046FFF741FE00F009BE28B92021B14018
:1074000041F0010100F079BD012840F0FF85202105
:10741000B14041F001011A68C9B23046FFF72CFEB5
:1074200000F0F4BD28B92021B14041F0070100F07F
:1074300064BD012840F0EA85CA4B0B4483F89402EE
:107440003A682021B140002A41F00701B8BF5242FA
:10745000C9B23046FFF710FE00F0D8BD80B9202138
:10746000B14041F00201C9B23046FFF77EFE10F490
:10747000000318BF4FF07F4303433B6000F0C6BDDD
:10748000012C00F0C18500F0C1BD50B9B64B2020E1
:107490001B68884040F0070003EB8000436800F061
:1074A0009CBC012840F0B285AF4B3A682021B14026
:1074B0001B6841F00704002AB8BF524203EB840363
:1074C0005A60C9B23046FFF750FE002840F09E8552
:1074D0003A68E1B2002AB8BF524200F091BD28B923
:1074E0002021B14041F0060100F007BD012840F025
:1074F0008D852021B14041F006011A68C9B230469D
:10750000FFF7BAFD00F082BD60B92021B14041F023
:107510001001C9B23046FFF728FEC0F307203860DB
:1075200000F074BD012840F0718520248C4044F0A7
:107530001004E4B221463046FFF717FEC3B20193B0
:107540003B78002200932146C0F307433046FFF703
:107550005BFD00F05BBD50B92021B14041F010014E
:10756000C9B23046FFF701FEC0B200F0CABC012824
:1075700040F04C8520248C4044F01004E4B22146B5
:107580003046FFF7F2FD3B7800220193C0F307235A
:1075900000932146C0F307433046FFF735FD00F066
:1075A00035BD00287FF46CAF2021B14041F01501BA
:1075B000C9B23046FFF7D9FDC0F3402000F0A1BCAE
:1075C00000287FF45DAF2021B14041F01501C9B220
:1075D0003046FFF7CAFDC0F34000386000F016BD2A
:1075E00000287FF44DAF2021B14041F01501C9B210
:1075F0003046FFF7BAFD00F0010000F082BC58B938
:107600002021B14041F01401C9B23046FFF7ADFD71
:10761000C0F3400000F075BC012840F0F78420243E
:107620008C4044F01404E4B221463046FFF79DFD3F
:107630003B6820F00202002BCCBF022300231A4338
:1076400021463046FFF718FD21463046FFF78DFDF5
:107650003B6820F00802022B0CBF082300231A43CA
:1076600021463046FFF708FD00F0D0BC60B920216C
:10767000B14041F01401C9B23046FFF776FD00F089
:107680000100386000F0C2BC012840F0BF84202413
:107690008C4044F01404E4B221463046FFF765FD07
:1076A0003A6820F00100002AD4BF024640F00102EF
:1076B00021463046FFF7E0FC21463046FFF755FDF6
:1076C0003B6820F00402022B0CBF042300231A4362
:1076D00021463046FFF7D0FC00F098BC28B92021A5
:1076E000B14041F0140100F008BC012840F08E8444
:1076F0002021B14041F014011A68C9B23046FFF7A9
:10770000BBFC00F083BC20B92021B14041F0040152
:10771000F3E3012840F07A842021B14041F00401D4
:107720001A68C9B23046FFF7A7FC00F06FBC50B929
:107730002021B14041F00501C9B23046FFF715FDE7
:10774000386000F063BC012840F060842021B14023
:1077500041F005011A68C9B23046FFF78DFC00F010
:1077600055BC00BFDC580020D858002020B920218B
:10777000B14041F00801C0E3012840F047842021D6
:10778000B14041F008011A68C9B23046FFF774FCF5
:1077900000F03CBC20B92021B14041F00A01ACE32B
:1077A000012840F033842021B14041F00A011A68D9
:1077B000C9B23046FFF760FC00F028BC50B9202168
:1077C000B14041F00301C9B23046FFF7CEFC38604A
:1077D00000F01CBC012840F019842021B14041F088
:1077E00003011A68C9B23046FFF746FC00F00EBC30
:1077F00020B92021B14041F00B017EE3012840F087
:1078000005842021B14041F00B011A68C9B230460D
:10781000FFF732FCFAE320B92021B14041F00C011E
:107820006BE3012840F0F2832021B14041F00C01CC
:107830001A68C9B23046FFF71FFCE7E34CB92021B4
:10784000B14041F01101C9B23046FFF78EFC3860FB
:10785000DCE3012C40F0DA832021B14041F011013A
:107860003A68C9B23046FFF707FCCFE348B9202198
:10787000B14041F01201C9B23046FFF776FC3860E2
:10788000C4E3012840F0C2832021B14041F012013D
:107890001A68C9B23046FFF7EFFBB7E320B92021E1
:1078A000B14041F0130128E3012840F0AF832021CB
:1078B000B14041F013011A68C9B23046FFF7DCFB52
:1078C000A4E350B9090141F06C0101F0FC0130461C
:1078D000FFF74BFCC0F3804013E3012840F0968390
:1078E0000C0144F06C04E4B221463046FFF73DFC45
:1078F0003B6820F480229B0403F480231A43214632
:107900003046FFF7B9FB81E300287FF4B9ADC54BE2
:1079100053F821303B6079E370B9090141F06C0103
:1079200001F0FC013046FFF720FC4FF4807300F0BB
:107930000F0043FA00F0E4E2012840F067831B687F
:10794000102B1FD00CDC022B18D003DC012B1FD115
:1079500008231FE0042B13D0082B19D1052319E0AD
:10796000402B11D003DC202B12D1032312E0802BFB
:107970000CD0B3F5807F0BD100230BE0072309E087
:10798000062307E0042305E0022303E0386002E059
:107990004FF0FF333B603B68013300F03783340125
:1079A00044F06C04E4B221463046FFF7DEFB3B684E
:1079B00020F070621B0603F070631A4321463046C4
:1079C000FFF75AFB22E350B9090141F06C0101F0C5
:1079D000FC013046FFF7C9FBC0F3C13091E201283A
:1079E00040F014830C0144F06C04E4B221463046AC
:1079F000FFF7BBFB3B6820F4C032DB0303F4C0336A
:107A00001A4321463046FFF737FBFFE25CB93101EC
:107A100041F06C0101F0FC013046FFF7A6FBC0F31A
:107A200040303860F2E2012C40F0F082340144F042
:107A30006C04E4B221463046FFF797FB3B6820F424
:107A400000525B0303F400531A4321463046FFF70C
:107A500013FBDBE250B9090141F06C0101F0FC01BC
:107A60003046FFF782FBC0F300304AE2012840F0C5
:107A7000CD820C0144F06C04E4B221463046FFF79D
:107A800074FB3B6820F480521B0303F480531A43B9
:107A900021463046FFF7F0FAB8E20D0145F06C05DB
:107AA000EDB229463046FFF760FBC0F3803874B969
:107AB00029463046B8F1000F04D0FFF756FBC0F35B
:107AC000C3101EE2FFF751FBC0F3021054E0012C7B
:107AD00040F09C8229463046B8F1000F0DD0FFF7E8
:107AE00044FB3B6820F4F062DB0103F4F0631A43CB
:107AF00029463046FFF7C0FA88E2FFF736FB3B68BD
:107B000020F4006213F0080F14BF4FF40063002349
:107B10001A4329463046FFF7AFFA29463046FFF7A9
:107B200024FB3B6820F070021B0103F0700344E06B
:107B30000D0145F06C05EDB229463046FFF715FB07
:107B4000C0F38038DCB929463046B8F1000F05D0C3
:107B5000FFF70BFBC0F30210386057E2FFF705FB9D
:107B6000C0F3C310386029463046FFF7FEFA3B6881
:107B7000000A00F0080018433860404647E2012C34
:107B800040F0448229463046B8F1000F0DD0FFF78F
:107B9000ECFA3B6820F070021B0103F070031A43FB
:107BA00029463046FFF768FA30E2FFF7DEFA3B6815
:107BB00020F4F062DB0103F4F0631A4329463046F7
:107BC000FFF75AFAD9E750B9090141F06C0101F009
:107BD000FC013046FFF7C9FA00F00F0091E10128DF
:107BE00040F014820C0144F06C04E4B221463046AB
:107BF000FFF7BBFA3B6820F00F0203F00F031A43B4
:107C000021463046FFF738FA00E268B9090141F031
:107C10006D0101F0FD013046FFF7A7FAC0F3C03057
:107C20006FE100BFDC580020012840F0EF810C011B
:107C300044F06D04E4B221463046FFF796FA3B6803
:107C400020F40042DB039BB21A4321463046FFF783
:107C500013FADBE158B9090141F06D0101F0FD01B2
:107C60003046FFF782FAC0F341303860CEE1012898
:107C700040F0CC810C0144F06D04E4B22146304662
:107C8000FFF773FA3B6820F4C0425B0303F4C04380
:107C90001A4321463046FFF7EFF9B7E150B9090121
:107CA00041F06D0101F0FD013046FFF75EFAC0F3CF
:107CB000032026E1012840F0A9810C0144F06D0465
:107CC000E4B221463046FFF750FA3B6820F4706278
:107CD0001B0203F470631A4321463046FFF7CCF9C8
:107CE00094E150B9090141F06D0101F0FD01304608
:107CF000FFF73BFAC0F3411003E1012840F0868111
:107D00000C0144F06D04E4B221463046FFF72DFA31
:107D10003B6820F060025B0103F060031A432146D8
:107D20003046FFF7A9F971E158B9090141F06D0139
:107D300001F0FD013046FFF718FA00F00F0038603F
:107D400064E1012840F062810C0144F06D04E4B26A
:107D500021463046FFF709FA3B6820F00F0203F096
:107D60000F031A4321463046FFF786F94EE150B91A
:107D7000090141F06D0101F0FD013046FFF7F5F911
:107D8000C0F30060BDE0012840F040810C0144F0E8
:107D90006D04E4B221463046FFF7E7F93B6820F076
:107DA00080721B0603F080731A4321463046FFF7AA
:107DB00063F92BE198B9090141F06D0101F0FD0172
:107DC0003046FFF7D2F9001410F0400F00F07F02A8
:107DD00014BF6FF07F03002313433B6092E0012840
:107DE00040F014810C0144F06D04E4B221463046A9
:107DF000FFF7BBF93B6820F4FE021B0403F4FE030B
:107E00001A4321463046FFF737F9FFE058B9090118
:107E100041F06C0101F0FC013046FFF7A6F9C0F318
:107E200040403860F2E0012840F0F0800C0144F05E
:107E30006C04E4B221463046FFF797F93B6820F422
:107E400000325B0403F400331A4321463046FFF747
:107E500013F9DBE000287FF413AB090141F06F0157
:107E6000C9B23046FFF781F9C0F3044049E080B958
:107E700020258D406DB245F01401C9B23046FFF7A0
:107E800074F9C0F3802010B145F0110135E038607D
:107E9000BDE0012840F0BA8020248C4064B244F058
:107EA000110144F014041A683046E4B2C9B2FFF775
:107EB000E3F821463046FFF758F93B6820F480622A
:107EC000002B14BF4FF4806300231A432146304631
:107ED000FFF7D2F89AE000287FF4D2AA090141F016
:107EE0006F01C9B23046FFF740F9C0F3090008E05E
:107EF00050B92021B14041F01901C9B23046FFF715
:107F000034F93860204682E001287FD12021B14039
:107F100041F019011A68C9B23046FFF7ADF875E0B3
:107F200048B92021B14041F01A01C9B23046FFF7EB
:107F30001CF938606AE0012868D12021B14041F085
:107F40001A011A68C9B23046FFF796F85EE0C0B968
:107F500061B101295AD101463046FFF706F900F018
:107F60006000A0F1200358425841CAE70846FFF7D5
:107F7000FCF800F01800A0F11002504250413860A7
:107F800044E0012842D1F9B101293FD10021304616
:107F9000FFF7EBF83B6820F02002002B14BF2023F2
:107FA00000231A4300213046FFF766F800213046CF
:107FB000FFF7DBF83B6820F04002002B0CBF4023AA
:107FC00000231A4300211BE00846FFF7CEF83B6868
:107FD00020F00802002B0CBF082300231A4331466F
:107FE0003046FFF749F831463046FFF7BEF83146D4
:107FF0003B6820F01002002B14BF102300231A430B
:108000003046FFF739F801E0042000E0002002B01C
:10801000BDE8F08107B50129019205D8024601AB00
:108020000120FFF70AF900E0082003B05DF804FB27
:108030000129134603D802460020FFF7FEB80820A6
:10804000704708B522210020FFF78FF850B9422170
:108050000120FFF78AF828B9034B1868BDE80840EB
:1080600009F004BB002008BDD858002070B53D4E73
:108070003D4809F07BFAF5683C4C6B6803F5AA7241
:10808000626003F5B872A26003F56F72E26003F5F7
:10809000767203F1C800226103F57D7203F58263F5
:1080A000A3612B686261DB68206098472B68E068F9
:1080B000DB6898472B68E0689B6998472B68606885
:1080C0001B6998472B68A0681B6998472B68A069B3
:1080D0001B6998472B6820691B6998472B68606962
:1080E0001B6998473269224B22491A606B6802204B
:1080F00003F537735360204B5A690A601F49C2F871
:1081000004121F49C2F80812012111700021517098
:108110001C4A18741A621C4ADA611C4A9A611C4A89
:108120005A621C4A9A631C4A5A631C4A9A621C4A45
:10813000DA621C4A9A641C4A5A641C4A5A651C4AF0
:108140001A651C4ADA641C4A1A661C4ADA6532222D
:10815000DA604FF48C729A60194A9A65BDE87040F3
:10816000FEF708BF28660208DC580020D816002059
:10817000745B0020D8580020183900204380010883
:108180000D6F010809710108697101086571010825
:108190006171010831800108158001089F70010894
:1081A000197201089570010809720108E16E010851
:1081B000196F0108BD6E0108756F0108D56E0108C1
:1081C000B56F010818B9034B1B680B607047082096
:1081D000704700BF7C5B0020014B00225A60704753
:1081E000183900200428F8B5144677D007D801289C
:1081F0003BD011D3022856D0032864D00AE00628C9
:1082000000F09780C0F08E80072800F09E80FC2848
:1082100000F0A7800420F8BD136833F0030240F09B
:10822000B28013F0010F594D594E03D0F3681B680B
:108230001B6906E0F76868683B68DB6898473B683D
:108240009B6968689847206810F0020404D0F368BE
:1082500028681B681B6935E0F66828683368DB68A6
:108260009847336828689B6935E0136844F62062B4
:10827000934200F3888042F210729342444A434B87
:10828000D268586A1268CCBF52699269904742F22C
:108290001172206890FBF2F302FB13003D4B80B299
:1082A0009B6898470FE01468394B74B1DC686068CC
:1082B000236800F50670DB689847236860689B694F
:1082C00000F5067098470020F8BDDB6858681B6809
:1082D00000F506709B6898472046F8BD16682B4D40
:1082E0002B4B4EB1012E11D1DF6828693B68DB684A
:1082F00098473B685B6906E0DF6828693B68DB6894
:1083000098473B689B692869984709E0DE682869B7
:1083100033681B699847336828691B6A9847064683
:108320002660D0E71A4B194ADB68D0691B681B6AC4
:1083300005E0174B154ADB68106A1B681B6A9847F3
:10834000003018BF01202060BDE71368104A012BE0
:10835000D2680E4B126898690CBF526992699047B7
:10836000B1E71468094D0A4B44B1DC6828692368F9
:10837000DB689847236828699B69A3E7DB6828695D
:108380001B681B69A7E71020F8BD00BF001700207D
:1083900028660208B80900201C4B70B5DD681C4C2B
:1083A0002B68A0689B6998472B68A06A9B689847D0
:1083B0002B68606A9B6898472B68E0689B689847C1
:1083C0002B6820699B6898472B6860699B68984771
:1083D0002B6820689B6898472B6860689B68984763
:1083E0002B68E0699B6898472B68206A9B689847D0
:1083F0002B68A0699B6898472B68A0689B68984782
:10840000BDE87040034B5B68184700BF2866020850
:1084100000170020B8090020034B01461B68034ADF
:10842000002007F00CBA00BF785B00207C5B0020C6
:10843000014B186807F03BBA785B0020022804BFA4
:108440000B4B93F8D00020B90A4BDB681B685B69C3
:108450000AE001280BD1064B93F8D030012B06D14E
:10846000044BDB681B689B69034A90681847704798
:108470001839002028660208001700202DE9F0476F
:1084800088460446924699461A4D002155F82030F8
:1084900048F080009B689DF820709DF82460984704
:1084A00055F8243000219B685046984755F82430F1
:1084B00000219B684846984755F8243000219B6866
:1084C0003846984755F8243030469B680121984734
:1084D000094B49EA0A2953F8243047EA092708F0EA
:1084E0007F0803EB880846EA0726C8F80460BDE861
:1084F000F08700BF085E0020785B002007B5D3B28C
:108500000193C2F307230093C2F30743120EFFF750
:10851000B5FF03B05DF804FB0A4601460020FFF7F3
:10852000EDBF38B50D46044690B902462021FFF74D
:10853000E5FF084B20461B682721D3F8A020FFF752
:10854000DDFF20462A462D21FFF7D8FF204638BD03
:10855000082038BD785B002037B50D460446A0B929
:1085600081EAE172A2EBE1722721FFF7C7FF002D3C
:10857000ACBF0123022301932046009423462246E8
:108580002021FFF77BFF204600E0082003B030BD2C
:108590000021E1E74942DFE7DEE72C4A4FF423738D
:1085A00070B503FB002301F07F04234493F80C32E1
:1085B0000546DB0706D4264B53F8203003EB840432
:1085C000606870BD234E002156F8203020469B681D
:1085D000984756F8253000219B680846984756F87A
:1085E000253000219B680846984756F82530002121
:1085F0009B680846984756F8253001219B68002063
:10860000984756F8253000219B682046984756F831
:10861000253000219B680846984756F825300021F0
:1086200004029B680846984756F8253000212043ED
:1086300004029B680846984756F8253020430402F8
:108640009B68012100209847204370BD7C5B00207F
:10865000785B0020085E002010B50C460146002023
:10866000FFF79BFF206010BD38B50C46054648B9A2
:108670002121FFF792FF2168014421602846BDE8CF
:1086800038404EE7082038BD8C2AF8B505460C4620
:108690001E4600F0698359D80E2A00F0F98127D8C8
:1086A000062A00F0418111D8022A00F0DD8007D8A7
:1086B000002A00F0B080012A00F0C38000F056BF0D
:1086C000042A00F0F88040F2E2801AE10A2A00F061
:1086D000768107D8072A00F04781082A00F06381D5
:1086E00000F044BF0C2A00F0898140F27881AAE1B1
:1086F000152A00F0598211D8112A00F0058207D8F6
:108700000F2A00F0D981102A00F0EA8100F02EBF74
:10871000132A00F0218240F20B8231E21C2A00F081
:10872000B88209D8182A00F080821B2A00F09182B2
:10873000172A40F01B874DE2212A00F0D682222A18
:1087400000F0F2821D2A40F01187C2E2B32A00F045
:1087500039852CD8A82A00F05D8412D8A42A00F00C
:10876000918307D8A22A00F05183A32A00F06C83DA
:1087700000F0FCBEA62A00F0EB8340F2A18300F0DB
:108780002CBCAB2A00F09F8407D8A92A00F05F8494
:10879000AA2A00F07A8400F0E9BEAD2A00F0CE8467
:1087A000C0F0AF84AE2A00F0E78400F0DFBEBB2A41
:1087B00000F0018615D8B62A00F0708507D8B42AD3
:1087C00000F01E85B52A00F0278500F0CFBEB92A3B
:1087D00000F0AA8500F2C685B82A00F0878500F06F
:1087E000C5BECC2A00F071860AD8BF2A00F02A86BE
:1087F000C02A00F04986BC2A40F0B88600F008BEC6
:10880000D12A00F08C86D22A00F09E86CE2A40F033
:10881000AD8600F078BE38B92D212046FFF7BDFEA9
:108820000027306000F0A9BE012802D0002700F028
:10883000A4BE1A682D212046FFF760FE002700F035
:108840009CBE38B921212046FFF7A7FE2F46306095
:1088500000F093BE0128E9D11A6821212046FFF7D4
:108860004DFE002700F089BE38B927212046FFF7CA
:1088700094FE2F46306000F080BE0128D6D11A68E1
:1088800027212046FFF73AFE002700F076BE68B9A0
:1088900022212046FFF781FE10F4000318BF4FF09D
:1088A0007F43034333602F4600F067BE012DBDD1E7
:1088B000042700F062BE40B9C54B002753F82130B1
:1088C000D3F8A030336000F058BE0128AED1C04BC1
:1088D000204653F8212033682021002BB8BF5B428B
:1088E000C2F8A030FFF759FE074600289ED1326833
:1088F0002721002AB8BF52422046FFF7FFFD00F0B3
:108900003CBE38B926212046FFF747FE2F4630608F
:1089100000F033BE012889D11A6826212046FFF7CE
:10892000EDFD002700F029BE48B910212046FFF7D1
:1089300034FEC0F3042030602F4600F01EBE012834
:108940007FF474AF10212046FFF727FE336820F430
:10895000F8521B0203F4F8531A4310212046FFF784
:10896000CDFD002700F009BE48B910212046FFF7D1
:1089700014FE00F01F003060002700F0FEBD01284B
:108980007FF454AF10212046FFF707FE336820F034
:108990001F0203F01F031A4310212046FFF7AEFD0C
:1089A000002700F0EABD002880D135212046FFF7DE
:1089B000F4FDC0F3402030602F4600F0DEBD0028FB
:1089C0007FF474AF35212046FFF7E7FD10F0020F6A
:1089D0000CBF0123002333602F4600F0CEBD0028DA
:1089E0007FF464AF35212046FFF7D7FD00F001008A
:1089F00080F0010030602F4600F0BFBD48B934213F
:108A00002046FFF7CAFDC0F340003060002700F0A9
:108A1000B4BD01287FF40AAF34212046FFF7BDFD25
:108A200037683FB940F0020234212046FFF766FD67
:108A300000F0A3BD20F0020234212046FFF75EFDC6
:108A4000002700F09ABD48B934212046FFF7A5FD64
:108A500000F0010030602F4600F08FBD01287FF448
:108A6000E5AE34212046FFF798FD37683FB940F066
:108A7000010234212046FFF741FD00F07EBD20F0C9
:108A8000010234212046FFF739FD002700F075BDB3
:108A900038B934212046FFF780FD2F46306000F0C2
:108AA0006CBD01287FF4C2AE1A6834212046FFF75E
:108AB00025FD002700F061BD38B924212046FFF7CD
:108AC0006CFD0027306000F058BD01287FF4AEAE89
:108AD0001A6824212046FFF711FD002700F04DBD44
:108AE00038B925212046FFF758FD2F46306000F0A9
:108AF00044BD01287FF49AAE1A6825212046FFF76D
:108B0000FDFC002700F039BD38B928212046FFF7C9
:108B100044FD2F46306000F030BD01287FF486AE62
:108B20001A6828212046FFF7E9FC002700F025BD40
:108B300038B92A212046FFF730FD2F46306000F07B
:108B40001CBD01287FF472AE1A682A212046FFF767
:108B5000D5FC002700F011BD38B923212046FFF7CE
:108B60001CFD0027306000F008BD01287FF45EAED8
:108B70001A6823212046FFF7C1FC002700F0FDBC46
:108B800038B92B212046FFF708FD2F46306000F052
:108B9000F4BC01287FF44AAE1A682B212046FFF767
:108BA000ADFC002700F0E9BC38B92C212046FFF7C6
:108BB000F4FC2F46306000F0E0BC01287FF436AEB4
:108BC0001A682C212046FFF799FC002700F0D5BC3D
:108BD000785B002090B915212046FFF7DEFCC64BDC
:108BE00038B14FF08072B2FBF0F0984228BF1846BF
:108BF00000E018463060002700F0BFBC01287FF479
:108C000015AE1A68BC493AB14FF0807393FBF2F28B
:108C10008A42A8BF0A4600E00A4632601521204673
:108C2000FFF76CFC002700F0A8BC38B933212046C0
:108C3000FFF7B3FC0027306000F09FBC01287FF4F1
:108C4000F5AD1A6833212046FFF758FC002700F0E5
:108C500094BC48B96C212046FFF79FFCC0F3C0408C
:108C600030602F4600F089BC01287FF4DFAD6C2115
:108C70002046FFF792FC336820F40022DB0403F463
:108C800000231A436C212046FFF738FC002700F030
:108C900074BC48B96C212046FFF77FFCC0F38040CC
:108CA00030602F4600F069BC01287FF4BFAD6C2115
:108CB0002046FFF772FC336820F480229B0403F403
:108CC00080231A436C212046FFF718FC002700F090
:108CD00054BC00287FF4EAAD4FF423735C43874B08
:108CE00007461B59336000F048BC48B900212046B4
:108CF000FFF753FC00F001003060002700F03DBC9E
:108D000001287FF493AD00212046FFF746FC33682D
:108D100020F0010203F001031A4300212046FFF76F
:108D2000EDFB002700F029BC48B901462046FFF7BB
:108D300034FCC0F3400030602F4600F01EBC012818
:108D40007FF474AD00212046FFF727FC336820F044
:108D500002025B0003F002031A4300212046FFF7E2
:108D6000CDFB002700F009BC60B96C212046FFF75D
:108D700014FC4FF48073C0F3036043FA00F03060DA
:108D80002F46FAE301287FF451AD1B68102B1FD04A
:108D90000CDC022B18D003DC012B1FD108231FE0B1
:108DA000042B13D0082B19D1052319E0402B11D027
:108DB00003DC202B12D1032312E0802B0CD0B3F55F
:108DC000807F0BD100230BE0072309E0062307E097
:108DD000042305E0022303E0306002E04FF0FF339C
:108DE00033603368013300F0C3836C212046FFF702
:108DF000D4FB336820F070621B0603F070631A43E3
:108E00006C212046FFF77AFB0027B6E340B96C21BE
:108E10002046FFF7C2FBC0F3C13030600027ACE34F
:108E200001287FF403AD6C212046FFF7B6FB3368C1
:108E300020F4C032DB0303F4C0331A436C21204614
:108E4000FFF75CFB002798E340B96C212046FFF751
:108E5000A4FBC0F3803030602F468EE301287FF4FE
:108E6000E5AC6C212046FFF798FB336820F4804284
:108E70009B0303F480431A436C212046FFF73EFB1B
:108E800000277AE340B96C212046FFF786FBC0F348
:108E9000003030602F4670E301287FF4C7AC6C21AE
:108EA0002046FFF77AFB336820F480521B0303F45B
:108EB00080531A436C212046FFF720FB00275CE318
:108EC0006C212046FFF769FBD5B910F4804708D024
:108ED0006C212046FFF761FBC0F3C31030602F46C2
:108EE0004BE3C0F3021300F40060034314BF0823F4
:108EF0000023336041E300BFFFFF0F007C5B0020D5
:108F0000012D7FF493AC10F4804710D06C212046E3
:108F1000FFF743FB336820F4F062DB0103F4F063F6
:108F20001A436C212046FFF7E9FA002725E332684F
:108F300011074CBF40F4006020F40060120120F0E3
:108F40007000D2B202436C212046FFF7D7FA14E337
:108F50006C212046FFF721FBADB910F4804708D003
:108F60006C212046FFF719FBC0F302103060002788
:108F700003E3C0F3C31300F40060034314BF0823EA
:108F800000233360F9E2012D7FF450AC6C212046C0
:108F9000FFF703FB10F480474FF06C0120460ED022
:108FA000FFF7FBFA336820F070021B0103F0700337
:108FB0001A436C212046FFF7A1FA0027DDE2FFF7F4
:108FC000ECFA336820F4F062DB0103F4F0631A4337
:108FD0006C212046FFF792FACFE240B96C2120467F
:108FE000FFF7DBFA00F00F0030602F46C5E20128E2
:108FF0007FF41CAC6C212046FFF7CFFA336820F0D9
:109000000F0203F00F031A436C212046FFF776FA94
:109010000027B2E240B96D212046FFF7BEFAC0F347
:10902000C03030602F46A8E201287FF4FFAB6D21ED
:109030002046FFF7B2FA336820F40042DB039BB20C
:109040001A436D212046FFF759FA002795E240B9EF
:109050006D212046FFF7A1FAC0F3413030600027B0
:109060008BE201287FF4E2AB6D212046FFF795FAF1
:10907000336820F4C0425B0303F4C0431A436D21FC
:109080002046FFF73BFA002777E240B96D212046E2
:10909000FFF783FAC0F3032030602F466DE201280A
:1090A0007FF4C4AB6D212046FFF777FA336820F4D4
:1090B00070621B0203F470631A436D212046FFF7B0
:1090C0001DFA002759E240B96D212046FFF765FAE5
:1090D000C0F3411030602F464FE201287FF4A6AB69
:1090E0006D212046FFF759FA336820F060025B01DA
:1090F00003F060031A436D212046FFF7FFF90027B4
:109100003BE240B96D212046FFF747FA00F00F001F
:1091100030602F4631E201287FF488AB6D21204674
:10912000FFF73BFA336820F00F0203F00F031A43F6
:109130006D212046FFF7E2F900271EE240B96D21BC
:109140002046FFF72AFAC0F300603060002714E2DF
:1091500001287FF46BAB6D212046FFF71EFA3368C0
:1091600020F080721B0603F080731A436D212046A5
:10917000FFF7C4F9002700E280B96D212046FFF710
:109180000CFA001410F0400F00F07F0214BF6FF0D3
:109190007F030023134333602F46EEE101287FF461
:1091A00045AB6D212046FFF7F8F9336820F4FE0245
:1091B0001B0403F4FE031A436D212046FFF79EF9BA
:1091C0000027DAE140B96C212046FFF7E6F9C0F349
:1091D000404030602F46D0E101287FF427AB6C215E
:1091E0002046FFF7DAF9336820F400325B0403F419
:1091F00000331A436C212046FFF780F90027BCE1B9
:1092000000287FF453AB6F212046FFF7C6F9C0F367
:10921000044030600027B0E1D0B934212046FFF788
:10922000BCF9430511D514212046FFF7B6F9C04B10
:1092300038B14FF08072B2FBF0F0984228BF184668
:1092400000E018463060002797E135602F4694E132
:1092500001287FF4EBAA34212046FFF79EF93268FB
:1092600020F48060920202F480620243342120469E
:10927000FFF744F9326842B14FF0807393FBF2F28A
:109280009A4208BF6FF07F4201E06FF07F42326088
:1092900014212046FFF732F900276EE188B9142126
:1092A0002046FFF77AF9A24B38B14FF08072B2FB3B
:1092B000F0F0984228BF184600E0184630600027BA
:1092C0005BE101287FF4B2AA1A6842B14FF08073C3
:1092D00093FBF2F2964B9A42C8BF1A4600E0944ABA
:1092E00014212046FFF70AF9002746E140B96C2116
:1092F0002046FFF752F9C0F3403030602F463CE182
:1093000001287FF493AA6C212046FFF746F93368C1
:1093100020F400525B0303F400531A436C212046EF
:10932000FFF7ECF8002728E140B96C212046FFF751
:1093300034F9C0F30350306000271EE101287FF4A8
:1093400075AA6C212046FFF728F9336820F47002D3
:109350001B0503F470031A436C212046FFF7CEF877
:1093600000270AE188B913212046FFF716F9704B50
:1093700038B14FF08072B2FBF0F0984228BF184627
:1093800000E0184630600027F7E001287FF44EAA7D
:109390001A6867493AB14FF0807393FBF2F28A4240
:1093A000A8BF0A4600E00A46326013212046FFF7B4
:1093B000A5F80027E1E040B970212046FFF7EDF85D
:1093C000C0F3072030602F46D7E001287FF42EAA93
:1093D00070212046FFF7E1F8326820F47F40120246
:1093E00092B2024370212046FFF788F80021204600
:1093F000FFF7D3F8336820F00402002B14BF0423D6
:1094000000231A4300212046FFF778F80027B4E034
:1094100038B970212046FFF7C0F8C0B230602F463F
:10942000ABE001287FF402AA70212046FFF7B5F8CF
:10943000327820F0FF00024370212046FFF75EF8EB
:1094400000279AE040B970212046FFF7A6F8C0F344
:1094500001403060002790E001287FF4E7A91B68F5
:10946000032B00F2878070212046FFF796F83368BF
:1094700020F440321B0403F440331A437021204689
:10948000FFF73CF8002778E040B970212046FFF74D
:1094900084F8C0F3804030602F466EE001287FF4EE
:1094A000C5A91B68012B67D870212046FFF775F806
:1094B000336820F480229B0403F480231A43702134
:1094C0002046FFF71BF8002757E040B970212046DF
:1094D000FFF763F8C0F3015030602F464DE00128DC
:1094E0007FF4A4A970212046FFF757F8336820F4D1
:1094F00040121B0503F440131A4370212046FEF767
:10950000FDFF002739E000287FF4D0A96F21204615
:10951000FFF743F8C0F3090030602F462DE048B94B
:1095200039212046FFF739F80027306025E000BFD9
:10953000FFFF0F0001287FF479A91A68392120461E
:10954000FEF7DCFF002718E030B93A212046FFF78C
:1095500024F82F46306010E001287FF467A91A68CC
:109560003A212046FEF7CAFF002706E0042704E060
:10957000102702E0102700E010273846F8BD07B595
:10958000019229B9024601AB0120FFF77DF800E006
:10959000082003B05DF804FB10B4134604460846E7
:1095A00019B9224610BCFFF76FB8082010BC7047ED
:1095B00038B522210020FEF7F0FF18B90A4B1868D1
:1095C00006F06CF9094B0A4CDD68606A2B689B69F0
:1095D00098472B6820681B6998472B6860681B694F
:1095E0009847012038BD00BF785B0020286602083C
:1095F000001700202DE9F041544E554806F0E6F8DA
:10960000F568544C6B68002703F1C802A26003F5AB
:109610008072E26003F58E72226103F5B8722260F7
:1096200003F5C672626003F5F072626203F5FE72C2
:10963000A26203F5617203F1E400A26103F56872AE
:1096400003F56F73E3612B6822621B6960619847C1
:109650002B6820691B6998472B68E0681B6998474D
:109660002B68E0691B6998472B68206A1B6998473B
:109670002B68A069DB6898472B6820681B699847AE
:109680002B6860681B6998472B68A068DB6898475F
:109690002B68606ADB6898472B68A06ADB6898478C
:1096A0002B68A0699B69984732692B4B01261A6089
:1096B0006B68022003F537735360284B284A5969B9
:1096C0001160284A0E70C1F80422274A4F70C1F871
:1096D0000822264A1E741A62254ADA61254A9A61CE
:1096E000254A5A62254A9A63254A5A63254A9A624C
:1096F000254ADA62254A9A64254A5A64254A5A65F7
:10970000254A1A65254ADA64254A1A66254ADA6521
:109710003222DA604FF4F0729A60234A9A65FEF7BB
:109720008DFEA36A0222197C5A741868324608F02A
:10973000EFFC2B68A06A1D4C1B689847236898476C
:10974000A3683846BDE8F041184700BF2866020804
:109750007C5B002000170020085E002018390020E4
:10976000785B0020B1950108318401085985010812
:109770009985010895850108918501089995010849
:109780007F9501082385010869860108198501086C
:109790005986010819840108E5810108C58101087D
:1097A0003D840108D981010899830108B809002086
:1097B00018B9034B1B680B6070470820704700BF47
:1097C000145E0020014B00225A60704718390020B7
:1097D0000428F8B514464FD005D8022833D000F23B
:1097E0008F8038B104E0062871D069D3FC287AD084
:1097F0000420F8BD136833F0030240F0888013F0B2
:10980000010F444D444E03D0F3681B681B6906E00A
:10981000F76868683B68DB6898473B689B696868DD
:109820009847206810F0020404D0F36828681B6889
:109830001B6964E0F66828683368DB68984733681A
:1098400028689B6915E01468334B64B1DC68606874
:10985000236800F50670DB6898476068236800F5A8
:1098600006709B694BE0DB6858681B6800F5067062
:109870009B6898472046F8BD1668264D264B4EB18A
:10988000012E11D1DF6828693B68DB6898473B6887
:109890005B6906E0DF6828693B68DB6898473B68DE
:1098A0009B692869984709E0DE68286933681B6965
:1098B0009847336828691B6A9847064626601FE068
:1098C000154B144ADB6890691B681B6A05E0124B54
:1098D000104ADB68D0691B681B6A9847003018BFC4
:1098E000012020600CE014680A4D0B4B54B1DC6879
:1098F00028692368DB689847236828699B6998472B
:109900000020F8BDDB6828691B681B69B1E71020DF
:10991000F8BD00BF3817002028660208144B70B548
:10992000DD68144C2B68A0689B6998472B68E06839
:109930009B6898472B6820699B6898472B686069EB
:109940009B6898472B6820689B6898472B686068DD
:109950009B6898472B68A0699B6898472B68E069CB
:109960009B6898472B68A0689B68BDE870401847C3
:109970002866020838170020034B01461B68034A7B
:10998000002005F0D6BF00BF105E0020145E00204E
:10999000014B186806F005B8105E0020022804BFCD
:1099A0000B4B93F8D00020B90A4BDB681B685B694E
:1099B0000AE001280BD1064B93F8D030012B06D1D9
:1099C000044BDB681B689B69034A90681847704723
:1099D0001839002028660208381700202DE9F047C2
:1099E00088460446924699461A4D002155F8203083
:1099F00048F080009B689DF820709DF8246098478F
:109A000055F8243000219B685046984755F824307B
:109A100000219B684846984755F8243000219B68F0
:109A20003846984755F8243030469B6801219847BE
:109A3000094B49EA0A2953F8243047EA092708F074
:109A40007F0803EB880846EA0726C8F80460BDE8EB
:109A5000F08700BF0C5E0020105E002007B5D3B277
:109A60000193C2F307230093C2F30743120EFFF7DB
:109A7000B5FF03B05DF804FB0A4601460020FFF77E
:109A8000EDBF73B50D460646E0B9104C94F8203092
:109A900043B10F4B27211B68D3F8A020FFF7DEFF4F
:109AA00084F8206000242A462D210020FFF7D6FFED
:109AB000204601940094234622462021FFF78EFF82
:109AC000204600E0082002B070BD00BF381700201B
:109AD000105E002037B50D460446C0B90D4B01227B
:109AE00083F8202081EAE172A2EBE1722721FFF7DF
:109AF000B5FF002DACBF0123022301932046009443
:109B0000234622462021FFF769FF204600E0082077
:109B100003B030BD381700200021DBE74942D9E708
:109B2000D8E72C4A4FF4237370B503FB002301F0F0
:109B30007F04234493F80C320546DB0706D4264BFA
:109B400053F8203003EB8404606870BD234E00217D
:109B500056F8203020469B68984756F8253000215B
:109B60009B680846984756F8253000219B680846B0
:109B7000984756F8253000219B680846984756F8C4
:109B8000253001219B680020984756F82530002198
:109B90009B682046984756F8253000219B68084668
:109BA000984756F82530002104029B6808469847DC
:109BB00056F825300021204304029B680846984748
:109BC00056F82530204304029B6801210020984765
:109BD000204370BD145E0020105E00200C5E00204B
:109BE00010B50C4601460020FFF79BFF206010BD1A
:109BF00038B50C4621210546FFF793FF2168014443
